:020000040000FA
:080000000002040000000000F2
:020000040000FA
:10040000AF6C21000E7F22000E018800000000006A
:100410000C000700E0C529000100200011000700C2
:10042000000020000000E000020032000000020096
:100430000000000074B50200000000000040DA0077
:100440000000FE004440A900E04B21000000E00055
:100450000300320000002000A00188004440A800F2
:100460000000060091018800800078000000EB0089
:1004700015003700E280400032A0B4009101BA00BC
:10048000E280400032A0B4009102BA00E280400055
:1004900032A0B4000002EB00472BDE00F507B200EB
:1004A000602CE10004003A000059EB008301E900F0
:1004B000FDFF3E00040037006128E100010032002A
:1004C0000082EB00040007001101BA000200E00006
:1004D000E8FF3A00000006003159BA008301E90044
:1004E0000C0032002159BA008301E90008003200F3
:1004F0000400E00003003A00E280400032A0B400B3
:10050000F5FF370011D9BA008301E900FAFF3A007C
:100510008100E800E180400032A0B4000000060045
:1005200052D204000000000054D204000000000079
:1005300028D2040000000000BACF04000000000030
:1005400008D00400000000004ED0040000000000AD
:100550001670040000000000187004000000000085
:10056000247004000000000076AF040000000000CA
:1005700078AF040000000000E0AF040000000000BD
:10058000C0D40400000000004AD4040000000000B1
:1005900096D4040000000000F6A90400000000004A
:1005A00010AA0400000000002EAA040000000000B1
:1005B0004CAA04000000000052AA04000000000041
:1005C0006AAA040000000000B4AA040000000000B1
:1005D000CEAA040000000000F0AA04000000000001
:1005E00020AB0400000000005CAB04000000000031
:1005F0008CAB040000000000BEAB04000000000053
:10060000EEAB04000000000038AC04000000000065
:100610003EAC0400000000004AAC040000000000F2
:1006200056AC0400000000005EAA040000000000B8
:1006300086BA040000000000A4BA04000000000014
:10064000DEBA040000000000E2BA0400000000006E
:10065000EEBA040000000000FEBA04000000000032
:1006600048BB04000000000066BB0400000000005E
:10067000B0BB040000000000CEBB0400000000007E
:1006800018BC04000000000046BC0400000000008C
:10069000D6A5040000000000F0A504000000000042
:1006A0000EA60400000000002CA6040000000000BC
:1006B00032A60400000000003EA604000000000076
:1006C000E6A604000000000000A7040000000000EF
:1006D00030A704000000000062A704000000000032
:1006E00068A7040000000000E2A70400000000006A
:1006F0006AA704000000000076A7040000000000C4
:10070000A6A704000000000088A604000000000066
:100710000040DA000000FE00020AB900001BB90028
:100720000200B80081004200810043000000060082
:100730001004B100030035009001B10001003C003D
:100740001000050000000500800078001104B100D1
:10075000030035009101B10001003C000050A000F1
:10076000000006001004B100070035009001B10040
:10077000040034007000B100030035009001B100A6
:1007800001003C0010000500000005006900E100C8
:10079000040035006D00E100030034000002B100E8
:1007A0000100320000000500100005002002E200F8
:1007B00004003D002342AB00020032002302AB00E4
:1007C000FEFF32000040DA00FEFF37000A00FA00A8
:1007D00080017800E20F500028003E0030B2800017
:1007E000E10F500008003200802320000000E000EC
:1007F000050032000423200025232000462320008A
:100800008001780004003700042220002522200007
:100810004622200083222000144090000004E000C3
:10082000040035008009EB00144090000074A00023
:1008300010429800154090000028A30003003A00E1
:10084000154090000024A000904298008001EB0029
:1008500007003700154090000008A300FDFF32009C
:1008600063C078000000FB00000B78008301E80003
:10087000828F5100F7FF3A00080037003000200057
:10088000B0BF9F00C3BF9F00D1BF9F00E2BF9F00CA
:100890006A80570000C0DA006FB997000200780044
:1008A0000080FA00000006000A00FA001100200093
:1008B000B1BF9F00C0BF9F006A80570000C0DA0030
:1008C0004FB897000080FA00000006000A00FA0006
:1008D00051002000B1BF9F00C0BF9F006A80570039
:1008E00000C0DA005FB897000080FA000000060040
:1008F0000A00FA00881F7800800178000000E000FC
:1009000029003A0030B28000E10F500008003200A8
:10091000802320000000E0000500320004232000B6
:100920002523200067232000800178000400370081
:10093000042220002522200067222000832220009C
:10094000144090000004E000040035008009EB0032
:10095000144090000074A000104298000002EB00C8
:100960000C003700130A2000154478006140640031
:1009700002003A008301E900FBFF3A000402E800AC
:100980009541780061C061000500320017007800D1
:100990008058780004035100820F5200F1FF3A00A2
:1009A000060051000800370020002000A0BF9F0073
:1009B000B3BF9F00C1BF9F00D2BF9F006C80570094
:1009C00000C0DA005FB897004F0478000080FA009A
:1009D00000000600889FBE008004780040B28000BE
:1009E0000000E00003003A00100007000000E000F3
:1009F0000A00350040B280000900E00002003A0021
:100A00000004780006003700000478000900400068
:100A1000060007000000E00001003D000084EB003C
:100A2000080078004F04BE00000006008000780037
:100A30000000E00004003A00A064210040B28800F9
:100A400001017800060037000081EB00A06C210056
:100A5000808F500002003E0041B288000001EB0090
:100A600002007800000006006022B80006022000A4
:100A70000000D0008180D2000482D2008582D200A2
:100A80000000A0000202520083825A0003003100DD
:100A90000202420083824A000000A1000603E9002E
:100AA000F3FF3A0000000600889FBE008A9FBE0048
:100AB000010578000100E0000400350008003C005A
:100AC0000000E00020003200050037006000100048
:100AD000E080180002003B0001F02C001A003700F3
:100AE0000004BE006011B8006B0920000982CF002D
:100AF000020039000882CF000441B0006942520070
:100B00000E00320008003B00828171006101640028
:100B10008904D1000884D3008B05E8000442E80072
:100B2000F9FF3A00050037000804440089844C00AE
:100B30008B05E9000442E900FBFF3A005B02070075
:100B40000AF0A70001F0A0004F05BE004F04BE0050
:100B50000000060003F0A200889FBE008A9FBE002E
:100B60008C1F7800770207007E0233006450E1009A
:100B70004F0032006420E1005200320003826C001A
:100B800007003B000905D0000306D000820F540087
:100B90000C065D0002003900020032008901780075
:100BA000030678008582550004003D000003FD0027
:100BB0008103FD008502EA008B854200840F7200EC
:100BC00002003B0060001000E08018006011B800D7
:100BD0000005EB007A28E1000A00390006007800E1
:100BE000C75DDD00F707B200878075002D00370074
:100BF000828171000A017800610560008180D10066
:100C00000080D3008502E900F9FF3B0006044000A4
:100C10008784480002003B0060041400E0841C004C
:100C20000988A300070032008A8171008281710067
:100C3000610164008904D1000884D3008B05E800B9
:100C4000170037000978A30013003A000B00E000FA
:100C5000130034008B05E9000804440089844C002B
:100C60000A4474000978A3000D003A000B00E0006C
:100C7000070034008B05E9000804440089844C0017
:100C800001003A000B0020000978A300F7FF3200B2
:100C90000001EB0002003700828171000A01780038
:100CA000020207000CF0A70001F0A0003602370096
:100CB0006420E10002003A00838F6C0036023300AA
:100CC0000801BE000200BE002F0237000001EB0049
:100CD00034020700040032000200200003F8230061
:100CE00001F0A6009CFF0700000006000001BE0006
:100CF000530207000470A70003F0A10003F8A3004B
:100D000013003A006509B1001000320009003500F7
:100D10006928E100020035000100280000000500FC
:100D200000004000818048008502E900FCFF3A0095
:100D300000000600F88F4200050035008100D10058
:100D40000080D3008502E800FCFF3A0000000600A6
:100D50008000EB0000000500889FBE008A9FBE0057
:100D60008C1F7800F7010700FE01330003866C003A
:100D70006450E1002E0032006420E10033003200B4
:100D80006150E1002F0032006120E10031003200AB
:100D900085855500EB07B0000900200008042000FD
:100DA000050037000804440089844C000A00310023
:100DB0000603430087834B000001530081815B00E1
:100DC000F8FF33000203BE000800A000080444003E
:100DD00089844C00F6FF3900C639DD0083017300B9
:100DE00001003200130020008904D1000884D300E0
:100DF0000998A300050032000800A7000300A00026
:100E00008904D1000884D3008B05E8008904D1004F
:100E10000884D3000001EB000281D200A301070087
:100E200001F0A1000CF0A70001F0A000D6013700EE
:100E30006420E100D80132000801BE000200BE00BB
:100E4000F7FF37006120E100D30132006000B800F5
:100E5000F3FF37000000200001F82700F0FF370003
:100E6000040020000B023700889FBE008A9FBE004E
:100E70008C1F7800B3010700BA01330003866C00B1
:100E80006450E100240032006420E10027003200B9
:100E90006150E100220032006120E10021003200B7
:100EA0008B854200EB07B1000134B800003AB8006E
:100EB0000804420089844A00013AB8000030B800B2
:100EC0008880400009014A0004003300000040000F
:100ED00081804800020149008B05E900C909DD0055
:100EE000830170000100320013002000C814DE00EE
:100EF0004814DD004709DE001200B200C808DE0019
:100F0000088470006901070001F0A1000CF0A7003F
:100F100001F0A0009C0137006120E1009E01320039
:100F20000801BE000200BE00F7FF37006150E1007B
:100F3000FCFF3A00980137000001BE00C001070025
:100F40000470A70003F0A1006509B100160032008B
:100F50000D0035006828E10006003500F0FF2F0085
:100F6000F1FF27000300E00013003B000100280010
:100F70000000050000004000818048008502E90073
:100F8000FCFF3A0008003700F88F420002003C00E6
:100F90008000EB00000005008100D1000080D3003C
:100FA0008502E800FCFF3A000300E00002003B007D
:100FB00060001000E080180000000600AAFE070094
:100FC0000400BE0000000600889FBE008A9FBE008D
:100FD0008C1F78000205BE000004BE000006EB0076
:100FE000E00F5000E08F5800E00F5900E08F5900EB
:100FF00007003D006000B8006011B8000804500010
:10100000898458000A0559008B8559001C0020006E
:10101000E00F5200E08F5A00E00F5B00E08F5B00B2
:1010200002003D000F0007000C00A2000800BE00F7
:101030000A01BE00B20107000203BE000002BE00AA
:101040000C00E00001003200060007000400BE00B2
:101050000601BE004F0678004F05BE004F04BE00DB
:10106000000006006000B8006011B80004025000E3
:101070008582580006035900878359000000060046
:10108000881F7800000478005001BE004000BE00B8
:10109000040040008580480006014900878149001E
:1010A000009CBE000294BE000400E1000588E1003F
:1010B0000690E1000798E10002003100680044005A
:1010C0001008E8004F04780000000600F48747008D
:1010D000889FBE008A9FBE008C9FBE008E1F780036
:1010E0000205BE000004BE00D4B79F00E5B79F0014
:1010F000F6B79F0087BF9F000000EB00C0B79F00BE
:10110000B0B79F00A0B79F0090B79F0080B79F0027
:101110000D042000BFB097004FB0970000014000C1
:101120000000E0000F003D004F08DE0000007100ED
:10113000C0B79F009E00070001003D001200200084
:10114000A100070001003D0012002000A6000700DA
:10115000B1000700B60007000F004000C8FF0700FD
:10116000220037004F08DE0000067100CCB79F0058
:101170008F00070001003D001200200092000700D0
:1011800001003D001200200097000700A2000700A8
:101190000FB297009FB297002FB39700BFB397008D
:1011A000A90007000000520081805A0002015B0084
:1011B00083815B0080B79F0091B79F00A2B79F001B
:1011C000B3B79F000007EB009F0007000020E1007D
:1011D00001A8E10002B0E10003B8E1000100310024
:1011E0001E0020000E005600C0B79F004FB29700AF
:1011F0000400E0000700350010002000010020007E
:101200006011B80008047000898470000A0571003C
:101210008B8571008D06E900BEFF3A000400E000F6
:1012200003003D00820007000F00400094FF07000C
:101230004FA897000000E00004003A000FB49700A8
:101240009FB497002FB59700BFB597009400070093
:101250004F0778004F06BE004F05BE004F04BE008A
:101260004F01B10000000600881F78001800200020
:10127000881F780095FF07008F87E9004F047800EA
:1012800000000600801FEB0090FF07008F87E90039
:1012900000000600889FBE008A9FBE008C1F780059
:1012A0006E00070007003D0073000700E00F5B00C1
:1012B000E08F5B0007003D00320007000006EB00F6
:1012C000040037003400070002003D002A00070038
:1012D0001C00200072000700E3FF07000203BE00AD
:1012E0000002BE000C00E0000100320022000700F6
:1012F0000400BE000601BE004F0678004F05BE0088
:101300004F04BE0000000600889FBE008A9FBE00FA
:101310008C1F78005100070005003D0056000700B3
:10132000E00F5B00E08F5B0006003D00040037002B
:101330001900070003003D006000B8006011B8000C
:101340001000070056000700CEFF07000203BE0092
:101350000002BE000C00E0000100320006000700A1
:101360000400BE000601BE004F0678004F05BE0017
:101370004F04BE00000006006000B8006011B80015
:10138000000037000402500085825800060359000F
:1013900087835900000006000006EB00E00F5200B2
:1013A000E08F5A00E00F5B00E08F5B00000006005A
:1013B0000180400090B79F000001EB008FB09700C4
:1013C0000100E000000006000200700090B79F00DE
:1013D0000180400080B79F000001EB00FFA897004C
:1013E0000100E000000006000200700080B79F00CE
:1013F000018040006FAA9700CF20DE00010070003E
:10140000F0AF9F0004024200250007004F18DE00E5
:101410000002720000000600E4AF9F0008044400D0
:1014200089844C000A054D008B854D0000000600A4
:101430003FB29700CFB297005FB39700EFB397002A
:1014400000FE2F00000006003FB09700CFB09700CD
:101450005FB19700EFB19700000006000205BE00E3
:101460000004BE00E00F5000E08F5800E00F59006C
:10147000E08F5900000006006000B8006011B8005D
:1014800008045000898458000A0559008B855900CA
:101490001C002000E00F5200E08F5A000000060000
:1014A0000800BE000A01BE00000006008100200006
:1014B000618055000B003D000B00200061FE2F00F5
:1014C0000100E1001D0034008281710061016400AF
:1014D0008904D1000884D3000000E800FAFF3A0034
:1014E00071002000610064000300700002006000D1
:1014F0000900320061044400E0844C000988A50022
:10150000050032008B05E8006808E10002003A009F
:101510008904D1000884D300F20F20000258E100B2
:1015200005003D00C75DDD00F907B2008980750048
:1015300008007800000006000BF827008B007800F8
:10154000000005000004BE003D0007000003BE00CF
:101550000405BE000200BE0039000700844F75007C
:10156000000006000200BE006450E10005003600E5
:101570006420E100020036000968A30001003A007F
:101580000800BE000160A0004F0678004F05BE00B5
:101590004F04BE0000000600F0FF2F00F1FF2700FF
:1015A000F9FF3700889FBE008A9FBE000003BE007F
:1015B0002300070085057800828152000200200088
:1015C0006220E10004003A00F307B1000400350096
:1015D0007718E100040035000600BE001400370053
:1015E0006000B8000F003700F50F2000FAFF2F0051
:1015F0008502D1000A85D3008301E900FCFF3B008E
:101600008184620000046500890F7400F2FF3200DB
:101610008582EA000A85EA00818462000004650090
:10162000A2FF070007F0A70001F0A0000081EB0077
:101630000200E0004F05BE004F04BE00000006009F
:10164000C70ADE00F107B200F50FB2000800320051
:10165000E1CF4200020032000170A000240005002A
:10166000810F7000010032000408050044000500ED
:10167000810F700002003A00140005008502E900A5
:101680000000400081C04800FCFF3B000170A0004A
:1016900024000500889FBE008A9FBE00841F78003A
:1016A000A8FF07004F00780011003300F0FF2F0063
:1016B000838F6C0006003B00040565000A00A7004C
:1016C0000800370009F0A6001000200008003700CD
:1016D000820F5400838F5C0003003900100020004B
:1016E00001003E000000200009F0A7000000EA0011
:1016F0004F05BE004F04BE000000E00000000600E1
:10170000889FBE008A9FBE008C9FBE000404B80064
:101710000506B8008904460060854E000606B8003C
:101720000A054600E0854E000706B8008B05460016
:10173000040EB800890446000A854E00E0854D007D
:10174000050EB8000A0546008B854E00060EB8004F
:101750008B0546000416B8000A0546008B854E002E
:101760000516B8008B054600041EB8008B05460020
:101770000800BE000A01BE004F06BE004F05BE00B5
:101780004F04BE00000006000400FA00E0BF9F0006
:10179000E4815700812978000002EB000F00370038
:1017A0006FB89700904078007FB89700104078009D
:1017B0000402E80080CF5000040032008180FB006A
:1017C0000080FB0000805000070037006FB89700D2
:1017D0000000E800E0BF9F009309E800820F52007C
:1017E000EFFF3A000000EB000080FA000000060066
:1017F00010417800B141510003003A000000E800B8
:101800000204E000FAFF3A000300FB0000000600BB
:10181000800178000001780031407800005978009C
:101820000004E000FCFF3A0003007800000006001E
:101830008001EB0002003700817178008301E8002D
:10184000828F5100FCFF3A00000006000000FA0001
:10185000CFB8970068815700CC0007000080FA00DD
:1018600000000600810178000000E9000081EB0023
:10187000E50F500004003E0080004000A0622100FF
:101880006081780003B07800020078000000060054
:10189000000178000000E900E50F50000F003E0055
:1018A00080004000A0622100E08078000100E0009C
:1018B00002003A001000200069030700E18F400099
:1018C000060032000000EB00E18F500004003200FF
:1018D0000200780001000100000005000080EB001C
:1018E0000000060010002000E9FF070010002000A3
:1018F0005B0307000C00FA00889FBE00000478001C
:10190000CFB09700F0FF2700D0BF9F008004EB000E
:1019100099BF9F0088BF9F00A8BF9F00200C200098
:10192000B0BF9F0078815700708057009700070074
:101930000FB89700094878000FB8970008045000C6
:10194000080078004F04BE000080FA000000060086
:101950008002780080017800010037008301E800F0
:101960001304E000FDFF3A000002EB00820F52007A
:101970000600320064C07800805978000402E80054
:101980000004E00002003200F8FF37008049EB005D
:101990000500780000000600800078003004E000B8
:1019A000FEFF3A00010050000000E90000000600C0
:1019B000810178000002EB000B003700E440780062
:1019C0000104E000030032000402E80093CF50005D
:1019D000040032008180FB001380FB000080500077
:1019E000000006008301E800820F5200F3FF3A0076
:1019F000000005000C00FA00A0BF9F00C0BF9F00C0
:101A0000E5FF0700B0BF9F00F0BF9F00100C200053
:101A1000D0BF9F0074815700EFB097006C805700D3
:101A20003F0307000080FA00000006001041780024
:101A3000814F5100040032000000E8000204E00081
:101A4000FAFF3A000000EB0000000600889FBE008D
:101A50008A9FBE008000780000C2B30001003700FA
:101A6000890078008104780039447800804F540060
:101A7000FBFF3200E94F5400F9FF3200D0C2B3003F
:101A8000804F540004003A00194478008184E80033
:101A90001AC0B300060037000045EB00B0C2B30027
:101AA000804F540002003A00194478008184E80015
:101AB0006022B8000A003700A200200003002000C6
:101AC0000400BE0014FB07000B4144000281FB0030
:101AD000030020000002410081824900394478005F
:101AE0000880FB000BFD2F000B004000E90F5000A9
:101AF000F1FF36000A04E00002003200600212002A
:101B0000E0821A000400BE004F05BE004F04BE0074
:101B100000000600000378008002780002027800CE
:101B20008001EB00080037000402E90063C0780080
:101B3000805A78008301E8000004E00002003A00C7
:101B40008000EB0006003700828F5100F6FF3A005C
:101B5000FBFF37000040EB0080F07A008100E800D6
:101B6000848F5000FBFF3A0006007800000006005A
:101B70008001EB000200370061F079008301E8008A
:101B8000828F5100FCFF3A0000000600FE874700EC
:101B9000889FBE008A9FBE008C9FBE008E1F78006B
:101BA000F0B79F000107780082BF9F000000EB00A4
:101BB000A0B79F009F0237008006EB0050C2B30021
:101BC00080CF5000090032000100FB00FFB09700F9
:101BD000F4030700E10F400096023200AFB0970017
:101BE0008100E800A1B79F00920237009E40780074
:101BF000D0C2B30080CF50000C00320007003C0080
:101C00006D40500080CF50000A0032006B40400011
:101C100080CF50000E003A000800370000C3B30028
:101C200080CF50000A003A00060037000D30A000B7
:101C3000050037000D00A000030037000D10A000C4
:101C4000010037000D20A0000E07E800E7FF370075
:101C50000D18A300010032000D00A1000D38A300F3
:101C6000010032000D20A1000100FB0002FD2F0049
:101C700002004000E90F50000E003E000002EB00A1
:101C8000C4B79F0082017800CFB297006A28B900DC
:101C90001E01FB000001410003014100C2B79F008B
:101CA0005E00FB0003004000E90F50000B003E0007
:101CB000F5FF37000006EB00CCB79F00A0C2B300D1
:101CC00080CF500005003A000FB89700C0007800A0
:101CD00080BF9F00C1B79F000E07E8000001EB0026
:101CE000B2B79F00E0C2B3009E4F100018003A0048
:101CF0000DE0A0008E00E80064405000914F1000FD
:101D000002003200010778000C0037000FBA97007C
:101D1000C402780084BF9F00B5B79F000E87E8001B
:101D20000B0037003FB697006A60B9000000410021
:101D300003004000B0B79F000E07E8001E01FB0043
:101D400003FD2F0003004100E90F5000F5FF3600AE
:101D5000BE407800E1D79F00C0C6B30080CF5000DE
:101D6000220032000F003C006940500080CF50003C
:101D70007700320004003C000104E0003102320030
:101D80006B4050000F00370040C6B30080CF5000BA
:101D9000930032006540400080CF50008B003A0035
:101DA0008F00370030C7B30080CF50001A003200D8
:101DB00007003C006440500080CF5000110032000A
:101DC0000040E80080CF500080003A000F0037004C
:101DD00050C7B30080CF5000800032006340400005
:101DE00080CF500079003A00090037000000280039
:101DF0000D48A30001003A00000120008086760013
:101E0000D3FF37000D60A000750037000D50A00013
:101E10000D70A000720037008FB897004100780065
:101E200081BF9F00000478000000E00001003A003C
:101E3000A85D21008004EB00010037008104E80068
:101E400089007800088044001004E000FBFF3A009D
:101E50003FB197000200E00003003200890F5100FB
:101E600001003100820478000002EB00E4AF9F0023
:101E7000CFB29700898F52000200360009805200CD
:101E8000E0AF9F004368DE00E10660001B003A00FF
:101E90000D06780009003700FFB09700000220000F
:101EA00040030700E10F4000030032002FB097000D
:101EB0000000E800A0B79F000C06E800EFA897001C
:101EC000810F5600F4FF3A000081EB00E2AF9F0063
:101ED0000A003700880078003100FB000104780018
:101EE000FFB097002F030700E10F4000030032000E
:101EF0002FB297000402E800A4B79F000900E90090
:101F000080047800E10F4000F2FF3A000006EB0089
:101F10000D00E0000A003A00C6013700FFB097004C
:101F2000000220001F030700E10F40000300320001
:101F3000AFB297008502E800A5B79F000C06E80045
:101F40006FA89700800F5600F4FF3A00B9013700E0
:101F50008FB897004100780081BF9F00CF80DE00DE
:101F600001017800820178000205BE000004BE0075
:101F70000203BE000002BE004822DE00482EDD0043
:101F800004027600E4D79F000D48A3000A00320047
:101F90000404E00008003200E14F42000600320075
:101FA00071FD2F0001804700044878001840980018
:101FB0002900200002003700F0D79F001900200000
:101FC00072FD2F0002844700A1FF370064FD2F003F
:101FD00004844700190020009DFF37000D0CB3005A
:101FE0000D007800000CB20028003A000D00E0005F
:101FF00005003D008FBA97004505BE004504BE00B0
:1020000085BF9F00140037000D48A3000B0032006D
:102010000FBE97004C00BE008CBF9F004F89DE00B2
:10202000CF91DE000002BE00020378008203780038
:102030000605BE000404BE00070037008FB89700F5
:102040004100780081BF9F0000047800CFC4DE000B
:10205000090578008A057800E00F5400E08F5C00E5
:10206000E00F5D00E08F5D001F003D003D00B3000C
:102070006000B8006011B80008045000898458005E
:102080000A0559008B855900170037000D00E00044
:1020900005003D000FB997004205BE004204BE0096
:1020A00082BF9F00100037000D48A30007003200D8
:1020B0000FBA97004400BE0084BF9F006011B800B3
:1020C0000205BE000004BE00070037008FBA97006B
:1020D0004500780085BF9F000004780009002000BB
:1020E0000A0020000B0020003FB697000C00E00023
:1020F00007003A00E00F5400E08F5C00E00F5D0045
:10210000E08F5D0002003A0010002000B0B79F0091
:102110008D007800010CB200E1B79F0000042000A0
:10212000808F50003000320003003C000100E000CE
:102130000800320040003700000820006FB197000F
:10214000800F510014003200000C2000800F51005D
:1021500039003A0014C0B300A55321000B0037002A
:102160000400FB004300DD00050040005001BE00FC
:102170004000BE000040E10001C8E10002D0E100E3
:1021800003D8E1002B0039000442E800F44F52006C
:10219000F3FF3A0027003700000120000100200073
:1021A0006011B80014C0B3000040E10001C8E100B4
:1021B00002D0E10003D8E1001E00390045002000F4
:1021C0000000D0008180D2000281D2008381D20041
:1021D0008502E900FAFF3A000442E800F04F52009D
:1021E000F1FF3A00130037008000200001002000BA
:1021F0006011B80014C0B3000040E10001C8E10064
:1022000002D0E10003D8E1000A0039003C002000C0
:102210000000D0008180D2000281D2008381D200F0
:102220000C06E900FAFF3A000442E800F54F5200BC
:10223000F1FF3A00E4D79F00EFD097000100FB00C8
:102240003FB19700820F500002003D00E2D79F008F
:10225000040037003FB29700800F520001003D009C
:10226000B0B79F00CFB297000500E0000400320035
:1022700063806600020032008502E900C5B79F0056
:102280000DE8A3000B0032004FB697003FB0970057
:10229000800F560003003C008000EB00C1B79F0098
:1022A000040037004FB197003FB29700040151007E
:1022B000C2B79F00EFD297000500FB000006EB00BD
:1022C000DCAF9F00CFB09700808F50000200340039
:1022D00000805000D0AF9F000D28A30037003200CF
:1022E000E18066000D18A3000C003200D00220002F
:1022F0000100E00001003A000080E900FFB0970013
:1023000028020700E10F40000E0032002FB19700B5
:102310000201E800A2B79F000A0037000100E000B8
:1023200008003200FFB09700000220001D020700E5
:10233000E10F4000030032002FB297000402E800D2
:10234000A4B79F00DFAA97000500E0000F0032004D
:102350000006EB00FFB09700000320001102070009
:10236000E10F4000030032002FB097000000E800AA
:10237000A0B79F000C06E800DFA89700810F560069
:10238000F4FF3A000001EB00D2AF9F003FB297008C
:10239000C320DD00205321008080400091B79F00C2
:1023A0004220DD006400500080B79F006320B90028
:1023B000F0AF9F006306500084003700DFAA97004B
:1023C0000500E00011003200688066000F003A004E
:1023D00000067800FFB0970000022000F10107001E
:1023E000E10F4000030032002FB097000000E8002A
:1023F000A0B79F000C06E800DFA89700810F5600E9
:10240000F4FF3A000001EB00D2AF9F00E1806600CC
:102410000D18A3000C003200D00220000100E000E3
:1024200001003A000080E900FFB09700DD010700DD
:10243000E10F4000D5FF32002FB297000402E80000
:10244000A4B79F00D1FF37000100E000CFFF3200AA
:10245000FFB0970000022000D2010700E10F40000A
:10246000CAFF3200AFB297008502E800A5B79F000F
:10247000C6FF370000042000EFB09700808F5000A7
:102480003100320003003C000100E000080032008F
:102490003E003700000820006FB19700800F510008
:1024A00011003200000C2000800F510037003A006C
:1024B0001FB097003002BE002003BE000800BE001F
:1024C0000A01BE0068FB0700A400200005002000F0
:1024D0006033B8006BFB070004C3B3000442400044
:1024E000E4D79F0029003700155E2100D5B79F0073
:1024F0000D58A30002003A00205F2100D0B79F00D2
:1025000014002000050020006033B8008FB0970051
:102510008100E900050033000402D0008582D2006A
:102520000683D2008783D200F9FF37000800BE007F
:102530000A01BE004CFB07006F0060005FB197000E
:1025400062407800100037001400200005002000D1
:102550006033B8000C0078000000E900050033008B
:102560000402D0008582D2000683D2008783D20085
:10257000F9FF37000800BE000A01BE003AFB070061
:10258000674060000043B000E0D79F00EFD09700A5
:102590000100FB00FFB0970082010700E10F40003F
:1025A000030032002FB197000201E800A2B79F009C
:1025B0001FB297006802520094B79F008FB2970035
:1025C000E482520085B79F0063065600D0FF2F00BB
:1025D0003FB197000090B9007FAA97000000420029
:1025E00063005000800F5600A2FF3A000D38A30090
:1025F00010003200DFAA97000500E0000D00340053
:102600000006EB00FFB09700000220006501070004
:10261000E10F4000030032002FB097000000E800F7
:10262000A0B79F000C06E800DFA89700810F5600B6
:10263000F4FF3A00BE407800E1D79F000104E000BB
:102640005DFD3A002FB097004F0778004F06BE009F
:102650004F05BE004F04BE00EF01B10000000600B0
:102660000004780096010700080078004FF8070082
:10267000889FBE00000478008144780000FD2F0090
:1026800000004400E90F500002003E000001780005
:102690000D0037000800780025F807000000E00072
:1026A000030032000800780027F8070000047800D3
:1026B000080078002BF807000000E0000700320057
:1026C00090FA2F00000144000980FB00800F5100A8
:1026D00002003D000280FB0001003700F00F2000E7
:1026E0004F04BE0000000600881F7800E0B18000A3
:1026F000810107000004780024F807000000E000D2
:10270000FAFF3A00E10F440003003200E1B180001B
:1027100008007800AC0107004F04780000000600B4
:10272000EC874700889FBE008A9FBE008C9FBE003A
:102730008E1F780081BF9F0002077800E0B18800FB
:102740008046EB00040137008884FB000900780014
:102750000EF80700800078000000E0000200320060
:10276000E1FF0700FC00370050C2B300804F540067
:10277000F0003A000FBD970020C0B300C0EF9F00EB
:10278000D1EF9F0081EF9F000300370040C0B300EE
:10279000C0EF9F000FBD97000FB99700B2407800BF
:1027A00082BF9F008184FB0090C6B30080CF5000A1
:1027B0003500320017003E006640500080CF5000C8
:1027C000620032000C003E007740500080CF500085
:1027D0002800320006003E000104E0009B003200A9
:1027E000A0C2B30080CF50006E003A001D00370039
:1027F00080C5B3001600370040C6B30080CF50003C
:10280000210032006440400080CF500065003A0053
:102810001200370030C7B30080CF50001E003200D6
:1028200007003E006740500080CF5000110032008A
:102830006340400080CF50005A003A001400370037
:1028400050C7B30080CF50000F00320063404000FB
:1028500080CF500053003A006500370020C0B3001D
:10286000CBFF3700DFE897008140E800D1EF9F0001
:10287000C8FF37004FE9970080C0B300E24F510016
:10288000C3FF3A00C1FF3700ACC0B30059003700A6
:102890008CC0B3005700370093FF0700DFE89700B4
:1028A0000104E00002003A004E017800D2B79F0018
:1028B000E0B180001001070000047800E10F400043
:1028C000A20032008FEC9700120037000A85E80062
:1028D0008ABF9F00160037008FB897001100FB00D9
:1028E000800F5400F9FF32005FE997000204E00016
:1028F00003003A005FB0970008587800D0B79F00F7
:102900008944E9000A003200E0B18000FA000700C3
:10291000000478000800E800E10F500004003600D1
:102920000800780099F707000000E000EAFF320095
:10293000DFE897000104E00087003A008D46E800D8
:102940005FB1970001497800830037005FE8970086
:102950000004E00003003A008D46E800CE00780055
:10296000D1B79F00E0B18000E3000700E10F400015
:10297000760032005FE997000204E00003003A00AD
:10298000DFB0970080587800D1B79F000FE997001B
:102990000241E90082EF9F004240A9006E0034002E
:1029A000F0FF37000180FB0008FD2F000800400009
:1029B000E90F50005F003E000A0078001F01070089
:1029C00080EF9F0088007800030037000FB8970061
:1029D0000000E80080BF9F000FB997001200FB00C5
:1029E00001004000E90F5000F8FF360069FF370092
:1029F0000CC1B3003CFF0700E0B18000BE0007003F
:102A0000000578000040EB00E0EF9F00D0022000BE
:102A1000800F550005003A00E0B18000B6000700C5
:102A20000005780011C0B300E1EF9F008C407800F2
:102A30000A0078000EFF0700E14F40000A003A004C
:102A4000E1B180000A007800DF0007000D04E0001B
:102A50004B003A00E0B18000300090000048A30035
:102A600043003200480037008FED97006044B80003
:102A70000C81FB00030020000800BE0026F70700C1
:102A80000004BE008C4078000A007800F8FE0700C1
:102A90000080FB00010020000804400089844800F9
:102AA0008B45E90007003200E0B18000920007008A
:102AB000000578008C407800EDFE0700E14F4000F3
:102AC000EBFF3A008C4078000A007800E8FE07002F
:102AD000E14F400003003A00E1B180000A007800B5
:102AE000B90007006FE997000204E000020032001D
:102AF00060041400E0841C005FE897000004E0001C
:102B000015003A008D46E800CFE89700E4CF50006A
:102B100003003A004E0078000888BE000E0037001F
:102B20000E81E9000207780012007800080878009A
:102B300009003700E0B180006F000700808F54006B
:102B400005003200E10F40000B003A000D04E000E8
:102B50000D0032000A0037008FB89700314478002A
:102B600081BF9F000804E000F7FE3A000400370030
:102B70000000EB0005003700E1B180009200070083
:102B80000D80FB00010037000080EB004F0778004C
:102B90004F06BE004F05BE004F04BE00CF00B1007F
:102BA00000000600889FBE00000178000104780044
:102BB000B10090000118A3003D0032000198A3006D
:102BC00003003A00180090000000E00038003A00CE
:102BD0000190A0003104980082047800F90FB2003F
:102BE000180090000000E00002003A002800900069
:102BF000000C7800EA8F540006003A00380090007C
:102C00000078A30003003A0088007800D00020007C
:102C1000E4FF07009800900058009000808F50005B
:102C20000B0032000100E800100498001800780042
:102C300009587800000C780011C0B300A06321008F
:102C400001487800EA8F540006003200190037006E
:102C500088007800094078009C0007008004780014
:102C600014003700380090000088A30011003200E3
:102C700018019000A800900048009000D3F60700CB
:102C800098009000810F500004003200380090003E
:102C90000003B300300498008084EB000000EB00D8
:102CA0001004980028009000000C78000100370004
:102CB0008084EB00090078004F04BE00000006008D
:102CC000881F7800F0B180000000E00001003200B1
:102CD000000001006860210008007800BE000700C5
:102CE0006C044400A0622100800F5400FAFF3A00F7
:102CF0004F04780000000600881F78000004780068
:102D0000B00090000148A30007003A000108A300AA
:102D1000050032000198A300080032001000900066
:102D20000000E00005003200380090000040A000E4
:102D3000300498008080EB00200037000190A10053
:102D400031049800180090000000E00006003400F4
:102D50000000E9001004980018007800B080FB0023
:102D6000000C780006003700380090000068A300CF
:102D7000EDFF3A0008007800CF00070080007800DF
:102D8000380090000078A3000C003A00FA8F500041
:102D900008003A00280090000000E000E2FF320046
:102DA000180090000000E80010049800180CE900DA
:102DB000DDFF3700ED8F5000E2FF320001007800A8
:102DC0004F0478000000060080017800E10F400009
:102DD00017003200310090000008A30014003200F8
:102DE0000098A30012003A00210290000400E000C5
:102DF0000F0032001101900051009000800F51002F
:102E00000B00320011007800840F500002003A00DD
:102E10008008E800020037000200E80090009800F7
:102E20001100E900800878000348780001003700AD
:102E30008081EB00030078000000060000017800AC
:102E400000C2B300010037000201E80092407800A0
:102E500080CF5000FCFF3200E9CF5000FAFF320073
:102E6000D0C2B30080CF500003003A000201E80056
:102E700014C0B300050037000042EB00B0C2B3003D
:102E800080CF500001003A000201E8008000EB0012
:102E900005FD2F00040037006A08B90000804100DA
:102EA000850040000201E8009201FB00058041001E
:102EB000E90F5000F8FF36000404E0000100320082
:102EC0008100EA0001007800000006000200FA001C
:102ED000889FBE00A0FF9F0001047800B100900011
:102EE000810478000904B200020032000000FB00F7
:102EF000360037000118A30005003A000103B300B3
:102F000031049800190498000080EB002F0037006E
:102F1000580090000000E00006003A0048009000D1
:102F200012002000E680570028F6070019049800D8
:102F300024003700280090000000E00008003A005C
:102F40006063210020049800000C7800200020001D
:102F500050049800100498000130A000310498003B
:102F600018019000A80090004800900017F6070094
:102F700028009000000C78000080EB0010049800FE
:102F800018007800AFF8970001587800000C78001E
:102F90002FF89700EA4F50000A003A0038009000DE
:102FA0000088A3000700320018019000A8009000DC
:102FB0004800900005F6070019049800A80090004A
:102FC000010C7800AFF897000100FB004F04BE0031
:102FD0000080FA0000000600889FBE008A1F78006B
:102FE000000478003000900063006000240032008C
:102FF000080078007E0007003805900080EF2F0061
:103000000000650030049800280090000000E000F7
:1030100004003200E804650002003A00AD00070039
:1030200029049800480090001FF60700E10F4000B7
:1030300013003200B80090000102B20010003A0004
:103040000AC8A3001800320010B280000000E0009F
:10305000150032000001780081047800012A200068
:1030600012289000880F5000070032004205B0007F
:103070004905B000818F54000B003200F8FF370083
:103080000080EB0009003700020078000FF607000F
:1030900010B28000090040008000EB001128980069
:1030A00001007800010037000000EB004F057800B8
:1030B0004F04BE00000006000200FA00889FBE0018
:1030C0008A1F7800000478000000EB0010049800CC
:1030D000380090008080EB000008A3003F00320021
:1030E000A06321001004E00010003200696021009C
:1030F000CA6021001A0078006C0545002010B2005B
:1031000021102000810F500002003A0009007800D1
:1031100037000700EC844400A0622100808F540037
:10312000F4FF3A00A06321000048EB004800900043
:10313000580190000200E0000D003A0012049800CF
:1031400012002000E8805700E9F50700E10F500069
:1031500003003A000FF897008080FB001F00370043
:10316000380090000040A0003004980012003700A2
:10317000A8009000DEF50700100498000000E000B1
:1031800003003200E10F40000D003A000300370059
:10319000380090000040A000020037003800900086
:1031A0000003B30030049800A8009000010C7800E0
:1031B0000000EB00100498008080EB00070037004F
:1031C000A8009000010C78000000E90010049800AD
:1031D00001007800B080FB00000C7800010078004E
:1031E0004F0578004F04BE000080FA000000060082
:1031F000881F780000047800300090000008A300C9
:1032000007003200800078000120B20004003A007C
:1032100011049800A8009000010C780017003700F6
:103220000018A300190032000098A3001700320014
:10323000A80090000100E000140032001801900086
:103240000200E00011003200480090005FF5070026
:1032500098009000810F5000030032003800900069
:103260000003B300300498000000EB001004980045
:1032700028009000000C7800380090000058A3004F
:10328000020032000080EB00010037000000EB007C
:103290004F0478000000060001B280000100E00049
:1032A000030032001100780000B2880003003700EC
:1032B00020002000C7F5070080007800E18F400063
:1032C00002003A00906E260020B2880001007800CB
:1032D0000000060001B280000108780000B28800FA
:0432E00000000600E4
:020000040000FA
:0200000401F009
:04000C00FBFF0000F6
:020000040000FA
:0200000401F009
:04001000FDFF0000F0
:020000040000FA
:0200000401F009
:040014007FFF00006A
:020000040000FA
:1000080088030000A6B3000076B300008EB300009A
:10001800BEB30000D6B300008803000088030000C8
:100028008803000080C100008803000086D5000016
:10003800880300008803000088030000880300008C
:1000480006B400008803000088030000D2D1000035
:10005800880300008803000088030000880300006C
:10006800880300008803000088030000880300005C
:10007800880300008803000088030000880300004C
:10008800880300008803000088030000FABE00000F
:10009800B6BF000088030000FED3000088030000FC
:1000A800880300008803000088030000880300001C
:1000B800880300008803000088030000880300000C
:1000C80088030000880300008803000088030000FC
:1000D8008803000088030000EEB3000088030000D6
:1000E80088030000880300008803000088030000DC
:1000F80088030000880300008803000088030000CC
:1001080088030000880300008803000088030000BB
:1001180088030000880300008803000088030000AB
:10012800880300008803000088030000880300009B
:10013800880300008803000088030000880300008B
:10014800880300008803000088030000880300007B
:10015800880300008803000088030000880300006B
:10016800880300008803000088030000880300005B
:10017800880300008803000088030000880300004B
:10018800880300008803000088030000880300003B
:10019800880300008803000088030000880300002B
:1001A800880300008803000088030000880300001B
:1001B800880300008803000088030000880300000B
:1001C80088030000880300008803000088030000FB
:1001D80088030000880300008803000088030000EB
:1001E80088030000880300008803000088030000DB
:0801F8008803000088030000E9
:020000040000FA
:1002080088030000A6B3000076B300008EB3000098
:10021800BEB30000D6B300008803000088030000C6
:100228008803000080C100008803000086D5000014
:10023800880300008803000088030000880300008A
:1002480006B400008803000088030000D2D1000033
:10025800880300008803000088030000880300006A
:10026800880300008803000088030000880300005A
:10027800880300008803000088030000880300004A
:10028800880300008803000088030000FABE00000D
:10029800B6BF000088030000FED3000088030000FA
:1002A800880300008803000088030000880300001A
:1002B800880300008803000088030000880300000A
:1002C80088030000880300008803000088030000FA
:1002D8008803000088030000EEB3000088030000D4
:1002E80088030000880300008803000088030000DA
:1002F80088030000880300008803000088030000CA
:1003080088030000880300008803000088030000B9
:1003180088030000880300008803000088030000A9
:100328008803000088030000880300008803000099
:100338008803000088030000880300008803000089
:100348008803000088030000880300008803000079
:100358008803000088030000880300008803000069
:100368008803000088030000880300008803000059
:100378008803000088030000880300008803000049
:100388008803000088030000880300008803000039
:100398008803000088030000880300008803000029
:1003A8008803000088030000880300008803000019
:1003B8008803000088030000880300008803000009
:1003C80088030000880300008803000088030000F9
:1003D80088030000880300008803000088030000E9
:1003E80088030000880300008803000088030000D9
:0803F8008803000088030000E7
:020000040000FA
:1032E40074650000787400002F7000006C610000A9
:1032F400696E00000074000065780000742F0000FF
:10330400687400006D6C00000074000065780000B3
:10331400742F0000786D00006C00000074650000DC
:10332400787400002F6300007373000000690000CC
:103334006D610000676500002F670000696600008A
:10334400006900006D610000676500002F700000D7
:103354006E670000006900006D6100006765000091
:103364002F6A0000706500006700000061700000B3
:10337400706C00006963000061740000696F0000F4
:103384006E2F00006A610000766100002D76000057
:103394006D00000061750000646900006F2F00007B
:1033A400782D0000776100007665000000000000C1
:1033B400729900007D9900007D9900007D990000BC
:1033C400879900009099000099990000A399000042
:1033D400AD990000B8990000CC990000D99900007B
:1033E4000D0A00000048000054540000502F000053
:1033F400312E000031200000323000003020000067
:103404004F4B00000D0A0000436F00006E6E000079
:1034140065630000746900006F6E00003A200000CC
:10342400636C00006F730000650D00000A0000006B
:1034340048540000545000002F3100002E31000089
:10344400203400003030000020420000616400009D
:10345400205200006571000075650000737400005F
:103464000D0A0000436F00006E6E000065630000EB
:10347400746900006F6E00003A200000636C000065
:103484006F730000650D00000A0D00000A3400008F
:10349400303000002042000061640000205200002F
:1034A4006571000075650000737400003A20000027
:1034B400636100006E270000742000006861000052
:1034C4006E6400006C650000204300006F6E000015
:1034D400746500006E7400002D4C0000656E0000E1
:1034E40067740000680D00000A00000048540000E2
:1034F400545000002F3100002E3100002034000011
:1035040030310000205500006E6100007574000029
:10351400686F0000726900007A650000640D0000A5
:103524000A570000575700002D4100007574000031
:10353400686500006E740000696300006174000037
:10354400653A0000204200006173000069630000D6
:1035540020720000656100006C6D00003D220000D7
:10356400507200006F740000656300007465000011
:10357400642200000D0A0000436F00006E6E00001C
:1035840065630000746900006F6E00003A2000005B
:10359400636C00006F730000650D00000A0D0000ED
:1035A4000A34000030310000205500006E61000034
:1035B40075740000686F0000726900007A6500008D
:1035C400643A00002050000061730000737700002B
:1035D4006F720000642000007265000071750000C5
:1035E40069720000656400000D0A000000480000D4
:1035F40054540000502F0000312E000031200000F0
:1036040034300000342000004E6F000074200000AD
:10361400666F0000756E0000640D00000A43000030
:103624006F6E00006E65000063740000696F000037
:103634006E3A0000206300006C6F000073650000A8
:103644000D0A0000436F00006E740000656E0000F8
:10365400742D000054790000706500003A200000C9
:1036640074650000787400002F680000746D000019
:103674006C0D00000A0D00000A3400003034000014
:103684003A200000466900006C650000206E0000CE
:103694006F740000206600006F7500006E64000007
:1036A4003C620000723E000055730000652000007B
:1036B4003C6100002068000072650000663D000067
:1036C400222F0000757000006C6F00006164000020
:1036D400223E00004D5000004653000020550000DB
:1036E400706C00006F610000643C00002F610000FA
:1036F4003E200000746F000020700000726F000014
:1037040067720000616D00002077000065620000B0
:103714002070000061670000657300000D0A00005E
:103724000048000054540000502F0000312E0000C7
:1037340031200000343100003420000052650000C4
:103744007175000065730000742D0000555200006F
:1037540049200000546F00006F2000004C6F0000EF
:103764006E6700000D0A0000436F00006E6E0000DB
:1037740065630000746900006F6E00003A20000069
:10378400636C00006F730000650D00000A0D0000FB
:103794000A3400003134000020520000657100003A
:1037A40075650000737400002D5500005249000037
:1037B400205400006F6F0000204C00006F6E00006A
:1037C400673A00002042000075660000666500004C
:1037D400722000006F76000065720000666C0000C5
:1037E4006F770000206400006574000065630000CA
:1037F40074650000640D00000A00000048540000D5
:10380400545000002F3100002E31000020350000FC
:1038140030300000204900006E7400006572000022
:103824006E6100006C200000536500007276000099
:103834006572000020450000727200006F72000083
:103844000D0A0000436F00006E6E00006563000007
:10385400746900006F6E00003A200000636C000081
:103864006F730000650D00000A0D00000A350000AA
:1038740030300000204900006E74000065720000C2
:103884006E6100006C200000536500007276000039
:103894006572000020450000727200006F72000023
:1038A4003A20000045780000706500006374000051
:1038B4006564000020640000617400006120000061
:1038C4006E6F0000742000007072000065730000C9
:1038D400656E0000740D00000A00000048540000EA
:1038E400545000002F3100002E310000203500001C
:1038F40030310000204E00006F74000020490000A9
:103904006D7000006C6500006D6500006E74000051
:10391400656400000D0A0000436F00006E6E000035
:1039240065630000746900006F6E00003A200000B7
:10393400636C00006F730000650D00000A0D000049
:103944000A35000030310000204E00006F74000082
:10395400204900006D7000006C6500006D6500007A
:103964006E740000656400003A2000004F6E000091
:103974006C790000204700004554000020610000DD
:103984006E640000205000004F53000054200000DB
:1039940073750000707000006F72000074650000A1
:1039A400640D00000A000000485400005450000058
:1039B4002F3100002E310000203200003030000092
:1039C400204F00004B0D00000A4300006F6E000002
:1039D4006E65000063740000696F00006E3A0000B9
:1039E400206300006C6F0000736500000D0A000086
:1039F400436F00006E740000656E0000742D0000BB
:103A040054790000706500003A20000074650000DD
:103A1400787400002F680000746D00006C0D0000C5
:103A24000A0D00000A3C0000687400006D6C000080
:103A34003E3C0000626F00006479000020730000C7
:103A4400747900006C6500003D2200006D61000087
:103A540072670000696E00003A31000030300000E7
:103A640070780000223E00003C6600006F72000087
:103A74006D2000006D650000746800006F64000034
:103A84003D7000006F73000074200000616300004B
:103A9400746900006F6E00003D2200002F75000065
:103AA400706C00006F61000064220000206500005B
:103AB4006E63000074790000706500003D22000010
:103AC4006D7500006C740000697000006172000084
:103AD400742F0000666F0000726D00002D640000FA
:103AE40061740000612200003E3C0000623E000060
:103AF4004D50000046530000204900006D61000055
:103B04006765000020550000706C00006F610000C4
:103B1400643C00002F6200003E3C0000703E000048
:103B24003C6900006E700000757400002074000091
:103B340079700000653D0000666900006C65000056
:103B4400206E0000616D0000653D000069200000EA
:103B5400736900007A6500003D340000303E0000C7
:103B6400202600006E620000737000003B200000FD
:103B74003C6900006E700000757400002074000041
:103B840079700000653D000073750000626D0000EF
:103B94006974000020760000616C00007565000007
:103BA4003D220000557000006C6F0000616400004D
:103BB400223E00003C2F0000666F0000726D000082
:103BC4003E3C00002F6200006F640000793E00005C
:103BD4003C2F0000687400006D6C00003E00000083
:103BE40048540000545000002F3100002E310000D2
:103BF4002032000030300000204F00004B0D000048
:103C04000A4300006F6E00006E65000063740000DC
:103C1400696F00006E3A0000206300006C6F0000C2
:103C2400736500000D0A0000436F00006E7400000D
:103C3400656E0000742D000054790000706500006A
:103C44003A20000074650000787400002F680000BA
:103C5400746D00006C0D00000A0D00000A3C0000A9
:103C6400687400006D6C00003E3C0000626F000050
:103C74006479000020730000747900006C65000012
:103C84003D2200006D61000072670000696E000053
:103C94003A3100003030000070780000223E00000D
:103CA4003C6200003E4D00005046000053200000DE
:103CB400557000006461000074650000205300002A
:103CC400756300006365000073730000667500008F
:103CD4006C3C00002F6200003E3C0000703E00007F
:103CE4003C6100002068000072650000663D000031
:103CF400222F0000223E000053690000746500007A
:103D0400206D0000616900006E20000070610000F9
:103D1400676500003C2F0000613E00003C2F00005E
:103D2400626F0000647900003E3C00002F680000D0
:103D3400746D00006C3E0000004800005454000004
:103D4400502F0000312E00003120000035300000DB
:103D540030200000496E000074650000726E00009F
:103D6400616C00002053000065720000766500005D
:103D74007220000045720000726F0000720D000096
:103D84000A4300006F6E00006E650000637400005B
:103D9400696F00006E3A0000206300006C6F000041
:103DA400736500000D0A0000436F00006E7400008C
:103DB400656E0000742D00005479000070650000E9
:103DC4003A20000074650000787400002F68000039
:103DD400746D00006C0D00000A0D00000A3C000028
:103DE400687400006D6C00003E3C0000626F0000CF
:103DF4006479000020730000747900006C65000091
:103E04003D2200006D61000072670000696E0000D1
:103E14003A3100003030000070780000223E00008B
:103E24003C6200003E4D000050460000532000005C
:103E3400496D00006167000065200000436F0000C9
:103E44007272000075700000742000006F72000030
:103E540020570000726F00006E67000020560000BB
:103E640065720000736900006F6E00003C2F000053
:103E7400623E00003C7000003E3C000061200000F7
:103E840068720000656600003D2200002F75000086
:103E9400706C00006F610000642200003E5400005A
:103EA400727900002061000067610000696E000003
:103EB4003F3C00002F6100003E3C00002F620000E8
:103EC4006F640000793E00003C2F0000687400001D
:103ED4006D6C00003E000000485400005450000087
:103EE4002F3100002E31000020330000303200005A
:103EF400204600006F7500006E6400000D0A00008B
:103F0400436F00006E6E000065630000746900007A
:103F14006F6E00003A200000636C00006F730000B5
:103F2400650D00000A4C00006F630000617400001E
:103F3400696F00006E3A0000200000004854000041
:103F4400545000002F3100002E31000020340000B6
:103F540030330000204600006F72000062690000E8
:103F640064640000656E00000D0A0000436F0000E9
:103F74006E6E000065630000746900006F6E0000DF
:103F84003A200000636C00006F730000650D0000B0
:103F94000A0D00000A3400003033000020460000FF
:103FA4006F7200006269000064640000656E0000C6
:103FB4003A200000535300004C20000052650000DA
:103FC400717500006972000065640000202D000016
:103FD4002075000073650000204800005454000060
:103FE400505300000D0A000000000000F599000085
:103FF400F59900001A9A0000789A0000F99A0000D6
:10400400939B0000009C0000709C0000D69C000064
:10401400D9990000F29D00009F9E00006E9F000051
:10402400A09F0000436F00006F6B000069650000F3
:104034003A00000041750000746800006F720000CF
:10404400697A000061740000696F00006E3A000034
:10405400004300006F6E0000746500006E74000081
:104064002D4C0000656E000067740000683A000083
:104074000000000014A000001CA000002BA0000001
:104084007478000074000000687400006D00000083
:10409400687400006D6C0000006300006769000034
:1040A400007800006D6C0000006300007373000072
:1040B4000067000069660000007000006E67000081
:1040C400006A000070670000006300006C6100007B
:1040D400007700006176000000000000000000008E
:1040E4000000000042A0000046A000004AA000001A
:1040F4004FA0000053A0000057A000005BA00000E8
:104104005FA0000063A0000067A000006BA0000097
:104114006FA0000068650000616400006572000023
:104124002E6900006E630000006600006F6F0000DF
:1041340074650000722E0000696E000063000000C8
:10414400214400004546000000470000455400009B
:10415400005000004F530000540000007570000030
:104164006C6F000061640000006600006F63000073
:1041740075730000657200002E680000746D000005
:10418400000D00000A0D00000A0000000D0A0000E6
:104194000D0A00004D5000004653000002010000CB
:1041A400000D00000A0D00000A3300003034000046
:1041B400205200006564000069720000656300001D
:1041C400743A000020000000436F00006E74000089
:1041D400656E0000742D00005479000070650000C5
:1041E4003A200000004300006F6E00007465000078
:1041F4006E7400002D4500006E6300006F640000C3
:10420400696E0000673A0000206700007A690000C8
:10421400700D00000A0000004361000063680000A4
:10422400652D0000436F00006E740000726F000083
:104234006C3A0000200000006E6F00002D63000047
:104244006163000068650000006D00006178000093
:104254002D610000676500003D000000363000005D
:104264003000000053650000742D0000436F00000F
:104274006F6B0000696500003A2000000000000038
:10428400000000000000000000000000000000002A
:10429400000000000000000000000000000000001A
:1042A400000000000000000000000000000000000A
:1042B40000000000000000000000000000000000FA
:1042C40000000000000000000000000000000000EA
:1042D40000000000000000000000000000000000DA
:1042E40000000000000000000000000000000000CA
:1042F40000000000000000000000000000000000BA
:1043040000000000000000000000000000000000A9
:104314000000000000000000000000000000000099
:104324000000000000000000000000000000000089
:104334000000000000000000000000000000000079
:104344000000000000000000000000000000000069
:104354000000000000000000000000000000000059
:104364000000000000000000000000000000000049
:104374000000000000000000000000000000000039
:104384000000000000000000000000000000000029
:104394000000000000000000000000000000000019
:1043A4000000000000000000000000000000000009
:1043B40000000000000000000000000000000000F9
:1043C40000000000000000000000000000000000E9
:1043D40000000000000000000000000000000000D9
:1043E40000000000000000000000000000000000C9
:1043F40000000000000000000000000000000000B9
:1044040000000000000000000000000000000000A8
:104414000000000000000000000000000000000098
:104424004375000072720000546500006D70000056
:10443400203D000020250000730000004E6F0000A6
:1044440020500000726F000062650000004300000D
:104454007572000072530000746500007020000043
:104464003D200000256C0000750000005461000030
:10447400726700005374000065700000203D000066
:10448400202500006C75000000490000734D0000F9
:104494006F760000696E0000672000003D20000078
:1044A4002575000000490000734800006F6D00008E
:1044B400696E0000672000003D20000025750000A3
:1044C4000049000073200000486F00006D65000083
:1044D400642000003D200000257500000054000009
:1044E400656D000070500000726F000062200000D3
:1044F4003D2000002575000000520000656D00009D
:104504006F740000654900004F2000003D2000004A
:10451400257500000048000043530000746100004A
:1045240074750000732000003D2000002575000014
:104534000000000000000000000000000000000077
:104544000000000000000000000000000000000067
:104554000000000000000000000000000000000057
:104564000000000000000000000000000000000047
:104574000000000000000000000000000000000037
:104584000000000000000000000000000000000027
:104594000000000000000000000000000000000017
:1045A4000000000000000000000000000000000007
:1045B40000000000000000000000000000000000F7
:1045C40000000000000000000000000000000000E7
:1045D40000000000000000000000000000000000D7
:1045E40000000000000000000000000000000000C7
:1045F40000000000000000000000000000000000B7
:1046040000000000000000000000000000000000A6
:104614000000000000000000000000000000000096
:104624000000000000000000000000000000000086
:104634000000000000000000000000000000000076
:104644000000000000000000000000000000000066
:104654000000000000000000000000000000000056
:104664000000000000000000000000000000000046
:104674000000000000000000000000000000000036
:104684000000000000000000000000000000000026
:104694000000000000000000000000000000000016
:1046A4000000000000000000000000000000000006
:1046B40000000000000000000000000000000000F6
:1046C400004E0000696300006B6E0000616D000025
:1046D400652000003D20000025730000004D00000F
:1046E40061780000537400006570000073200000BE
:1046F4003D200000256C00007500000044650000AA
:10470400762000005479000070650000203D000010
:104714002025000063000000544300006F6D00007A
:10472400702000004F6E0000203D00002025000096
:104734003175000000540000434D00006F64000018
:104744006520000025630000203D000020250000B6
:10475400640000004375000072720000656E000082
:1047640054430000203D00002025000063000000A9
:10477400424C0000436F00006D7000004F6E00005B
:10478400203D00002025000075000000424C000080
:10479400435300007465000070730000203D000066
:1047A4002025000075000000544300002053000041
:1047B4007461000072740000203D00002025000098
:1047C40075000000484F00006E5300007461000043
:1047D40072740000203D00002025000075000000D8
:1047E40000000000000000000000000000000000C5
:1047F40000000000000000000000000000000000B5
:1048040000000000000000000000000000000000A4
:104814000000000000000000000000000000000094
:104824000000000000000000000000000000000084
:104834000000000000000000000000000000000074
:104844000000000000000000000000000000000064
:104854000000000000000000000000000000000054
:104864000000000000000000000000000000000044
:104874000000000000000000000000000000000034
:104884000000000000000000000000000000000024
:104894000000000000000000000000000000000014
:1048A4000000000000000000000000000000000004
:1048B40000000000000000000000000000000000F4
:1048C40000000000000000000000000000000000E4
:1048D40000000000000000000000000000000000D4
:1048E40000000000000000000000000000000000C4
:1048F40000000000000000000000000000000000B4
:1049040000000000000000000000000000000000A3
:104914000000000000000000000000000000000093
:104924000000000000000000000000000000000083
:104934000000000000000000000000000000000073
:104944000000000000000000000000000000000063
:104954000000000000000000000000000000000053
:104964000000000000000000000000000000000043
:1049740043750000727200005374000065700000FB
:10498400203D0000202500006C750000005400004C
:10499400617200006753000074650000702000001D
:1049A4003D200000256C00007500000043750000E8
:1049B400726500006E74000050410000203D00004C
:1049C400202500006C750000005400006172000096
:1049D4006765000074500000412000003D20000085
:1049E400256C000075000000497300004D6F000045
:1049F400766900006E670000203D0000202500005D
:104A04007500000049730000486F00006D690000E4
:104A14006E670000203D00002025000075000000A6
:104A240049730000204800006F6D000065640000B9
:104A3400203D00002025000075000000000000005B
:104A44000000000000000000000000000000000062
:104A54000000000000000000000000000000000052
:104A64000000000000000000000000000000000042
:104A74000000000000000000000000000000000032
:104A84000000000000000000000000000000000022
:104A94000000000000000000000000000000000012
:104AA4000000000000000000000000000000000002
:104AB40000000000000000000000000000000000F2
:104AC40000000000000000000000000000000000E2
:104AD40000000000000000000000000000000000D2
:104AE40000000000000000000000000000000000C2
:104AF40000000000000000000000000000000000B2
:104B040000000000000000000000000000000000A1
:104B14000000000000000000000000000000000091
:104B24000000000000000000000000000000000081
:104B34000000000000000000000000000000000071
:104B44000000000000000000000000000000000061
:104B54000000000000000000000000000000000051
:104B64000000000000000000000000000000000041
:104B74000000000000000000000000000000000031
:104B84000000000000000000000000000000000021
:104B94000000000000000000000000000000000011
:104BA4000000000000000000000000000000000001
:104BB40000000000000000000000000000000000F1
:104BC4000000000000000000000000004E6900002A
:104BD400636B00006E6100006D650000203D000005
:104BE40020250000730000004D6100007853000090
:104BF4007465000070730000203D00002025000053
:104C04006C7500000044000065760000205400002C
:104C140079700000652000003D2000004200000083
:104C2400424C0000436F00006D7000004F6E0000A6
:104C3400203D00002025000075000000424C0000CB
:104C4400435300007465000070730000203D0000B1
:104C54002025000075000000484F00006E5300003E
:104C64007461000072740000203D000020250000E3
:104C7400750000006952000065760000657200004E
:104C840073650000203D0000202500007500000031
:104C94004D610000785300007065000065640000F9
:104CA400203D000020250000750000004E65000036
:104CB4007720000057690000466900002073000057
:104CC40065740000746900006E67000073200000C2
:104CD4006172000065200000696E0000636F0000CF
:104CE400727200006563000074000000556E0000DD
:104CF400616200006C650000207400006F200000F9
:104D0400636F00006E6E0000656300007420000095
:104D1400746F0000205700006946000069200000FD
:104D2400426F0000617200006400000045720000E0
:104D3400726F000072200000746500007874000037
:104D4400206E00006F74000020640000656600009F
:104D5400696E000065640000005400006861000092
:104D6400742000006465000076690000636500003B
:104D7400207400007970000065200000646F00005A
:104D840065730000206E00006F7400002065000051
:104D940078690000737400002E000000546800005D
:104DA40065200000636F00006D6D0000616E0000FF
:104DB4006420000069730000206900006E76000022
:104DC400616C0000696400002077000068690000DD
:104DD4006C650000206E00006F2000007465000008
:104DE4006D7000006572000061740000757200004F
:104DF40065200000707200006F62000065200000F2
:104E04006973000020610000747400006163000095
:104E140068650000642E000000540000686500000E
:104E2400206300006F6D00006D6100006E6400007F
:104E34002069000073200000696E000076610000A4
:104E44006C6900006420000062650000636100007A
:104E54007573000065200000746800006520000080
:104E64006465000076690000636500002069000045
:104E740073200000686F00006D6900006E67000019
:104E84000054000068650000206300006F6D00009E
:104E94006D6100006E640000207200006563000014
:104EA40065690000766500006420000077610000F9
:104EB40073200000666F000072200000616E000025
:104EC400206900006E760000616C000069640000D7
:104ED4002074000061720000676500007420000007
:104EE40064650000766900006365000000540000FA
:104EF40068650000207200006563000065690000B9
:104F0400766500006420000069640000656E00009E
:104F14007469000066690000657200002077000073
:104F240061730000206E00006F74000020720000A6
:104F3400656300006F6700006E6900007A65000019
:104F440064000000546800006520000072650000E1
:104F5400636500006976000065640000206300005A
:104F64006F6D00006D6100006E640000206300003E
:104F74006F6E000074610000696E000065640000DB
:104F8400206900006E760000616C00006964000016
:104F94002070000061720000616D00006574000003
:104FA4006572000073000000546800006520000072
:104FB40072650000636500006976000065640000A6
:104FC400206300006F6D00006D6100006E640000DE
:104FD4002077000061730000207400006F6F0000F0
:104FE400206C00006F6E0000670000005468000031
:104FF40065200000726500006365000069760000AA
:1050040065640000206300006F6D00006D610000A6
:105014006E6400002069000073200000666F0000C9
:10502400726D00006174000074610000746500001A
:1050340064200000696E0000636F0000727200005B
:1050440065630000746C000079000000705F00006C
:1050540061700000705F0000636F00006E66000006
:105064006967000000730000726300002F480000AD
:10507400756200002F480000756200002E63000076
:1050840000250000733A0000256900002025000077
:10509400732000002D2D00002061000073730000B8
:1050A40065720000746900006F6E000020660000E5
:1050B400616900006C650000640A000000000000E3
:1050C40000000000000000000000000000000000DC
:1050D40000000000000000000000000000000000CC
:1050E40000000000000000000000000000000000BC
:1050F40000000000000000000000000000000000AC
:10510400000000000000000000000000000000009B
:10511400000000000000000000000000000000008B
:10512400000000000000000000000000000000007B
:10513400000000000000000000000000000000006B
:10514400000000000000000000000000000000005B
:10515400000000000000000000000000000000004B
:10516400000000000000000000000000000000003B
:10517400000000000000000000000000000000002B
:10518400000000000000000000000000000000001B
:10519400000000000000000000000000000000000B
:1051A40000000000000000000000000000000000FB
:1051B40000000000000000000000000000000000EB
:1051C40000000000000000000000000000000000DB
:1051D40000000000000000000000000000000000CB
:1051E40000000000000000000000000000000000BB
:1051F40000000000000000000000000000000000AB
:10520400000000000000000000000000000000009A
:10521400000000000000000000000000000000008A
:10522400000000000000000000000000000000007A
:10523400000000000000000000000000000000006A
:105244000000000000000000000000000046000014
:10525400697200006D770000617200006520000033
:105264003D200000257500002E250000752E00004D
:1052740025750000004C0000454400004272000007
:1052840069740000652000003D20000025750000C1
:1052940000480000616E0000644300007472000066
:1052A4006C2000003D200000300000005769000021
:1052B400726500006420000049500000203D000099
:1052C40020250000642E0000256400002E25000027
:1052D400642E0000256400000057000069460000A9
:1052E400692000004D6F0000642000003D20000094
:1052F400256400000057000069460000694300006F
:105304006F6E00006E2000003D2000002564000048
:10531400005700006946000069460000564F00002F
:105324006B2000003D2000002564000000570000B1
:1053340069460000694600005665000072200000BE
:105344003D200000257500002E250000752E00006C
:1053540025750000005700006946000069530000ED
:1053640053490000442000003D2000002573000044
:1053740000570000694600006941000064640000B1
:10538400722000003D200000256400002E2500004E
:10539400642E0000256400002E2500006400000037
:1053A400576900004669000053650000634D000022
:1053B400203D000020250000630000005769000024
:1053C4004669000053650000634B0000203D000067
:1053D4002025000073000000707200006F7400004C
:1053E4006563000074000000736E00006D700000BF
:1053F40000610000646D0000696E0000006D000033
:1054040069630000726F0000636800006970000047
:1054140000730000656E0000644300006D640000CA
:10542400006600006F630000757300006572000081
:10543400312E0000687400006D00000070720000DE
:105444006F74000065630000742F0000636F000038
:105454006E660000696700002E680000746D00002D
:10546400006900007000000067770000007300000E
:1054740075620000006400006E73000031000000DB
:10548400646E000073320000006D00006163000070
:10549400006800006F73000074000000646800007E
:1054A40063700000002F0000707200006F74000031
:1054B40065630000742F000072650000626F0000D5
:1054C4006F7400002E680000746D00003F0000003F
:1054D4002F700000726F0000746500006374000098
:1054E4002F6300006F6E000066690000672E0000E5
:1054F400687400006D000000417500006720000022
:10550400203300002032000030310000362000003B
:10551400313000003A350000333A000032390000DF
:1055240000760000352E000034320000006E0000CA
:10553400616D0000650000006E6F000074200000C3
:1055440073650000740000003C6200003E550000DA
:10555400706C00006F610000642000006120000096
:10556400466900006C6500003C2F0000623E0000AC
:105574000063000068650000636B00006564000060
:1055840000660000616900006C00000054680000BF
:1055940065200000447900006E6100006D69000020
:1055A40063200000444E000053200000436C0000C0
:1055B400696500006E74000020690000732000001B
:1055C4006E6F000074200000656E000061620000D0
:1055D4006C650000642E0000006E00006F6E000019
:1055E40065000000626C00006F6300006B00000047
:1055F4000000000000000000000000000025000082
:105604006C750000000000000000000000000000B5
:105614000000000000000000000000000000000086
:105624000000000000000000000000000000000076
:105634000000000000000000000000000000000066
:105644000000000000000000000000000000000056
:105654000000000000000000000000000000000046
:105664000000000000000000000000000000000036
:105674000000000000000000000000000000000026
:105684000000000000000000000000000000000016
:105694000000000000000000000000000000000006
:1056A40000000000000000000000000000000000F6
:1056B40000000000000000000000000000000000E6
:1056C40000000000000000000000000000000000D6
:1056D40000000000000000000000000000000000C6
:1056E40000000000000000000000000000000000B6
:1056F40000000000000000000000000000000000A6
:105704004574000068200000536F0000636B0000C4
:10571400657400002044000069730000636F00009A
:105724006E6E00006563000074200000436F00008B
:10573400756E0000743A0000203D00002025000032
:10574400750000004574000068200000536F0000DD
:10575400636B000065740000204300006F6E00005E
:105764006E65000063740000204300006F75000044
:105774006E7400003A2000003D20000025750000F2
:1057840000450000746800002042000079740000A5
:105794006573000020520000783A0000203D0000AC
:1057A400202500006C750000000000004745000043
:1057B400544400004E4E00000047000045540000D1
:1057C40053540000410000004745000054430000CA
:1057D40046470000004400004F480000414C0000D0
:1057E4005400000053450000544400004E4E000095
:1057F400004D00004F5600004142000053000000DD
:10580400444F0000484F00004D4500000043000095
:10581400454E00005445000052000000534500006E
:10582400544200004345000000530000455400006A
:105834004243000053000000534500005448000058
:105844004F5300000053000045540000544300002F
:105854004500000053450000545400004353000029
:10586400004400004F4D00004F560000450000006A
:10587400444F0000535400004F50000000530000F8
:1058840045540000544300004D00000053450000FF
:1058940054540000434300000052000045530000EC
:1058A40045540000460000005345000054440000E5
:1058B40045560000004E0000696300006B6E000056
:1058C400616D0000652000003D20000000250000FF
:1058D4006C750000002500007500000047450000BD
:1058E400544400004E4E00000047000045540000A0
:1058F4005354000041000000474500005443000099
:1059040046470000004400004F480000414C00009E
:105914005400000053450000544400004E4E000063
:10592400004D00004F5600004142000053000000AB
:10593400444F0000484F00004D4500000053000054
:1059440045540000484F000053000000444F00003D
:105954004D4F000056450000004400004F53000026
:10596400544F000050000000524500005345000011
:1059740054520000005300004554000052450000FA
:1059840056000000534500005444000045560000F2
:10599400005300004554000042430000450000004D
:1059A400534500005442000043530000004D0000E2
:1059B4004F56000045500000410000004E690000B1
:1059C400636B00006E6100006D650000203D000007
:1059D40020000000256C0000750000002575000003
:1059E400000000003000000073720000632F00000C
:1059F400436C0000696500006E740000436F000092
:105A04006E6E000065630000746900006F6E000034
:105A1400732F0000436C0000696500006E74000081
:105A24002E63000000250000733A00002569000081
:105A340020250000732000002D2D000020610000AF
:105A44007373000065720000746900006F6E0000DB
:105A540020660000616900006C650000640A0000B3
:105A6400007000005F6300006C690000656E000058
:105A7400742D00003E770000726900007465000018
:105A84000021000000450000525200004F52000067
:105A940020490000442000003D200000256400004F
:105AA40000450000525200004F52000020540000F4
:105AB40045580000542000003D20000025730000DC
:105AC400004500004E4400000021000000000000DA
:105AD4000000000047450000544300004647000012
:105AE40000530000455400004C45000044000000F1
:105AF40047450000544400004247000000520000A3
:105B0400454200004F4F0000540000005245000081
:105B1400534500005448000000570000465300005D
:105B2400534900004400000057460000534500005C
:105B3400434D000000570000465300004543000059
:105B44004B0000005746000057450000504B000032
:105B54000050000055530000485700004600000064
:105B64005752000045530000455400000057000000
:105B74004946000049520000440000002575000019
:105B8400005300004554000000530000544F00002F
:105B94005245000000440000454600004155000005
:105BA4004C540000530000005245000053450000CF
:105BB400540000000100000058020000960000009C
:105BC40008000000C80000002C01000008000000CC
:105BD400C80000002C01000008000000C8000000FC
:105BE4002C01000008000000C80000002C01000087
:105BF40009000000C80000002C0100000D0A00008C
:105C040044480000435000002F5000006F7700000C
:105C14006572000020650000766500006E74000067
:105C2400206F00006363000075720000726500005D
:105C340064000000474500004D4900004E49000043
:105C4400000000004D500000465300000201000017
:0C5C5400000000003130000032000000B1
:020000040000FA
:105C60008040780032D5BF00814F500017003200CD
:105C7000E24F400008003200E2C1B3000440BC0023
:105C800060AB20000001410040A320000E0009008D
:105C900030197800E201B1000100780032F5B70058
:105CA000E2CF40000900320001407800E2C1B300B9
:105CB0000440BC0060AB20000001410040A3200074
:105CC0000E00090032187800E201B1000000060061
:105CD00011002000E54F500009003E00E0FF0700E2
:105CE00061528000000021000080600002003A0044
:105CF00080007800020037004D8AA90011002000C2
:105D000001007800000006008000EB00E54F500025
:105D100006003E00D2FF07008000EB0050528000DA
:105D2000E70F500001003A00110020000100780048
:105D300000000600E54F500012003E00C8FF0700BB
:105D40004ACABF00E74F500002003200EB4F50003C
:105D50000C003A00D1518000E05180000101500058
:105D6000808F500005003900A0518000360AB50030
:105D7000020040000000E900000006000200E90007
:105D80000000060000000500889FBE0080447800E7
:105D90000000EB00E5CF540009003E000940780008
:105DA000AFFF0700A8518000B051800008045000E8
:105DB0000804E90009407800DEFF070000005400F5
:105DC0004F04BE00000006008000EB00E54F5000CD
:105DD0000D003E00A2FF0700F2518000015280003A
:105DE000810F510002003900810051000600370088
:105DF000C051800081005000B0518000000051006F
:105E0000808040008100E80001007800000006006A
:105E1000889FBE00804478000000EB00E5CF54006E
:105E200008003E00094078008DFF0700B85180004F
:105E3000C05180000804500009407800E2FF0700CC
:105E4000000054004F04BE0000000600881F7800C8
:105E50000004780010007800B496020000000000F2
:105E6000000C780018009000B496020000000000BA
:105E70001004980028009000B8009000C696020018
:105E800000000000200498003104980048009000B1
:105E9000D8009000C6960200000000004004980060
:105EA0005104980078009000B496020000000000B1
:105EB0007004980008089000B496020000000000EA
:105EC000000C980018089000B49602000000000032
:105ED000100C98004F047800000006000200FA0041
:105EE000889FBE00C0002000E8CD02000000000036
:105EF0004856020000000000000FB2004280DE00A1
:105F0000F444500033003200710020000000EB0028
:105F10006E560200000000002B00370048560200B9
:105F2000000000000004E0002A003200E14F5000B1
:105F300025003200E24F500017003A00E2CF540033
:105F4000240036000000EB00D0BF9F00485602003E
:105F500000000000E44F500006003A0048560200DE
:105F600000000000B0FF9F00485602000000000043
:105F7000A0FF9F00DFB8970070212000808F5000A5
:105F800014003600D039B000808F500012003E005F
:105F90000100780010003700E1CF54000D003600FA
:105FA00048560200000000000044780080CF5400F2
:105FB000080039008080FB000000EB006E560200F4
:105FC0000000000088C454008944E900E1CF440087
:105FD000D2FF3A00802120004F04BE000080FA006A
:105FE00000000600889FBE008A1F78000005780028
:105FF00002047800840478000304E00015003200F5
:10600000E1CF51002A003A000104E000080032000C
:10601000E1CF500026003A000401780088007800A3
:106020000A007800B80D02000000000020003700D0
:10603000E10F4500030032000A0078005C5D0200B9
:10604000000000000800BE002E5702000000000003
:10605000170037000104E0000C003200E1CF5000CF
:1060600013003A00E10F4100030032000200780003
:10607000225D020000000000890078000A0078001C
:106080006E5602000000000009003700040178008D
:10609000880078000A007800C65A0200000000005C
:1060A000B05A0200000000000000E000FCFF3200D7
:1060B0004F0578004F04BE000000060033D5BF0036
:1060C00021532100914078000104E10018003200C2
:1060D000E24F40000B003200E2C1B3000440BC00BC
:1060E0007C03410065AB200062807A008002B10031
:1060F0008402200013C0B300E2A82000E6C07A00AA
:10610000B8FF070032D5BF0033F5B70082FD2F007E
:10611000A1518000010141008402200003A520005C
:106120009341780011C0B300E0A82000ADFF070044
:1061300000000600E1FF0700F05480007052880064
:10614000A0518000D0518800E0518800B0518000FB
:10615000F051880000528800400020004C6AAB00DB
:1061600001003A00D0002000505288004C0AA900DB
:106170004C2AA9004C4AA9004C8AA9004CAAA900A3
:106180004CCAA9004CEAA9004D0AA9004D2AA90051
:106190004D4AA9004D6AA9004D8AA800B00AA9007D
:1061A000B02AA900B06AA900B08AA900A051800055
:1061B000D05488004A9302000000000090548800E8
:1061C0004A93020000000000A0548800AEAAEF002D
:1061D0001000200000558800000006008000EB0041
:1061E000E54F500009003E009DFE0700B3FF070089
:1061F00080A2200041AA200009000900315878003F
:10620000E05480009051880081A2200001007800B5
:1062100000000600889FBE008A9FBE003415E20081
:1062200007003A00A893020000000000F27F20005F
:10623000020060000240200002004000A0A9880087
:10624000C20320008000EB0020A52000180C0200F3
:106250000000000049F920000005EB00D8DD2A000D
:106260000A4078007EFE07000800E80090007800F1
:1062700063004400100178001804E00008003A00B0
:106280000280400000804400AB0220008085450071
:1062900000ED2100808F550002003600FDFF370021
:1062A000FFFF3700506AEF00800220000900400025
:1062B000A0518800010040000000E800B0518800B3
:1062C00002004000C0518800D000200050528800D9
:1062D0004C6AA90079FF070078F89700B5EAB70083
:1062E00094FF07000A05E80066044400E60F550025
:1062F000020032008B047800D9FF37004F05BE0042
:106300004F04BE00000006002600FA00889FBE0071
:106310008A9FBE008C1F78000044780001457800F9
:1063200066FF07000808A300020032004D6AA800BB
:106330000804A1004CAAA9004CCAA9004CEAA90073
:106340004D2AA9004D4AA9004D0AA900CA5F0200C2
:10635000000000000000E000FCFF3200E6006400E6
:106360008004EB0056003A00D0518000D2548000E7
:10637000820F500002003A00810478004500370087
:1063800003558000820F50001300360002005000B9
:10639000830F5000010036000300780099558000FB
:1063A000890F500002003E00800478000100370091
:1063B0004D4AA8000902780003A520009341780007
:1063C0008040EB00909D200006FF07000900780048
:1063D0009A2AB4002F003700B15180000282500089
:1063E00084B79F0080004200A051800000805000D0
:1063F000830F50000100360003007800995580009B
:10640000890F500002003E00800478000100370030
:106410004D4AA800890F52000100360089B79F003D
:106420000FB2970003A52000934178008040EB0055
:10643000909D2000EBFE07000FB0970000825400F3
:1064400084B79F0009003200A2518000D054800020
:10645000360AB500919D20000100400003A52000F0
:10646000934178008040EB00DEFE0700D0548000AE
:1064700080804400D1548800B2518000828F500047
:1064800004003900A051800000005100008050003D
:10649000D05488004D6AAB000700320000558000E0
:1064A000808F54000400320090558000808F54008B
:1064B000010032000804A0000900E00002003A00D8
:1064C000630064001600320009007800A02AB500BD
:1064D0000900E000010032000834A0000A08A3000F
:1064E00005003200B46AEF00A1252600715488002F
:1064F00021002000815488001ED502000000000009
:106500007254800083548000000141008181490061
:1065100012528800235288004C8AA8002B003700B2
:10652000625280008A80FB000118A3000E00320036
:106530008240E800E780600080FF2F0000006100DB
:10654000010070006052880090548000A1548000C7
:1065500061005000E080580090548800A1548800E9
:1065600019002000190037007000610002003A0095
:1065700080047800150037000108A3000A003A00E3
:10658000B4CABF00080032000040E900B4EAB70016
:1065900070548000815480008100D1000080D300BD
:1065A00070548800815488001ED50200000000004D
:1065B00072548000835480000001410081814900B1
:1065C00012528800235288008004EB00F1548000AE
:1065D00091B79F00E2548000A2B79F0092548000C0
:1065E000A3548000B2B79F00C3B79F00B05480008F
:1065F000C1548000D0B79F00E1B79F007FB09700E3
:10660000F1FF23000100600001FF2F000100600086
:10661000F0B79F00F8EF9F000000EB00A0BF9F00C5
:1066200009014100E081490092548800A354880088
:106630008880FB000100D100610060008045780087
:106640000004E000130032000148A30003003A00F8
:106650006000B800D0B79F00E1B79F00B02AAB0040
:10666000070032003FB09700CFB0970061005000A4
:10667000E0805800B0B79F00C1B79F000500370009
:1066800061014100E081490092548800A3548800D0
:10669000B02AA8000808A30001003200B00AA80030
:1066A000F251800001528000810F51000500390035
:1066B000B0518000380AB50081005100010050003F
:1066C00002003700028050000000E90080BF9F00F8
:1066D000485F0200000000008000780080AF9F004B
:1066E000F0032000808F500003003E008000EB008C
:1066F00081AF9F000300370000FC2F0000804000A6
:1067000080AF9F008FA897007E8657000FB8970034
:10671000810F50000100360081BF9F000C007800FF
:10672000CAFD070074854400F2F02F007FB0970087
:10673000820060000105B300F1B79F000B04E00088
:106740000A0032007885440020C0B300A0D79F0023
:1067500040C0B300B0D79F0020802100A0AF9F00B1
:10676000028060000006B300F0B79F00219F200068
:10677000914078008180FB00F3C9BF004800DD0034
:1067800001017000419F2000914078008180FB0052
:10679000F5C9BF004800DD008101700060FD2F00D9
:1067A00000844700028CBE002055800031558000D7
:1067B000D0AF9F00E1AF9F000040EB00E0DF9F0003
:1067C00069C0B300F9DF9F008AB79F000A00780014
:1067D000B49602000000000080B79F00C1002000B6
:1067E00008007800F4960200000000000080EA0033
:1067F00090BF9F00109B20005C5D02000000000025
:106800000A0178008940780040AA200014CE0200D6
:1068100000000000410120000C0078002E5702000B
:10682000000000000B04E0000500320041002000E1
:1068300022FD2F00028047002E57020000000000BA
:10684000509C2000225D0200000000000A00780039
:10685000385C02000000000080AF9F00509D2000C7
:106860005C5D0200000000002100200000FD2F0000
:106870000F0040002E57020000000000965D02004D
:10688000000000004F0678004F05BE004F04BE0018
:106890000080FA0000000600889FBE008A9FBE00AC
:1068A000010478000205780083447800E54F500029
:1068B00054003E00EAFC07000800E00001003A0036
:1068C00018002000A0518000380AB5008005E900BA
:1068D0000A0444008B0F54004A003E00F7FD0700F5
:1068E0006380640001003A003940B300088055001D
:1068F0008981FB000318A30002003A000A01780016
:10690000040037000308A300010032000000D1009A
:1069100000014500A0518000000041000004E80093
:10692000F151800072558000E10F410009003200F2
:10693000105580000000410080804000C051800060
:10694000808F500003003600360AB50000804000FA
:106950008000E90000528000810F500002003900E1
:1069600005003600B0518000800F5400040036004E
:106970000328A30023003A0008528800F851880039
:1069800000528000808F5000110031000328A300C6
:106990000F003200B25180000282500003A5200097
:1069A0009341780083407800080078008DFD07004F
:1069B000F151800000528000808F500004003100AF
:1069C00008007800360AB50000805000F0518800B9
:1069D000B8518800A0518000D0548800E051880050
:1069E000D05188001100200050528000E70F500065
:1069F00005003A0000C1B30043FE0700110020006B
:106A0000010037008000EB00010078004F05BE0058
:106A10004F04BE0000000600881F78000044780084
:106A2000E9FC07000000E0000700320008407800A1
:106A30008BFC0700F05180000052880011C0B300A9
:106A400000C1B30030FE07004F04780000000600CC
:106A5000E54F500009003E0081FC070097FD07004C
:106A6000D1518000D0548000808F5000030032004C
:106A700011C0B30000C1B30023FE070000000600F0
:106A8000E54F500036003E0075FC0700F0518000D5
:106A90000052880050528000E50F50001200320072
:106AA00006003E00E10F50000D0032000E003900DC
:106AB000E30F500026003E000B003700EB0F5000A4
:106AC0001500320003003E00E70F500020003E009A
:106AD00006003700EE0F50001D003A001900370085
:106AE000868902000000000092FD370011C0B3004B
:106AF00010C1B30004FE0700A00AE2000400320047
:106B0000D1518000D0548000808F5000F7FF3A00B0
:106B1000800020000C00370011C0B30010C1B3008A
:106B2000F9FD0700A00AE20004003200D151800004
:106B3000D0548000808F5000F7FF3A00C000200042
:106B400001003700D00020005052880000000600ED
:106B50008040EB0040C1B300EBFD070075FD07006E
:106B600000000600881F780000447800E54F5000C0
:106B700004003E003AFC07004C6AA9000840780077
:106B8000BFFF07004F047800000006000400FA0071
:106B9000889FBE008A9FBE008C1F780090BF9F0018
:106BA000A1BF9F0002447800030578008445780067
:106BB0008004EB00094678000940780028FC0700B3
:106BC00050528000ED0F500063003A003BFD07007B
:106BD0000B407800B54AE3005F003A0080212000B6
:106BE000905588000804E00006003A00FA54880036
:106BF0004C6AA80040002000505288007A52880059
:106C00005300370000C02F003415B40081F8200075
:106C1000810F50000200360000402000A0A988002B
:106C2000A0A98000F05488000000E800A0A9880016
:106C3000EA5488001ED502000000000010528800AF
:106C4000215288004C8AA800E34F540016003200FD
:106C500003003E00E14F54003D00390003003700BF
:106C6000E44F54003A003A00210037001FB8970063
:106C7000AFB8970020558800315588000814A2004D
:106C80000880FB000000E9004F00DE004200DD004C
:106C9000815580000120A10080807000815588000E
:106CA0004A2AEF002A0037002FB897009FB89700B4
:106CB000010040000A004000F1548000010068001B
:106CC000705288001FB89700AFB897002055880011
:106CD00031558800B46AEF008109200071548800A2
:106CE000902AEF0020002000505288001800370042
:106CF0001FB99700224090000080FB00B240900036
:106D0000C808DD00808070009281FB001240900076
:106D10004800DD0003007000808040008A80400051
:106D2000F0548000808068007152880040AA2000E2
:106D30000900090032587800A200B100500020007C
:106D40005052880011C0B30020C0B3006EFD070090
:106D50000C80FB00040037008904E800E68F540033
:106D600094FF3A00E00F20004F0678004F05BE0068
:106D70004F04BE000080FA0000000600EF02B000E1
:106D8000889FBE008A9FBE008C9FBE008E1F780029
:106D900080057800820478001082FB00104090008B
:106DA0004800DD00040170002B4290000482FB00CB
:106DB0003B4090004800DD0084017000B2A79F00B6
:106DC000C3A79F001101BE00D2A79F00E3A79F00A9
:106DD0000040EB00E0CF9F0060C0B300F0CF9F0009
:106DE00089AF9F0009007800B496020000000000FF
:106DF00080AF9F00C100200060FC2F000F0040000A
:106E0000F4960200000000000004780009007800F9
:106E1000385C0200000000008880EA00808F50008B
:106E200035033A000000EB00E8CD0200000000004E
:106E300023FD2F0003844700410120000800780053
:106E40006E5602000000000008007800FFFB0700FB
:106E50007FA897004400DE006F4060004200DD0024
:106E6000744050000080FB000086540074075600F8
:106E7000AFA997000300E0001F0332002B409000F1
:106E80000080FB00BB409000C808DD0080807000DF
:106E90001B81FB001B4090004800DD0002007000D9
:106EA000808040009880400003856800E9CFB300EF
:106EB0000004EB000840780069FB07005052800096
:106EC000ED0F50002200320071528000E40F50009C
:106ED00005003A002FA89700808F50001C003A0050
:106EE000884478001A0037008A8F500018003A0052
:106EF00072FC0700AFA89700F0548000808F50000C
:106F000013003A0024FD2F0084804700E0548000E5
:106F1000910F10000E003A009B80FB001B40900078
:106F20004800DD0001017000AB4090008180FB0053
:106F30003B4090004800DD0081017000205580003A
:106F400031558000800F5100818F5900DD023200E1
:106F50000804E800E60F5400D6FF3A0025FD2F0094
:106F600005844700E2CF44000F003200094078005A
:106F70003BFB070051FC07007A52880046AA20001C
:106F8000090009003B5B7800AB00B10018047800F1
:106F9000E85488002FAC9700F8548800A95180006D
:106FA000D9548800C70237007FA897000098A30033
:106FB000D10232008A0AE200CF023A002FAB9700DA
:106FC000980278008004EB0024A6200014007800CA
:106FD0000000E00017003200860F500011003A0058
:106FE00054B89700850F50000E003A009B80FB00BC
:106FF0001B4090004800DD0001017000AB40900094
:107000008180FB003B4090004800DD008101700062
:1070100004B8970094B89700820F5000838F5800EF
:10702000870232008904E80074024200E38F5400B2
:10703000E6FF3A000004EB000840780008FB070078
:107040004C6AAB00050032001CFC0700F1548000C4
:107050002FA89700808F5000800232000804E800BB
:10706000E60F5400A4023200F3FF37001ED50200E1
:107070000000000042782D00730120000001410053
:1070800081814900125288002352880054528000A6
:10709000E40F520003003200E50F520047003A00AF
:1070A000160037000880FB00E400600006003A008C
:1070B0000048A300060032009A548800AB548800B0
:1070C0000440780090FC07001AFC07008A02370091
:1070D0000018A300FCFF32004FB09700DFB097000C
:1070E00061004000E0804800B0548800C15488002E
:1070F0007AFB0700905588002A0037008880FB0043
:107100000128A3007C023A004408DE006100600010
:10711000004678000004E00005003200985480002A
:10712000A9548000880F5500898F5D008C003A00BB
:107130000118A300700232004FB19700DFB1970031
:1071400061014100E0814900B2548800C3548800C5
:107150008FB197000355880060FB070090558800A9
:107160000C04E0000F00320011C0B30000C1B300F6
:1071700065FC070070002000505288001ED50200F8
:107180000000000042782D00730120000001410042
:107190008181490012528800235288004C8AA9003C
:1071A0005502370011C0B30020C1B30056FC0700E0
:1071B00060002000505288004F0237000883FB0017
:1071C000E1026300F5B79F00C5EF9F006FE89700ED
:1071D0000004E00002003A00BEB79F000200370042
:1071E00073065600BCB79F000884FB0088BF9F0051
:1071F0000818A300030032003FB197000201E80025
:10720000B2B79F00F251800001528000810F5100FF
:1072100005003900B0518000380AB50081005100E6
:107220000106500002003700028050000006E9000D
:10723000B0548000C15480004FB49700DFB4970071
:107240000001540081815C0082067800BFB4970081
:107250000900E0001F0032000C00E00028003200AE
:10726000E00F5100E08F5900040035006160B80064
:10727000820F5000838F58000A003E00BFB2970073
:1072800005004100E08049004240A90007003400A9
:1072900005005600CF80DE00800F5100818F59001D
:1072A00002003C0015002000010037008002EB00C6
:1072B0006160B800800F5100818F59000E003D00C1
:1072C0003FB49700088046004240A90010003C00EF
:1072D00009003700E00F5100E08F59000C00320028
:1072E000070035006160B800820F5000838F58009E
:1072F00007003E00020037000500E00004003A00ED
:107300008FBC97000928A300FB013A00E901370070
:10731000660063006CFF3A000FB897000048A300B6
:10732000F5013200EB0F520005003E00E70F52005E
:1073300015003100E60F5200D2003A00030037007A
:10734000EC0F5200CF003A00C6003700985480007E
:10735000A9548000880F5500898F5D000800320015
:107360009A548800AB54880011C0B30040C0B300E9
:10737000E5FB070098548800A9548800DE01370017
:107380007000200050528800D7548000D2518000F5
:107390008700510003003B00A0518000360AB50071
:1073A0008080400092548000A3548000010041007E
:1073B000E08049000000550081805D004240A90046
:1073C00009003400B00AAB0003003200E10F5000A6
:1073D000E08F5800020032008040EB00B601370019
:1073E00061055500E0855D00E65180000680530090
:1073F000CF80DE000002510081825900868F530049
:10740000020039000400BE0004003700A0518000D3
:10741000360AB50000005200E0805A000001550015
:1074200081815D004240A9002F003400A1518000FD
:10743000B9518000018454006140B800800F5100B0
:10744000818F590028003E00B06AA900B08AA900C7
:107450004D0AA900E051800002024000E45188007A
:10746000D1548000808F500004003900848F500078
:107470000D00310001005200040037000880400078
:10748000840F500008003100000052009254800028
:10749000A354800000004100E0804900905488001F
:1074A000A1548800D4548800B1518000810F52004B
:1074B00004003900A05180000080500000005200FC
:1074C000E0518800D2548000B1518000810F5100FA
:1074D0001C003900A05180000080500000005100C5
:1074E000D054880017003700870F53001500320072
:1074F000805580000038A300110032000048A3002E
:107500000E00320094548800A5548800D0548000A6
:10751000860F500007003100A0518000360AB500E8
:10752000CF80DE000000520081805A009054880015
:10753000A1548800D65488004D4AA800B08AA800FB
:10754000B06AA800E1518000D0518000808F5000C7
:1075500015003A004D6AAB000A003A001ED5020041
:107560000000000042782D0073012000000141005E
:107570008181490012528800235288004C8AA90058
:107580000900370090548000A15480008A0F5000F9
:107590008B8F580004003A00B00AAB0002003200A2
:1075A0004C8AA9004D6AA900905480008A005000BE
:1075B0000FB0970001005000A00AE20003003A005B
:1075C0000000E000010032004D2AA80000558800AC
:1075D00050528000E80F500013003A009054800091
:1075E000A15480008A0F50008B8F580025003A006C
:1075F000B00AAB00230032001ED5020000000000DC
:1076000022BC2E00B300200000014100818149000E
:1076100012528800235288004C8AA8009000200053
:107620005052880017003700E90F500008003A0058
:10763000FFB097000100E00012003A009A54880061
:10764000AB548800EFE8970040C1B3009DFE3700BF
:10765000EA0F50000B003A0090548000A1548000C3
:107660000400370092548000A35480006100410060
:10767000E08049008A0F50008B8F58001E013A00AD
:1076800091FE37008FBC97000902B2001A013A0040
:1076900050528000EB0F500017013200EA0F5000EB
:1076A00015013200EC0F5000130132000E00E00013
:1076B000980032000D0447000D00E0004C003C0033
:1076C0007FA897004200DE00C003B2000D0050000A
:1076D000E8CD0200000000008C0F540001003E00C5
:1076E00008067800B0548000C15480000C004000AF
:1076F000E0804800B0548800C1548800F5518000F3
:10770000C25180000C80420001A520009140780009
:10771000820F500013003600050451000804E800F1
:1077200008027800894178000081EB0005007800AC
:107730002CFA07000804560001A5200091407800AB
:10774000B051800008027800894178000081EB0088
:1077500024FA0700B051800000044400F85188006A
:10776000070037000C027800894178000081EB00A7
:10777000050078001BFA07000C0078003E2AB400D0
:1077800070558000E10F4000620032008C00500014
:1077900071558800105580000081400012003300B0
:1077A0000100E0005B003C00B0548000C154800048
:1077B00002004000E0804800B0548800C1548800B6
:1077C000F051800080004100F1518800C0518000DC
:1077D000808F500004003600360AB500008040005B
:1077E0000000E900F0518800AEAAEF004900370020
:1077F0008C0F5400010036000D0756007FA897003B
:107800004200DE00C003B200E8CD0200000000002C
:10781000F35180008D824100C25180000E804200F1
:10782000820F50001800360001A52000914078001A
:10783000030051000D0050000004E8000A0033006E
:1078400008027800894178000081EB00050078008B
:10785000E4F9070001A5200091407800B0518000B4
:10786000080257000500370002007800360AB5000C
:10787000008042000000E9000E0278008941780093
:107880000081EB000600370001A520009140780040
:107890000E027800894178000081EB000500780035
:1078A000D0F9070070558000E10F400003003A0056
:1078B0007D5588001E558800160037000D044700CE
:1078C00011558000808F56000B0031008100400070
:1078D000810F540002003E00800F5400020031006E
:1078E0001E558800020037000D805000105588009A
:1078F0007D5588000700370081004000810F54004B
:1079000004003600818F560002003E000000540043
:1079100010558800BFB097000100E000140032004D
:1079200050528000E70F500002003200F2518000F8
:10793000025288004CEAAB000500320011C0B300CF
:1079400000C1B30070FA0700DCF907000800370037
:107950004CEAA8004CCAAB0005003A004CCAA8008B
:107960003AD5020000000000D003B0004052880069
:10797000CFE997000304E0005F003200B4548000B8
:10798000C554800061014200E0814A003FB2970087
:107990004FB49700DFB4970004004400E0804C002F
:1079A000800F5100818F590053003A00B254880073
:1079B000C354880050528000E70F50000E00320080
:1079C00003003E00E60F50003A003A000500370081
:1079D000E80F50000F003200E90F500035003A0068
:1079E00014003700C00020005052880011C0B300BE
:1079F00010C1B30031003700B000200050528800A1
:107A00003AD5020000000000A007B00040528800F4
:107A10002800370090548000A15480008A0F500045
:107A20008B8F580003003200A000200050528800C5
:107A3000200037008040EB0000C1B300A1FD3700FB
:107A40003AD50200000000007449B90072014100FB
:107A500024A5200000317A0027003700744CB900BB
:107A60002AA520000A004400090009003B587800BC
:107A7000A000B100AB00B1006A0044009FAA9700CB
:107A800005307D000A0044003FA99700CFA9970068
:107A900062009800730098007000440001307D007F
:107AA0003AD50200000000007204440000347D005A
:107AB0001100370011C0B30000C1B30012FA070073
:107AC0000D0037007FDC97005FAD9700EFAD9700AA
:107AD0003FAA9700CFAA9700C4B79F00D5B79F00D1
:107AE0004C0AA9004C2AA9004C4AA9004C8AAB00B8
:107AF00066FD3A005DFD3700EA5802000000000014
:107B0000100020004F0778004F06BE004F05BE0052
:107B10004F04BE00EF02B100000006000400FA00AE
:107B2000889FBE008A9FBE008C1F78000006EB0075
:107B30008C4578000C40780049F8070060528000BE
:107B4000016020000100600031003200CA5F0200C5
:107B5000000000000000E0002D00320060528000B4
:107B60004A00DE006105600009C1B3002A00370049
:107B700052F907007440B9008001780022A5200066
:107B80000200400041AA200009000900B058780016
:107B9000A000B100EA804100E1007900E1548800D2
:107BA000EC80410082804000160020000700200089
:107BB00031024300A1824B00B4548800C5548800B0
:107BC000215580003755800087804000E2548000B6
:107BD00082804000F25480008280680071528800E8
:107BE0006100200051528800620214007422B90022
:107BF00061A620000181410013C0B30083407800DA
:107C0000F8F807008A2AEF0029C1B30031003700D5
:107C10008044EB000005EB004CAAAB0007003200EB
:107C2000385280003AD502000000000000045400E1
:107C30004240A90001003C0009C1B3004CCAAB009E
:107C400007003200485280003AD5020000000000D0
:107C5000000454004240A90001003C0009C1B300E7
:107C600050528000EB0F500009003A00485280004B
:107C70003AD5020000000000000454004240A90070
:107C800003003C00C00020005052880019C1B3001E
:107C900050528000E40F50000C003A0072528000F5
:107CA0000004EB0021A62000110078000000E00095
:107CB00006003200820F5000ADFF32000804E800D9
:107CC000F4804000E30F5400F7FF3A000904E0009D
:107CD0000400320011C0B3008AC05000094078008F
:107CE00089F907004C8AAB0026003A005052800008
:107CF000E70F5000EC003A001ED502000000000023
:107D000012528000235280000200500083805800ED
:107D1000E50033006152800067806000E60F50008C
:107D20000B003A00430CDE00614464000B40780015
:107D300053FB07000B40780051FB07000804E000EC
:107D4000D9003A00E000200050528800D6003700E9
:107D5000DAF8070021C0B30000C1B3006AF90700D8
:107D60001ED502000000000042782D0073012000A3
:107D7000000141008181490012528800235288008D
:107D8000C90037001ED5020000000000125280001A
:107D9000235280000200500083805800C20033004C
:107DA000C6F807005052800001002000EC0F500080
:107DB000E08F580094003E00006001000C00370086
:107DC000150037003A003700410037008E003700B9
:107DD0005F0037006A003700730037007B00370010
:107DE0008D0037007E0037006F00370081003700BC
:107DF0007A890200000000000000E00082003200EA
:107E0000110020005152880020558000A0890200F6
:107E1000000000007C0037006E805700648A02007A
:107E2000000000000000E0007700320086890200B8
:107E300000000000000478000000E00012003200A2
:107E40001FB89700AFB897002055880031558800BB
:107E5000200020005052880020558000A60AB4005F
:107E6000E154800001004000F154800001006800EE
:107E700070528800B46AEF008109200071548800B4
:107E8000902AEF00600037001ED5020000000000BD
:107E900042782D00730120000001410081814900DA
:107EA000125288002352880058528800560037002A
:107EB0003AD50200000000003052880040AA20009D
:107EC00010B8020000000000300020001900370048
:107ED00081AA200040AA2000E8B6020000000000AD
:107EE0000000E00015003A003AD502000000000052
:107EF000325280000200500072548000820F500005
:107F000041003600B4CABF00E54F500008003E00F3
:107F10000040E800B4EAB70070548000815480004B
:107F2000000040008180480070548800815488001F
:107F300020002000505288003300370050002000FD
:107F4000505288000004EB0029C0B30050003700F5
:107F500029C0B30040AB200032C0B300904F1100E5
:107F60007700360040C0B300B4EAB700045A2200DC
:107F70007454880064022000845488007000370024
:107F800040AB200015C0B30090CF12006700360050
:107F900060528000680060001F003A0029C0B300F2
:107FA000000478001E00370040AB200046C0B3003C
:107FB000904F13005F003600800020005052880070
:107FC00019C1B3000004EB001500370040AB2000DE
:107FD00047C0B30090CF1300580036000E003700A2
:107FE00040AB200041C0B30090CF100051003600DC
:107FF0000900370040AB200042C0B300904F110091
:108000004E003600040037000004EB000904E000D5
:1080100003003A002400370049C1B30018002000D3
:108020000A00E0001A003200B46AEC0070548000CC
:108030008154800000004000818048007054880016
:1080400081548800D0548000E35180000301500027
:10805000830F500003003100A0518000360AB500A4
:108060000001410090548000A154800002005000A3
:10807000E080580090548800A154880002007800E5
:10808000A02AB400D35488008040EB0001003700E0
:1080900011C0B300094078009BF807000800E00019
:1080A0000100320023F807000C06E800E60F560036
:1080B0009FFE3A008004EB007448B9000004780089
:1080C000700040002AA5200060007D000000E00054
:1080D0001D0032003AD50200000000007201440089
:1080E00062017D000200500072722000820F500079
:1080F0000A003600628214007422B90062A62000D1
:10810000020144000A00440013C0B3008340780019
:10811000B4F707008A2AEF008904E9008904E8001F
:10812000E28F540008003E00E3FF370029C1B3008E
:108130000300370009C1B3000100370019C1B300C3
:108140000004EB00B8FF37004F0678004F05BE0073
:108150004F04BE000080FA00000006000F03B000CC
:10816000889FBE008A9FBE008C9FBE008E1F780035
:1081700000447800E1B79F0082057800030578008D
:1081800084047800F5B79F00E54F50009A003E0048
:108190000200E00098003200B1F6070008407800C5
:1081A00009F707000A0650008B0F56009D003900A2
:1081B0000900E00003003200890F5600010036007C
:1081C000090678000052800000014500C15180007E
:1081D000810F51000400360001007800360AB50016
:1081E000000041000001E900028050000000E800AA
:1081F000C0B79F006FB39700364478007FB09700F8
:108200000000E00006003200F0C9B3000040440066
:10821000F94F500002003E0000CEB300004444007D
:108220008B047800AAB79F00D2B79F00060578009C
:108230008006EB0001C2B300E1E79F004FB1970059
:10824000FF0F510001003E00E2E79F00EFE09700C2
:108250000180FB008C0F500001003600ECE79F000E
:10826000EFE197000387FB000E02780003A52000D2
:10827000934178005FB1970011C0B30040FC2F001C
:108280000F00400086BF9F0056F707005FB09700C1
:108290000E004000D0B79F00CFB097008E805000F6
:1082A000C1B79F000FBB970004003A00B251800095
:1082B000D2B79F008081EB00C3B79F008003EB0023
:1082C00003CEB3007FB097000000E00025003A0025
:1082D000000178003D0037000081FB0040FC2F00CA
:1082E0000F0040008000410011427800F5C9B30042
:1082F00005404200F94F500001003E008348420013
:10830000914F540009003A008904E9003C00320012
:108310003A447800054044001D002000F94F500009
:108320000F003E00034444000D0037000D00E00044
:1083300002003A008B04780009003700EFB0970084
:108340001144780005404400F94F500001003E0000
:10835000034444008B047800060578008006EB0097
:108360008703E800074078006FE1970082CF530051
:10837000D9FF3900190037008080FB0043FC2F0033
:108380008F81410003804000904F540005003A0067
:108390008904E9001E0032003A4478001D002000E4
:1083A000090037000D00E00002003A008B0478005D
:1083B000050037006FB09700104478008B047800F8
:1083C000060578008006EB000201E8000240780014
:1083D000EFE09700814F5100E7FF39000E0656008D
:1083E000890F56000F0039002FB197000E01410090
:1083F000A2B79F008FFF37000000EB000A00370094
:10840000AFB197000B80510002004000030037001D
:108410002FB197000B005100010040000000E80060
:10842000010037000080EB004F0778004F06BE00C8
:108430004F05BE004F04BE000F03B1000000060050
:108440000200FA00E1FF9F00840278000302780036
:1084500082017800120020008F80E9003FFF0700B2
:108460000080FA0000000600889FBE008A9FBE00C0
:1084700000447800810578008204780003057800C4
:10848000E54F50002B003E000200E00029003200C2
:10849000F3F50700084078004BF6070080007800ED
:1084A00009004500810F5000010036008A84500009
:1084B0000052800000014500C1518000810F510031
:1084C0000400360001007800360AB50000004100C3
:1084D0000001E900028050000004E80050CABF001B
:1084E000888F540005003E00090278008041780022
:1084F00011C0B3000B0078000B00370008027800B1
:108500008041780011C0B3000B007800B5F6070079
:10851000B2518000088045000882540003A5200065
:108520009341780011C0B300AEF60700090178004E
:10853000010037000001EB00020078004F05BE008B
:108540004F04BE00000006000200FA00810178001E
:10855000120020008F80E900C3FF0700EFF89700AA
:108560000180FB000080FA0000000600889FBE002A
:108570008A9FBE00004578008104780002047800DC
:1085800011F60700800578000000E000320032009C
:108590000A407800B2F507008B0F54000100360046
:1085A0000B04780002528000C15180000800410095
:1085B0000005EB00810F50000E00360002805000D5
:1085C0000005E8000900E000070032000A02780018
:1085D00003A520009341780011C0B3000900780082
:1085E00080F607008A8444000A045400B0518000D9
:1085F000005288000900E0000700320002528000AB
:108600000802780003A520009341780011C0B30050
:108610000900780073F6070008007800402AB400CB
:108620000A04440008805500880F500002003E00F4
:108630004D4AA800070037004CAAAB0005003A00DD
:108640004CAAA8003AD5020000000000A007B00024
:1086500030528800080078004F05BE004F04BE006D
:1086600000000600889FBE008A1F780080447800C2
:1086700001057800D4F50700000478000000E00050
:10868000160032000940780075F507000A00E00086
:1086900007003200025280001400200003A52000D1
:1086A00093417800844078000A0078004DF6070076
:1086B000015280008100E80001528800C051800012
:1086C000808F500002003600B051800000528800B8
:1086D000E10F540003003A004D4AA800080078005A
:1086E00009003700100020004CAAAB0006003A0039
:1086F0004CAAA8003AD5020000000000A007B00074
:1087000030528800100020004F0578004F04BE0052
:1087100000000600889FBE008A9FBE008C9FBE009E
:108720000045780081057800820678000000EB00A3
:10873000E54F550042003E000A40780048F507002A
:108740000A4078007BF50700800478000000E00014
:1087500004003A000A407800BDF8070009007800DC
:10876000370037008D0F5000020036000D047800EE
:1087700001003700000478004D0AAB0008003A0001
:10878000A0518000360AB5000000D100808F54004F
:1087900003003E000A407800ADF807004D0AA8002B
:1087A000D5518000B1518000088042000006EB00E6
:1087B000810F50000C0039000586500001A52000F3
:1087C000914078000C02780013C0B3000B017800D0
:1087D0000500780003F607008C8545000C04540062
:1087E000A0518000D051880001A520009140780060
:1087F000D05180000802780013C0B3000B0178004C
:10880000F8F50700080078003A2AB4008D8F54006C
:1088100003003E000A4078008DF80700070037008B
:108820004CAAAB0005003A004CAAA8003AD50200B9
:108830000000000078004000305288000C00440026
:108840004F06BE004F05BE004F04BE0000000600EC
:10885000889FBE0080447800010478000100780001
:10886000CC0C0200000000000001780088007800B5
:1088700009407800A7FF0700000044004F04BE0035
:10888000000006000200FA00889FBE0080447800C5
:10889000A1FF9F00E54F500033003E00F0F40700B9
:1088A0000940780023F50700000478000000E0008C
:1088B0002D003200E10F500002003A00094078001C
:1088C00063F807004D0AAB0008003A00A051800091
:1088D000360AB5000000D100800F540003003E00AE
:1088E000094078005AF807004D0AA80001A52000A9
:1088F00091407800D051800014002000844178001D
:1089000066815700B7F50700D15180008100E8006B
:10891000D1518800B0518000808F50000200390092
:10892000A0518000D0518800E10F540004003A00AB
:108930000940780046F80700080078000B0037006F
:10894000100020004CAAAB0008003A004CAAA80076
:108950003AD5020000000000780040003052880044
:1089600010002000010037000000EB004F04BE00A3
:108970000080FA00000006000ACEBF000080FB0065
:108980004200DD00E1C7B300E2E020006040790072
:108990004244040000000000889FBE000A6EEF0001
:1089A000210037000084FB00C9E020004244DD00C4
:1089B000090044000008EB0084C0B3000305200058
:1089C0000041EB006000B800C63502000000000066
:1089D0000884E80000F47C0028EEEF0029EEEF00A8
:1089E000A2E02000124178000281FB00690920000A
:1089F0000991B90000ED2100020040005C5D020019
:108A000000000000000478008900780040E12000A8
:108A10002E57020000000000080078005C5D020094
:108A2000000000000A6EEC000ACEBF00E14F5000CB
:108A3000DCFF36000A6EEF004F04BE0000000600A7
:108A4000889FBE008A9FBE00004578000ACEBF0006
:108A5000804F55001E0032000080FB006809200096
:108A60000880B9000BED2100008045005C5D02002C
:108A700000000000800478008800780040E12000B9
:108A80002E57020000000000090078005C5D020023
:108A9000000000000A80FB000880B900008045004B
:108AA000225D020000000000800478008800780049
:108AB00040E120006E56020000000000090078002E
:108AC000225D0200000000000A0078000AEEB700F4
:108AD0004F05BE004F04BE00000006000200FA0071
:108AE000889FBE008A1F780000047800CC0C02002A
:108AF00000000000800178000801780023003700A2
:108B000082047800B94078000305E900D0C3B300BF
:108B100080CF5000030032007740500080CF5000DB
:108B200002003A00005CEB0016003700B0C2B30050
:108B300080CF500002003A006B4050000E0037001A
:108B400050C2B30080CF50000D003A00E10F550035
:108B5000100036009944780099FF9F002240900051
:108B600080FF9F00E3044100638551004FB89700E8
:108B7000F295020000000000005C78000100370060
:108B8000015C78008A017800090178000300E000A8
:108B9000DBFF3A00005CEB0008007800004CEB00C3
:108BA0004F0578004F04BE000080FA000000060068
:108BB000889FBE000004BE001600370088007800C1
:108BC00009007800F80B0200000000000000E0003F
:108BD00006003A0009007800CC0C020000000000FA
:108BE000000044000000E8000D0037000800780095
:108BF000CC0C020000000000000044000004E8006B
:108C000008007800CC0C02000000000000004400C6
:108C10000004E8001804E000E8FF3A000000EB0060
:108C20004F04BE0000000600889FBE008A9FBE0061
:108C30008C9FBE008E1F7800A3E020009341780037
:108C4000CBE020000047780001067800820678001B
:108C50000004E0000B0032000380FB004200DD0056
:108C60000080E8000002EB00840178000401780035
:108C70008E40780060C07D002042020000000000AD
:108C8000060037000380FB004200DD000080E800A2
:108C900060C07D00E42E02000000000000057800A6
:108CA0002B002000E10F40006B003200E18F5600E6
:108CB00012003E000C00E00012003200A87080009C
:108CC000B97080000ACEBF000080FB004200DD00CA
:108CD0000A0178008000EB00E3E0200060C079002A
:108CE000B64202000000000000045400E0845C0072
:108CF000A8708800B9708800360037000C00E000CA
:108D000010003A00A8708000B97080000ACEBF0041
:108D10000080FB004200DD000A0178008000EB00CB
:108D2000E3E0200060C07900B642020000000000CD
:108D300000045400E0845C00A8708800B9708800CA
:108D4000340037000D81E900CBE02000A3E02000D3
:108D500093417800A8708000B9708000820F5000A5
:108D60001E0036000380FB004200DD000080E800AA
:108D70008C00780060C07D00B64202000000000058
:108D800000045400E0845C00A8708800B97088007A
:108D90000D0155000281E8000ACEBF000080FB00F3
:108DA0004200DD000080E8008000EB0060C07D0034
:108DB000B64202000000000000005400E0805C00A9
:108DC000A0708800B17088008D0046000040EB0064
:108DD000E0F89F001B0020000F0037000380FB001D
:108DE0004200DD000080E8000A0178008C00780075
:108DF00060C07D00B6420200000000000000540088
:108E0000E0805C00A0708800B17088000040EB003A
:108E100000757E008005EB000E04E0000E003200BD
:108E2000A8708000B97080000ACEBF000080FB00EF
:108E30004200DD008000EB00E2E0200060407900AD
:108E4000324302000000000000045400E0845C0093
:108E5000A8708800B97088000B0078004F07780070
:108E60004F06BE004F05BE004F04BE0000000600C6
:108E7000889FBE000004780001017800800078001F
:108E8000D0C3B30068FF0700800478000800E0004A
:108E9000040032001804E0000200320008007800EC
:108EA0000EFF0700090078004F04BE000000060016
:108EB000889FBE008A9FBE008C1F78000005780046
:108EC00001067800010178008000780060C2B300DC
:108ED00055FF070080057800E20F500012003A00AD
:108EE000A8708000B97080000ACEBF000080FB002F
:108EF0004200DD00E1E0200060C07800E42E0200C6
:108F00000000000001002000800F5400818F5C00F1
:108F100005003A000C0178008A0078000040EB0060
:108F200041FF0700800578000A00E00004003200DD
:108F30001A04E000020032000A007800E7FE070091
:108F40000B0078004F0678004F05BE004F04BE00AE
:108F5000000006004000FA00889FBE008A1F7800CB
:108F6000000178000071800011718000E00F500056
:108F7000E08F580010003A0002007800A67F02003F
:108F80000000000080447800E14F40003F003200C4
:108F90000A83020000000000007188001100370001
:108FA00009407800187E020000000000202EEF002B
:108FB000222EEF0035003700007180004C7F020048
:108FC0000000000080447800E14F40002F00320094
:108FD0001271800003002000210020002281020085
:108FE000000000000ACEBF000080FB004200DD0050
:108FF000E1E0200060C078009A2E0200000000002E
:1090000000057800180037000A01780000042000ED
:10901000800F55000100360000017800A1FB2F00F1
:109020008F80400009407800AE7E02000000000002
:10903000000478000000E000D9FF32000ACEBF0033
:109040000080FB004200DD0008017800A1FB2F003A
:109050008F804000E3E0200060C079008A43020076
:1090600000000000080555000A00E000E6FF3A0095
:1090700009407800F28202000000000010718800B0
:1090800009407800187E0200000000004F057800BB
:109090004F04BE000080FA0000000600E90F5000F7
:1090A000E08F58001F003E000060010009003700FB
:1090B0000A0037000B0037000C0037000D003700A6
:1090C0000E0037000F003700100037001100370086
:1090D00012003700C0082A0003003700EC750400B6
:1090E0000000000070092A009AFF3700FE75040096
:1090F000000000007E7604000000000032760400CC
:10910000000000005C76040000000000A876040067
:1091100000000000F0760400000000001A77040050
:10912000000000000ACEBF000080FB004200DD000E
:1091300042002000210A2A00E3E0200060C07900FC
:109140008A430400000000006F09B000889FBE0041
:109150008A9FBE008C9FBE008E1F78000007EB0028
:10916000EDE020008E4478001D407800E24F400082
:10917000BD063200682E0200000000000000E00082
:109180001E0032000E4078002DFE0700C8E02000CF
:109190000ACEBF000080FB004200DD000800400056
:1091A0000008EB0028CEBF00E14F40000300320072
:1091B000187E02000000000028EEEF0029CEBF005C
:1091C000E14F400003003200187E02000000000062
:1091D00029EEEF000ACEBF000080FB004200DD0058
:1091E0000080E80043C0B3000001EB001100200044
:1091F00060407C004C340200000000007DB8970005
:109200000000E00005003A001D407800E42E020056
:10921000000000000000E0009306320009407800E2
:1092200007FE07000ACEBF000081FB00C210DD0070
:10923000C0E020006100780001002000EB0F50002A
:10924000E08F580088063E000060010018003700DB
:109250003F0037007A013700E70237000A03370082
:1092600013033700520437006F0437001A05370024
:10927000C50537004A0637005F0637000180FB004E
:109280004200DD000080E800220020008000EB00AA
:1092900060407E00B6420200000000000ACEBF001F
:1092A0000080FB004200DD00310020009901370002
:1092B000C9E020004210DD000080E80060C07C00B2
:1092C000E42E0200000000000000E000660632000C
:1092D00000E32000207188000ACEBF000080FB0060
:1092E0004200DD001800200008B07C002BEEEF00EB
:1092F0002A6EEF001ED5020000000000229D24000F
:10930000B30620000001410081814900E27088001D
:10931000F370880020AEEF0022AEEF00142EEF00B5
:10932000162EEF00A86EEF000ACEBF000080FB00F3
:109330004200DD000080E80053C0B3000001EB00F4
:109340008800780060C07C004C34020000000000FF
:10935000C9E020000ACEBF000080FB004200DD0013
:109360000080E8000002EB0084017800040178002E
:10937000A1C0B30060C07C002042020000000000D9
:10938000E10F40001D003A000ACEBF000080FB0044
:109390004200DD000080E80060C07C00082F020071
:1093A0000000000000017800180020000000E0002C
:1093B00008003A0050002000607188000ACEBF000B
:1093C0000080FB004200DD007100200001B07C0045
:1093D000020478001ED5020000000000E270800048
:1093E000F370800002005000838058004240A900C2
:1093F0001B063400C8E02000C30237001ED502005F
:1094000000000000229D2400B3062000000141005E
:1094100081814900E2708800F37088000ACEBF00A5
:109420000080FB004200DD000080E8000002EB004D
:10943000840178000401780001C2B30060C07C00A0
:109440002042020000000000E50F5000010036003D
:10945000500020000001E8000ACEBF000080FB00A1
:109460004200DD000080E80001E3200060C07C00D5
:10947000B64202000000000032002000710A2A00FB
:1094800000E32000C40B0200000000000000E00028
:109490000F00320042002000B10A2A0000E3200041
:1094A000C40B0200000000000000E00002003A00CF
:1094B0001000200006003700710020006171880054
:1094C0000ACEBF000080FB004200DD00270037000D
:1094D00060718800C9E020000ACEBF000080FB0058
:1094E0004200DD000080E8000002EB00840178000B
:1094F0000401780001C2B30060C07C002042020079
:1095000000000000000478000ACEBF000080FB00CD
:109510004200DD000080E8000002EB0088017800D6
:1095200004017800F1C3B30060C07C002042020057
:109530000000000000017800880F50000100360094
:1095400008017800A1E0200091407800B0062000DA
:10955000800F510007003600500020006071880025
:109560000180FB004200DD007100200001B07C00A2
:109570002CFF37000180FB004200DD000080E80086
:1095800001E3200060C07C00B64202000000000041
:109590007C0040004BE120000B0040000048EB0045
:1095A00000E320004DFD07000CE320000C007800D4
:1095B000CC0C0200000000000004780072002000C3
:1095C000010B2A0010E32000C40B02000000000081
:1095D0000000E0000E003A0010E3200028700200B6
:1095E000000000002BEEB700800020002C0EE200EF
:1095F0000100320090002000607188000ACEBF0098
:109600000080FB004200DD002200200072033700D2
:109610007B0044000B054000F9C2B3009ACF140050
:109620000400320010E32000A67F020000000000CA
:1096300028EEB70080E2200080C0EB0090CF100041
:109640000E003A009ACF1400030032007C00440060
:1096500009F07D000804E8000C004400710B2A00AA
:10966000080C0200000000006B04440010E320001E
:10967000A67F02000000000028EEB700F0E2200004
:109680000000440002E32000E1C2B3000300370001
:1096900090CF1000030032000000E900820F50005C
:1096A000FBFF3A000004E8002E2EEF00090037000F
:1096B0008000400040072A00E100780008007800A0
:1096C00074960200000000000004E0000400320074
:1096D0002E2EEC0070718000EA0F5000F4FF36006F
:1096E00010E3200028700200000000002BEEB700FD
:1096F00028CEBF00E14F40000B0032006A8202001A
:10970000000000000018A3000700320028CEBF00B0
:109710000A830200000000000000E8004C7F020005
:109720000000000029EEB700C9E020000ACEBF000B
:109730000080FB004200DD000080E8000002EB003A
:10974000840178000401780001C2B30060C07C008D
:109750002042020000000000000478000000E00049
:109760001D00320010C0B3002AEEB7000ACEBF00C1
:109770000080FB004200DD000080E800F2F52F00D1
:109780008280470060C07C0032430200000000007D
:109790000801E900A1E02000914078005007200076
:1097A000800F51006CFF3E00287180000180FB009B
:1097B0004200DD000080E80001E3200060C07C0082
:1097C000B6420200000000000004440060C2B30082
:1097D000005C780028718800C8E020000ACEBF0035
:1097E0000080FB004200DD000080E8000002EB008A
:1097F0008401780004017800A1C0B30060407C00BF
:1098000020420200000000000001E8000ACEBF0074
:109810000080FB004200DD000080E8008000EB00DB
:1098200060407C00B6420200000000000ACEBF008B
:109830000080FB004200DD002100200001307C00A0
:1098400018002000CCE020000ACEBF000080FB0002
:109850004200DD000080E8000002EB008401780097
:1098600004017800A1C0B30060407E0020420200E5
:109870000000000000057800E10F400027003A00DA
:109880000ACEBF000080FB004200DD000080E8003F
:1098900060407E00082F02000000000000017800F8
:1098A0000000E00008003A005000200060718800CD
:1098B0000ACEBF000080FB004200DD0071002000E6
:1098C00001307E00020478001ED502000000000076
:1098D000E2708000F3708000020050008380580026
:1098E0004240A900DE0434000ACEBF000080FB0025
:1098F0004200DD000080E80060407E00403502004C
:10990000000000000ACEBF000080FB004200DD0026
:10991000B100200001307E0042FE37001ED502005B
:1099200000000000229D2400B30620000001410039
:1099300081814900E2708800F3708800A1E0200076
:1099400091407800E10F55004CFE32000180FB0091
:109950004200DD000080E8000002EB008A01780090
:1099600004017800A1C3B30060407E0020420200E1
:1099700000000000800578008084E800A1E020005D
:1099800091407800F08F54000A0036000A01E80088
:109990000180FB004200DD000080E8008000EB0059
:1099A00060407E00B6420200000000000004EB00B0
:1099B000A4FF3700A3F72F00038447000180FB00BA
:1099C0004200DD000080E80009017800880078008E
:1099D00060407E00B6420200000000000B00E8007C
:1099E000080040000048EB00890555000004EB002A
:1099F000C9032A0099007800A2F72F0002804700CF
:109A0000F80B020000000000800078000000E00079
:109A1000EA003A000804E00069003A00C8E02000CB
:109A20000ACEBF000080FB004200DD000080E8009D
:109A30008102780001027800810178002200200074
:109A4000219F290060407C00AE4002000000000021
:109A50008004780060EA200021718000010050003D
:109A6000808F54005300390050002000607188003E
:109A70000ACEBF000080FB004200DD007100200024
:109A800001307C00BE003700CBE020000ACEBF00D2
:109A90000080FB004200DD000080E8000002EB00D7
:109AA0008401780004017800B1C3B30060C07D0078
:109AB0002042020000000000000478002A718000AB
:109AC00009017800808F5400010036000001780001
:109AD0000ACEBF000080FB004200DD000080E800ED
:109AE0008A00780060C07D00B642020000000000DD
:109AF0000000450061C2B300015878002071880061
:109B0000890F54001D0031000ACEBF000080FB0009
:109B10004200DD000080E8008000EB0060C07D00B6
:109B2000050037000ACEBF000080FB004200DD00C8
:109B30000080E80060407C0032430200000000002A
:109B4000C8E020000ACEBF000080FB004200DD001C
:109B50000080E8000002EB00840178000401780036
:109B600001C2B30060407C002042020000000000FF
:109B7000800078000000E000EAFF3200A6E020004C
:109B8000164378000683FB004233DD008002EB00C1
:109B9000050278008501780022002000219F29001D
:109BA000E0E0200066407800AE40020000000000C7
:109BB000800478000900E000B3FF3A00700037002D
:109BC000E14F540046003A002B4EE2006C00350095
:109BD000C8E020000ACEBF000080FB004200DD008C
:109BE0000080E800620020008000EB0060407C0004
:109BF000B6420200000000000ACEBF000080FB0059
:109C00004200DD000080E8008002EB0005027800E1
:109C10008501780022002000219F290060407C00FF
:109C2000AE4002000000000063044000C80FB20014
:109C300040022000800F540001003600000478002C
:109C4000A9F82F0089844700110037000ACEBF0011
:109C50000080FB004200DD00420020008900780007
:109C6000E3E0200060C07900B6420200000000007E
:109C7000330020000901780041002000090078002D
:109C8000069502000000000064045400E3844400D0
:109C90000800E000EDFF3A00884C7800A1F82F00A2
:109CA00081804700A2C3B30020FB2F000080470043
:109CB000914F1100030032008100E800808F5000B6
:109CC000FBFF3A008058EB00A0F82F00008047000F
:109CD00050700200000000002BEEB7002800370093
:109CE000E24F540026003A00C9E020000ACEBF002F
:109CF0000080FB004200DD000080E8008002EB00F5
:109D0000050278008501780022002000219F2900AB
:109D100060C07C00AE40020000000000000178003E
:109D2000E90F500005003600200020006071880017
:109D3000142EEF00162EEF001100370003F62F004F
:109D4000038447000ACEBF000080FB004200DD0014
:109D50000080E8008800780060C07C00B642020005
:109D600000000000080040000048EB0008007800F8
:109D7000260D020000000000A0708800B17088006D
:109D8000A5E02000954278008582FB00C22ADD0014
:109D90000002EB008401780004017800A1C0B30048
:109DA000E0E0200065407800204202000000000052
:109DB0008005780018002000050037000804E8003E
:109DC0008984E800E30F54000AFF3A000004EB0026
:109DD0000B01E8000ACEBF000080FB004200DD005E
:109DE0008000EB00E3E0200060C07900B642020092
:109DF0000000000093FE37002B4EE2000700350004
:109E000030002000607188004211DD0071002000E8
:109E1000C0E020000131780002FD37002071800091
:109E20000048EB0000E320002CFB070020718800B5
:109E3000CBE02000A1E0200091407800607180001C
:109E4000E80F500005003A000180FB004200DD00F1
:109E50007100200001B07D00F2FC37000180FB00A2
:109E60004200DD008B0040004000200080087800A8
:109E70002A4EE20002003A005000200080087800DC
:109E80002A6EEF00E7FC370074700200000000004B
:109E9000E20F5000740332000ACEBF000080FB00C6
:109EA0004200DD00C2E020005100200001307900B6
:109EB000C8E020000ACEBF000080FB004200DD00A9
:109EC0000080E80060407C00E42E020000000000FA
:109ED0006101B8000071800011718000800F510095
:109EE000818F590014003A001ED5020000000000C6
:109EF000E2708000F3708000020050008380580000
:109F00004240A9000C0034000ACEBF000080FB00D4
:109F10004200DD000080E80060407C004035020027
:109F2000000000000ACEBF000080FB004200DD0000
:109F3000B10020002E03370061718000E18F5000D6
:109F40000400320069805000E20F50000500360026
:109F500011013700B870020000000000F0DF9E0021
:109F6000D2003700EA8F500090003200EB8F500093
:109F700067003200E98F5000C8003A00C9E02000B5
:109F80000ACEBF000080FB004200DD000080E80038
:109F90008002EB0005027800850178004200200075
:109FA000310C2A0060C07C00AE40020000000000BE
:109FB00000017800A1E0200091407800E10F40000E
:109FC0003D0032000180FB004200DD000080E8001F
:109FD0008000EB0060C07C00B64202000000000080
:109FE000A2708000B370800000015100E081590030
:109FF000A2708800B37088000ACEBF000080FB000A
:10A000004200DD000080E80060C07C00E42E020019
:10A0100000000000E90F5000A0003600A0F62F005D
:10A02000008447000ACEBF000080FB004200DD0034
:10A030000080E800A20020008800780060C07C005A
:10A04000B642020000000000A2708000B3708000E1
:10A0500000015100E0815900A2708800B3708800AF
:10A06000A2002000810C2A0008007800C40B020026
:10A07000000000000000E0000B003A00A0002000FB
:10A0800060718800DA8102000000000028EEB7004D
:10A0900062002000E3F62F00838047006083020007
:10A0A0000000000002003700B0002000607188004E
:10A0B000200020007A0037000180FB004200DD0014
:10A0C0000080E80060C07C00E42E02000000000078
:10A0D000640150000ACEBF000080FB004200DD009A
:10A0E0000080E8008000EB0060C07C00B642020007
:10A0F00000000000A2708000B370800000015100D9
:10A10000E0815900A2708800B370880063003700B6
:10A11000A8708000B9708000CAE020000ACEBF009D
:10A120000080FB004200DD000080E80060407D0010
:10A13000E42E02000000000000045400E0845C00F3
:10A14000A8708800B97088000ACEBF000080FB00AC
:10A150004200DD000080E80060407D000C35020018
:10A1600000000000C0F92F00F1FF2F00A270800056
:10A17000B37080000200400083804800C2F92F00C5
:10A18000F3FF2700820F5000838F580043003600F2
:10A190000ACEBF000080FB004200DD0071002000FD
:10A1A00001307D000000EB003D0037000ACEBF000B
:10A1B0000080FB004200DD00E1E0200060C078008C
:10A1C000E42E02000000000080047800A2708000ED
:10A1D000B370800001002000820F5000838F580070
:10A1E0001C003600820478001A003700090178004C
:10A1F000F08F54000100360002012000A3F62F006A
:10A20000038447000ACEBF000080FB004200DD004F
:10A2100088007800E3E0200060C07900B6420200C8
:10A220000000000000017800A0708000B170800084
:10A2300002005000E0805800A0708800B1708800D3
:10A240008284540028CEBF0088007800608302001A
:10A25000000000000900E000E4FF3A00A070800068
:10A26000B1708000E00F5000E08F58000B003A0002
:10A270001000200044830200000000000ACEBF004E
:10A280000080FB004200DD00C2E0200071002000E1
:10A29000013079000900780001003700100020002B
:10A2A000F0DF9E000004E000470032007FD89600F7
:10A2B000E24F50000C003A000ACEBF000080FB00C5
:10A2C0004200DD00E1E0200060C07800E42E0200E2
:10A2D000000000000000E90001002000007188007B
:10A2E0001171880060023700E14F50002A003A00E7
:10A2F000C8E020000ACEBF000080FB004200DD0065
:10A300000080E80060407C00E42E020000000000B5
:10A310000100200000718800117188001ED5020024
:10A3200000000000229D2400B3062000000141002F
:10A3300081814900E2708800F3708800A27080007B
:10A34000B37080000071800011718000800F510097
:10A35000818F5900090036000ACEBF000080FB0043
:10A360004200DD000080E80060407C00082F020011
:10A37000000000000000E0003B023A006000200006
:10A38000607188000ACEBF000080FB004200DD0043
:10A3900071002000160237000ACEBF000080FB00CB
:10A3A0004200DD00C2E020006100200001307900A1
:10A3B00080E2200080C0EB0090CF100009003A003E
:10A3C00040002000607188000ACEBF000080FB00C2
:10A3D0004200DD0072002000C1E0200002B07800E1
:10A3E00090FB3700142EEF00162EEF0029CEBF0091
:10A3F000E14F400003003A0018AEEF001AAEEF0044
:10A400000300370081E12000888002000000000086
:10A410000ACEBF000080FB004200DD00C2E0200049
:10A420007100200001307900C8E020000ACEBF0092
:10A430000080FB004200DD000080E80023C0B30084
:10A440000001EB001100200060407C004C34020051
:10A4500000000000607180000000400081FF2900C2
:10A46000E08078000ACEBF000080FB004200DD00E3
:10A470000080E80060407C002844020000000000EA
:10A4800060718000EC0F500020003A000ACEBF003F
:10A490000080FB004200DD000080E80001E32000B6
:10A4A00060407C0028440200000000000ACEBF008B
:10A4B0000080FB004200DD000080E800310D2A0032
:10A4C00060407C0028440200000000000ACEBF006B
:10A4D0000080FB004200DD000080E80001E3200076
:10A4E00060407C0028440200000000000ACEBF004B
:10A4F0000080FB004200DD000080E800219F290071
:10A5000060407C0028440200000000006071800070
:10A51000E10F5000060036000ACEBF000080FB00AD
:10A520004200DD00B100200001307C00CE01370088
:10A5300070718000EB0F50001B0032000ACEBF008C
:10A540000080FB004200DD000080E800610E2A0070
:10A5500060407C0028440200000000007071800010
:10A5600000004000A19D2900E08078000ACEBF00D5
:10A570000080FB004200DD000080E80060407C00BD
:10A5800028440200000000000ACEBF000080FB004B
:10A590004200DD000080E800219F290060407C002F
:10A5A000284402000000000028CEBF006A8202009A
:10A5B000000000000008A300080032000ACEBF001F
:10A5C0000080FB004200DD000080E800510F2A00FF
:10A5D00060407C0028440200000000000ACEBF005A
:10A5E0000080FB004200DD000080E800E1102A004E
:10A5F00060407C0028440200000000006071800080
:10A60000E10F500005003200C0708000D170800062
:10A61000E10F4000E08F4800060032000ACEBF0084
:10A620000080FB004200DD000080E800E1112A000C
:10A630000D0037000ACEBF000080FB004200DD00A5
:10A640000080E80071122A0060407C00284402006B
:10A65000000000000ACEBF000080FB004200DD00C9
:10A660000080E80001132A0060407C0028440200BA
:10A6700000000000C8E020000ACEBF000080FB0000
:10A680004200DD000080E800219F290060407C003E
:10A690002844020000000000A1E020009140780062
:10A6A0002A4EE200040032000180FB004200DD007F
:10A6B000810020004E0137000180FB004200DD00D8
:10A6C0000080E800219F290060407C0028440200AF
:10A6D000000000004201370000E3200030718800D4
:10A6E000980037000180FB004200DD000080E80098
:10A6F00041132A0060C07D002844020000000000D1
:10A700003B00370000C2B30080CF500005003A0084
:10A710000ACEBF000080FB004200DD00B1C2B300E2
:10A720002F003700F0C2B30080CF50000B0036007E
:10A7300060CCB30000C04000E64F50000700360078
:10A7400050CAB30000C04000E54F5000030036007F
:10A75000A0C7B30080CF50001E003600C8E0200024
:10A760000ACEBF000080FB004200DD000080E80050
:10A7700051C2B30060407C0042440200000000006F
:10A780007FD896004E9602000000000080407800BE
:10A790000ACEBF000080FB004200DD000080E80020
:10A7A00060407C0042440200000000007FD8960018
:10A7B0006296020000000000804078000ACEBF00D0
:10A7C0000080FB004200DD000080E80060407C006B
:10A7D000050037000ACEBF000080FB004200DD000C
:10A7E000E2E02000604079004244020000000000E6
:10A7F00030718000B0407800F1DF9E003071880039
:10A800000104E000BFFF3A000ACEBF000080FB0059
:10A810004200DD00D1C3B3003700370000C2B300EF
:10A8200080CF500005003A000ACEBF000080FB0038
:10A830004200DD00B1C2B3002F003700F0C2B30008
:10A8400080CF50000B00360060CCB30000C0400049
:10A85000E64F50000700360050CAB30000C0400069
:10A86000E54F500003003600A0C7B30080CF500072
:10A870001E003600C8E020000ACEBF000080FB00AA
:10A880004200DD000080E80051C2B30060407C005F
:10A8900042440200000000007FD896004E9602005D
:10A8A00000000000804078000ACEBF000080FB005E
:10A8B0004200DD000080E80060407C00424402006D
:10A8C000000000007FD896006296020000000000A1
:10A8D000804078000ACEBF000080FB004200DD000F
:10A8E0000080E80060407C00050037000ACEBF0011
:10A8F0000080FB004200DD00E2E0200060407900C3
:10A90000424402000000000030718000B040780036
:10A91000F1DF9E00307188000104E000BFFF3A00C3
:10A920000ACEBF000080FB004200DD00219F29000D
:10A93000E2E02000604079002844020000000000AE
:10A940002A6EED00CBE02000A1E0200091407800CD
:10A950002A4EE20063FF3A000180FB004200DD0066
:10A960000080E800219F290060C07D00284402008B
:10A97000000000000ACEBF000080FB004200DD00A6
:10A980009100200001B07D000ACEBF000080FB00D6
:10A990004200DD00E1E0200060C078009A2E020055
:10A9A00000000000A4708000B5708000C2708000BC
:10A9B000D3708000040151008581590001002000FE
:10A9C000800F5100818F5900010036000001BE0048
:10A9D0008204780002004200E0804A00A0708800F3
:10A9E000B17088001A003700890078000204200046
:10A9F000828F54000100360082007800CBE02000F6
:10AA00002AFB2F000A85470028CEBF0001017800ED
:10AA10008A007800AE7E020000000000000478008A
:10AA20000000E000480032000ACEBF000080FB00BA
:10AA30004200DD000080E800080178008A0078000C
:10AA400060C07D008A43020000000000888454003A
:10AA50000900E000E4FF3A00A2708000B3708000BB
:10AA6000C0708000D1708000800F5100818F59002C
:10AA700040003A000ACEBF000080FB004200DD002B
:10AA8000C2E02000A100200001307900202EEF005C
:10AA9000222EEF0028CEBF0089007800307E020011
:10AAA0000000000028CEBF00E1F52F008F8040009D
:10AAB000307E0200000000000000E0000A003200CA
:10AAC000A2708000B370800061014100E081490004
:10AAD000A2708800B3708800E0C7B300EFD9960079
:10AAE00080CF5100EFFF3A00A0708000B17080006D
:10AAF00061004000E0804800A0708800B1708800CC
:10AB000029CEBF00C1E120008880020000000000C3
:10AB100029CEBF0081E120008880020000000000F3
:10AB2000000478000000E00012003A0018AEEF00C8
:10AB30001AAEEF0029CEBF00187E02000000000010
:10AB400029EEEF000C00370028CEBF00187E02006F
:10AB50000000000028EEEF000ACEBF000080FB00DE
:10AB60004200DD00B100200001B07D00180020008F
:10AB7000010037000004EB000ACEBF000080FB009C
:10AB80004200DD00E1E0200060C078009A2E020063
:10AB9000000000000000E00031003A003200370001
:10ABA000C8E020004210DD000080E80060407C002A
:10ABB0009A2E020000000000EF0F50002A0036001D
:10ABC000E0708000F170800034F9070000718000AF
:10ABD00011718000E00F5000E08F580022003A0011
:10ABE0000ACEBF000080FB004200DD009100200083
:10ABF00001307C008BF9370028CEBF00E14F4000C8
:10AC000003003200187E02000000000028EEEF0072
:10AC100029CEBF00E14F400003003200187E020041
:10AC20000000000029EEEF00C8E020000ACEBF00BF
:10AC30000080FB004200DD000080E80060407C00F6
:10AC400040350200000000000ACEBF000080FB007B
:10AC50004200DD00080040000008EB000200370061
:10AC60000800E0006FF932000E07E800E4864600B5
:10AC7000E20F57003BF93A004F0778004F06BE003D
:10AC80004F05BE004F04BE006F09B1000000060072
:10AC9000CD22A90041E2A9004342A80041E2A80058
:10ACA00000A023004012880040C2BF000018A3008B
:10ACB000FDFF3A0040C2BF000008A300FAFF3200C7
:10ACC00041E2A9004342A90041E2A80040128000ED
:10ACD000CD22A8000080FB00000006000200FA0060
:10ACE00000017800CD22A900A003200040128800B6
:10ACF0000200E000010032000201E90040C2BF0092
:10AD00000018A300FDFF3A0040C2BF000008A300E6
:10AD1000FAFF320040128000E0FF9F000002EB00CB
:10AD2000E18F50003000360041E2A9004342A80004
:10AD300041E2A8004822EF000482E80040C2BF00C0
:10AD40000018A300FDFF3A0040C2BF000008A300A6
:10AD5000FAFF3200431280000200E00004003200DB
:10AD60004818DE00104198000281E800034978008D
:10AD700004805000E10F5000EEFF3E0041E2A900C8
:10AD80004342A90041E2A800170037004822EF0023
:10AD90000402E8000200E0000A0032000201E800BC
:10ADA00040C2BF000018A300FDFF3A0040C2BF0030
:10ADB0000008A300FAFF320040128000004978002A
:10ADC0000900370040C2BF000018A300FDFF3A0091
:10ADD00040C2BF000008A300FAFF3200401280000A
:10ADE000E0FF9F000001EB00810F5200E7FF3900F8
:10ADF000CD22A800040078000080FA0000000600C0
:10AE00000200FA00CD22A90041E2A9004342A800B5
:10AE100041E2A8000080FB0001A0270001007000B3
:10AE20004012880040C2BF000018A300FDFF3A0096
:10AE300040C2BF000008A300FAFF320041E2A900AF
:10AE40004342A90041E2A80040128000E0FF9F00B9
:10AE5000CD22A8000080FA00000006000200FA00DF
:10AE60008001780001027800CD22A900A00720000F
:10AE70004012880040C2BF000018A300FDFF3A0046
:10AE800040C2BF000008A300FAFF32004012800059
:10AE9000E0FF9F00E10F520002003E008000EB0047
:10AEA0003B0037001380FB004800DD00F20FB200CA
:10AEB00000017100134090000080FB0001F02F00A2
:10AEC00001016100000171008381E80041E2A900F5
:10AED0004342A80041E2A800421288000482E9002F
:10AEE000E10F5200120036001380FB004800DD0025
:10AEF000F20FB20000017100134090000080FB00CF
:10AF000001016100000171008381E80040C2BF00BF
:10AF10000018A300FDFF3A0040C2BF000008A300D4
:10AF2000FAFF320040128000E0FF9F00EAFF370086
:10AF300040C2BF000018A300FDFF3A0040C2BF009E
:10AF40000008A300FAFF320040128000E0FF9F00DB
:10AF500041E2A9004342A90041E2A800CFFF370027
:10AF600063C078000080FB004012880040C2BF0030
:10AF70000018A300FDFF3A0040C2BF000008A30074
:10AF8000FAFF320040128000E0FF9F008100E800DD
:10AF9000848F5000F2FF3A00CD22A8000080FA0012
:10AFA0000000060000017800CD22A9008180FB008E
:10AFB0004112880040C2BF000018A300FDFF3A0004
:10AFC00040C2BF000008A300FAFF32004012800018
:10AFD0004822EF0040C2BF000018A300FDFF3A0066
:10AFE00040C2BF000008A300FAFF320040128000F8
:10AFF0004822EF0040C2BF000018A300FDFF3A0046
:10B0000040C2BF000008A300FAFF320040128000D7
:10B01000CD22A80000497800020078000000060058
:10B020000200FA00CD22A9000064A0000080FB000D
:10B030004012880040C2BF000018A300FDFF3A0084
:10B0400040C2BF000008A300FAFF32004012800097
:10B05000E0FF9F000180FB004012880040C2BF005B
:10B060000018A300FDFF3A0040C2BF000008A30083
:10B07000FAFF320040128000E0FF9F000000000055
:10B0800000000000CD22A8000080FA0000000600A9
:10B09000881F7800A1A780008100400074844000D0
:10B0A000109A2000800F54000200360020672F0005
:10B0B00000844000884078000040EB00D8FF070083
:10B0C000C840DE0010C0B300D5FF07004F04780071
:10B0D000000006000200FA00889FBE00000478000D
:10B0E00081447800D2BF9F0031CAB30020C0B300B2
:10B0F000CBFF070091C0B30030C0B300C8FF07000A
:10B10000009B2000DFB8970080804000D1BF9F00E7
:10B11000AFF8970060C0B300C1FF0700BFF8970009
:10B1200070C0B300BEFF0700610020000800780077
:10B130004AFF070061002000F0A1200047FF070040
:10B1400080C0B3002EFF070061C0B3000904E00017
:10B1500001003A00894078000140780028FF07008C
:10B160004F04BE000080FA00000006000200FA0052
:10B17000CD22A9000074A0000080FB0040128800CE
:10B1800040C2BF000018A300FDFF3A0040C2BF004C
:10B190000008A300FAFF320040128000E0FF9F0089
:10B1A0000180FB004012880040C2BF000018A300CD
:10B1B000FDFF3A0040C2BF000008A300FAFF3200C2
:10B1C00040128000E0FF9F00CD22A8000080FA001E
:10B1D00000000600881F7800F214E20011003A0017
:10B1E0001000200090A78800B8A780000804E9009C
:10B1F000109A2000800F54000100360000047800EF
:10B2000001C4B300E0C1B300D8FF07008840780054
:10B21000C0C0B30082FF0700C840DE00D0C0B3004A
:10B220007FFF07004F047800000006000200FA00CC
:10B23000CD22A9000080FB00000AB3004012880064
:10B2400040C2BF000018A300FDFF3A0040C2BF008B
:10B250000008A300FAFF320040128000E0FF9F00C8
:10B260000180FB004012880040C2BF000018A3000C
:10B27000FDFF3A0040C2BF000008A300FAFF320001
:10B2800040128000E0FF9F00CD22A8000080FA005D
:10B29000000006000200FA00F0BF9F0031C0B300BA
:10B2A000F0C1B300E1FF0700FFF89700F0C1B30061
:10B2B000AEFF07000080FA0000000600881F78003B
:10B2C0000044780050312000F2FF070088407800E9
:10B2D00050C1B30052FF07000000EB00EDFF070074
:10B2E0004F047800000006000400FA00881F780070
:10B2F00000447800D1BF9F0040212000E5FF0700F7
:10B300008840780040C1B30045FF0700AFF89700C0
:10B3100060C1B30042FF0700BFF8970070C1B300DF
:10B320003FFF0700A0302000DAFF0700A1C0B300F4
:10B33000648057001BFF07004FF897000008A30028
:10B34000FAFF3A000000EB00D2FF07004F0478003C
:10B350000080FA00000006000400FA00889FBE008A
:10B36000800478000144780040212000C9FF0700D4
:10B370008840780040C1B30029FF070011C0B30026
:10B3800020C1B30026FF0700A0302000C1FF070046
:10B39000A1C0B3006880570002FF07000FF89700B4
:10B3A00061446000FAFF3A0040212000B9FF070025
:10B3B0008840780020C1B30019FF070081C1B300A5
:10B3C00067805700F7FE07001FF897000080FB001A
:10B3D00001F02F00010464000004740091C1B30067
:10B3E00066805700EFFE07002FF897004800DD0049
:10B3F000F80FB200000474000000EB00A5FF070086
:10B40000880C7800090078004F04BE000080FA0024
:10B41000000006000200FA0011C0B3000F80E9002E
:10B42000CDFF07007FB897004200DE00610060009A
:10B430000080FA000000060000017800CD22A9007B
:10B440008180FB004112880040C2BF000018A300A9
:10B45000FDFF3A0040C2BF000008A300FAFF32001F
:10B46000401280004822EF0040C2BF000018A30035
:10B47000FDFF3A0040C2BF000008A300FAFF3200FF
:10B4800040128000CD22A800004978000200780018
:10B49000000006000200FA00881F780050312000EA
:10B4A0007CFF070051C1B30064805700E2FF070032
:10B4B0004FF897000084FB000000EB0075FF0700C9
:10B4C000080078004F0478000080FA0000000600B1
:10B4D0000200FA0001C2B300E0C1B30053FF07004D
:10B4E000D1C1B3000F80E900D3FF0700EFF8970048
:10B4F00061C06000FAFF320041C0B300F0C1B30088
:10B500001AFF07000080FA00000006000200FA009F
:10B5100041C0B300F0C1B30044FF0700D1C1B30084
:10B520000F80E900C4FF0700EFF8970064C06000D7
:10B53000FAFF3A00F1C1B3000F00E900BEFF0700B7
:10B540007FF897000038A300FAFF3A0001C2B30069
:10B55000E0C1B30005FF07000080FA00000006000C
:10B560000200FA00F1C1B3000F80E900B2FF07004A
:10B57000EFF897000180FB004500DE000000A2000C
:10B58000610060000080FA00000006001000FA0070
:10B59000889FBE008A9FBE008C9FBE00A0B79F0000
:10B5A000B1B79F00C2B79F000005EB008A05780085
:10B5B000E10F4000020032008A0678000C003700DC
:10B5C00021C0B300768057009BFF07002FE897004B
:10B5D0000080FB00A0B79F0031C0B300758057000A
:10B5E00095FF07003FE89700D0E79F001D0020006F
:10B5F0000006EB003FB09700E10F40000C003A005E
:10B600008040EB00748057008BFF07004FE89700E5
:10B610000080FB00B0B79F0011C0B30073805700DB
:10B6200085FF07005FE89700F0E79F001C002000FF
:10B63000CFB49700E18F54003F003E000C00E000C3
:10B640000C003A008C407800728057007AFF0700A7
:10B650006FE897000085FB0011C0B30071805700B0
:10B6600075FF07007FE897004800DD00FA0FB20081
:10B67000000575000D00E0000C003A0021C0B30089
:10B68000708057006CFF07000FF097008085FB006B
:10B6900031C0B3006F80570067FF07001FF09700AD
:10B6A0004800DD00FB0FB20080857500EFE09700D9
:10B6B0000040EB005AFE0700FFE0970010C0B30007
:10B6C00057FE0700CFE0970020C0B30054FE0700EC
:10B6D000DFE0970030C0B30051FE07000004EB002C
:10B6E000030037006AFD0700C5FD07000804E800F5
:10B6F000890F5400FBFF3A000C00E00006003A00FE
:10B700008A4078000C40780045FE0700C850DE00F3
:10B7100010C0B30042FE07000D00E0004F003A00E9
:10B720008B40780020C0B3003DFE0700C858DE0003
:10B7300030C0B300480037000D00E00009003200BF
:10B740002FB09700008444008840780020C0B300E8
:10B7500033FE07004844DE008840780030C0B30064
:10B760002FFE07003FB49700088544008A04E900D3
:10B77000C9B79F00F1C1B3006E8057002EFF0700CC
:10B780002FF097000058A300FAFF3A00EFE097006F
:10B7900000C1B30022FE0700FFE0970010C1B30014
:10B7A0001FFE0700CFE0970040C1B3001CFE07005A
:10B7B000DFE0970050C1B30019FE0700109A200087
:10B7C000800F540005003E00808F540003003600B7
:10B7D000D0652F0000004500C0B79F007885570056
:10B7E0009A40780020C1B3000DFE0700F78457008F
:10B7F0009940780030C1B30009FE070001C1B300D1
:10B80000F0C1B30089FE070001C2B300F0C1B3006C
:10B8100056FE07000C00E000100032004FB1970008
:10B820008200E800C1B79F00109A2000800F5400EA
:10B8300004003E00808F50000200360000005100DE
:10B84000C0B79F009A4078000040EB00F4FD07006D
:10B850009940780010C0B300F1FD07004F06BE000C
:10B860004F05BE004F04BE000080FA000000060035
:10B87000FA874700889FBE008A9FBE008C9FBE004B
:10B880008E1F7800800578008040EB0070805700A4
:10B89000E9FE07000FF097000080FB0001F02F0089
:10B8A000010565000005750011C0B3006F805700E9
:10B8B000E1FE07001FF797004870DD00FA0FB200A5
:10B8C000000575006066B8001C0037008B0078002A
:10B8D000F48F55000100360041012000A8FD2F0023
:10B8E0000F044400011C780008007800FBFC0700EE
:10B8F000DFA8970081855500618060000500320057
:10B900000040EB0080707C005FA897000000E8001A
:10B91000D0AF9F00DFA8970008017800040037002F
:10B920003200780000064600E0864E008180E90083
:10B930000100E000FAFF3A00D1AF9F000B00E000E9
:10B94000E2FF3A000C04BE008A4078000B40780009
:10B95000B3FD07008E40780010C0B300B0FD0700B3
:10B960006148B8000C004000E08048000100400041
:10B970000080EA004F0778004F06BE004F05BE006A
:10B980004F04BE00AF01B100000006000200FA0043
:10B99000889FBE008A9FBE0081057800A1A7800015
:10B9A0008100400074844000109A2000800F5400F1
:10B9B0000200360020672F00008440008040EB002A
:10B9C0006A8057009CFE07006A8057003081FB00A8
:10B9D00001F02F00010565000205750011C0B300DC
:10B9E00095FE0700FFF497004848DD00FA0FB2000B
:10B9F00000057500884078000040EB0088FD0700D6
:10BA0000C840DE0010C0B30085FD07000B007800C1
:10BA100097FF0700000478008A4078000040EB00A0
:10BA20007FFD07008940780010C0B3007CFD07004F
:10BA3000080078004F05BE004F04BE000080FA00E9
:10BA4000000006000400FA00881F78006681570095
:10BA5000001978008040EB000200780076FE0700B5
:10BA60004FF897000080FB0001F02F0001046400F4
:10BA70000004740011C0B300638057006EFE07001D
:10BA80005FF897004800DD000884FB0000047400A4
:10BA9000AFF897000040EB0061FD0700BFF897008A
:10BAA00010C0B3005EFD0700080078004F04780066
:10BAB0000080FA00000006000400FA00881F7800E9
:10BAC000668157000019780021C0B3000200780099
:10BAD00059FE07004FF897000080FB0001F02F008F
:10BAE000010464000004740031C0B3006380570097
:10BAF00051FE07005FF897004800DD000884FB0056
:10BB000000047400AFF8970020C0B30044FD0700A4
:10BB1000BFF8970030C0B30041FD0700080078006F
:10BB20004F0478000080FA00000006001000FA00C0
:10BB3000889FBE008A9FBE008C9FBE0001C8B300D4
:10BB4000F0C1B30089FD070001C8B300F0C1B30024
:10BB5000B6FD0700A1C0B300C0C1B300B3FD07002C
:10BB600081C0B300F0C1B30080FD0700F0D4BF0076
:10BB700065405000E14F500072003E000004EB00B1
:10BB8000C1C1B300748057002BFE07004FE8970037
:10BB90006A00600004003A000804E800803E2000CB
:10BBA000800F5400F6FF3A00C1C1B3007380570004
:10BBB00021FE07005FE897000018A30003003A0089
:10BBC000703E2000800F54005E00360081C0B3003C
:10BBD000F0C1B30095FD07008040EB007280570074
:10BBE00015FE07006FE897000080FB0008F02F00AB
:10BBF000888464008084740011C0B3007180570091
:10BC00000DFE0700FFED97004858DD00F90FB20068
:10BC10008084740061C0B3007080570006FE070086
:10BC20000FF097000080FB0008046400000474001B
:10BC300071C0B3006F805700FFFD07001FF0970031
:10BC40004800DD00F80FB200000474000804E800AA
:10BC500008467800884078000040EB00F0FC0700C0
:10BC60004844DE00084578008840780010C0B300E2
:10BC7000EBFC0700FC865700810020000D007800D7
:10BC800016FC070008C1B300C1C1B3006E805700A5
:10BC9000E9FD07002FF097000018A30023003200F1
:10BCA0003FB0970000D8A3002000320001C8B300C5
:10BCB000F0C1B3002DFD070001C8B300F0C1B3000F
:10BCC0005AFD0700A1C0B300C0C1B30057FD070073
:10BCD00081C0B300F0C1B30024FD0700C1C1B300AF
:10BCE0006D805700D4FD07003FF097006A006000A8
:10BCF000FAFF320081C0B300F0C1B3004BFD070072
:10BD00008C4078000040EB00C5FC07008A407800BA
:10BD100010C0B300C2FC0700810020000D007800B5
:10BD2000EEFB07000844E900D7FF3A00894078009D
:10BD30000040EB00BAFC07008B40780010C0B30055
:10BD4000B7FC07004F06BE004F05BE004F04BE0003
:10BD50000080FA00000006001600FA00889FBE006E
:10BD60008A1F780000057800810478009011200077
:10BD700048FD070091C1B30068805700AEFD070081
:10BD80000FFC97000000EB0042FD07000000EB00F5
:10BD90000804E0003A003200F214E20003003A0026
:10BDA0000CFD07000000EB0035003700B0A7800055
:10BDB000A0A78800414F2100914078000040EB008F
:10BDC00097FC0700514F21009140780010C0B3004C
:10BDD00093FC0700410120007C805700BFFB070057
:10BDE0003FB89700B496020000000000B0BF9F006B
:10BDF000AFB19700109A2000808F51000D003E00D7
:10BE0000CFE0970061C060000A003A004FB1970090
:10BE1000000128000000610006003A00BFB0970052
:10BE2000E05E2000808F500002003E000278A300F8
:10BE300001003A000000FE00B3A7880070805700A0
:10BE400005000900305D78006A00B1006000B100B3
:10BE500080CCEB007FF09700E84F500006003A00DE
:10BE60006FF097000004E00002003200E64F50003F
:10BE700001003A00804C7800F234EF0010002000FE
:10BE80004F0578004F04BE000080FA000000060055
:10BE90000600FA00889FBE008A1F780090112000DB
:10BEA000FCFC070091C1B3006C80570062FD0700E5
:10BEB0004FF49700E0002000F6FC0700E1C0B3005B
:10BEC0006B8057005CFD07005FF097000080FB006F
:10BED0000AF02F008A84640080847400F1C0B300EB
:10BEE0006A80570054FD07006FF097004800DD009E
:10BEF000F90FB2008084740090112000E5FC070067
:10BF000091C1B300698057004BFD07007FF0970097
:10BF1000884F5000E3FF3A00C0002000DDFC07001E
:10BF2000C1C0B3006880570043FD07000FF89700B9
:10BF30000080FB000A04640000047400D1C0B30058
:10BF4000678057003CFD07001FF897004800DD00A0
:10BF5000F80FB20000047400888F5400040036000B
:10BF600088805400109A200001005000050037001E
:10BF7000109A2000888F54000200320009005400FB
:10BF80000000E9004F0578004F04BE000080FA0071
:10BF9000000006000200FA00F1C1B3000F80E900C2
:10BFA00025FD0700EFF897000180FB004300DE004D
:10BFB0000000A200610060000080FA00000006009E
:10BFC0000400FA00889FBE00CD22A800C922A90063
:10BFD0004022EF00F0002000101288004422EF0001
:10BFE0004302A80042A2A80041E2A80001C2B30097
:10BFF000E0C1B3008DFC0700100020001AD702003A
:10C0000000000000CD22A900F00F2000401288009F
:10C0100040C2BF000018A300FDFF3A0040C2BF00AD
:10C020000008A300FAFF32004012800080FF9F004A
:10C03000CD22A800100020001AD702000000000046
:10C04000D1C1B30066805700FBFC07002FF89700B2
:10C050000080FB000038A300E4FF3A000080EA0003
:10C06000E1046000E1FF3A001800200098A7880072
:10C07000B9A788008940780080C0B300E8FB0700BA
:10C080008940780090C0B300E5FB070011CAB300F7
:10C09000C0C0B300E2FB070091C0B300D0C0B30042
:10C0A000DFFB070011CAB300A0C0B300DCFB070030
:10C0B00091C0B300B0C0B300D9FB070021CAB300E0
:10C0C00040C0B300D6FB070091C0B30050C0B3001E
:10C0D000D3FB070021CAB30020C0B300D0FB070088
:10C0E00091C0B30030C0B300CDFB07000940780019
:10C0F00043FB07000020200066FC0700D1C0B3000E
:10C1000009407800C6FB070021C3B30020C0B3007C
:10C11000C3FB070021C1B30040C0B300C0FB070050
:10C1200001C4B30030C0B300BDFB0700F1C3B300CE
:10C1300090C0B300BAFB070021C1B30060C0B300D8
:10C14000B7FB0700C1C0B30070C0B300B4FB070069
:10C15000E1CEB300A0C0B300B1FB070051C0B300F3
:10C16000B0C0B300AEFB07004030200049FC070020
:10C17000F1A120009140780040C0B300A8FB070067
:10C1800001A220009140780050C0B300A4FB07003A
:10C1900011A220009140780020C0B300A0FB07004E
:10C1A00021A220009140780030C0B3009CFB070022
:10C1B00031A22000914078000940780098FB0700E8
:10C1C00041A22000914078000840780094FB0700CD
:10C1D0008940780050C1B30091FB070021C1B30032
:10C1E0006580570094FC07003FF89700F0F4B70013
:10C1F0000110200000C1B3003BFC070021472300D1
:10C2000040C1B30038FC070089007800094078007D
:10C2100035FC0700090078001EFC070041C0B30090
:10C22000F0C1B300D1FB07004F04BE000080FA004C
:10C23000000006002E15E20003003A001000200066
:10C2400070A9880042F4EF0042D4BF00E14F4000E3
:10C2500003003200E09702000000000042F4EF000B
:10C260002000200060A288004E34EF001000200063
:10C2700020A288004674EF004694A8004634A80027
:10C280000000060042D4BF00E14F4000030032002E
:10C29000E09702000000000042F4EF004434EF0099
:10C2A000000006004414E20006003A0020002000CE
:10C2B00060A288004E34EF001000200020A2880009
:10C2C0004614A9000000060020A280000000E00043
:10C2D00001003200100020000000060030A28000A3
:10C2E000610060000000060030A280006200600073
:10C2F000020032004634A9001000200000000600B1
:10C3000030A280004300DE006100600000000600F3
:10C31000C0A28000D1A28000F2E9B7004801DE008F
:10C3200002007800F3E9B70001007800F4E9B700F3
:10C330004808DE00F5E9B700000006000800FA0032
:10C34000881F78000040EB00F0F79F0068805700DE
:10C35000D69A0200000000000FF89700E24F50004C
:10C36000E5003A00C0012000C09902000000000072
:10C37000F8A1200068805700D69A02000000000053
:10C380000FF89700984F5000F2003A000804E800B8
:10C3900050A22000800F5400F6FF3A004654AB0034
:10C3A00008003A0000012000C099020000000000CF
:10C3B0004100200080452100FA9A020000000000A0
:10C3C0006C14A800000F2000C099020000000000BB
:10C3D0006884570008007800D69A02000000000028
:10C3E0000000E000C40032008FF8970030C3B300B3
:10C3F00080CF50008E00320007003E00E3CF500097
:10C4000031003200E6CF500050003200E1CF500042
:10C41000AE003A001700370060C3B30080CF500071
:10C4200070003200E1CF4000B30032000040E9006C
:10C4300080CF5000A5003A0008007800D69A02008C
:10C44000000000000FF89700E14F5000C1003A00D3
:10C4500069805700D69A0200000000004654AB00E5
:10C46000DBFF32007FF09700E24F5000D8FF3A0028
:10C47000B800370008007800D69A020000000000DB
:10C480000FF89700E44F5000B2003A004654AB005A
:10C49000070032000044780068805700D69A0200F6
:10C4A000000000000844E900C9FF3200FAFF37002D
:10C4B0004100200000462100FA9A0200000000001E
:10C4C0006C54A800C2FF37006A805700D69A020059
:10C4D000000000006FF09700E34F50009D00360011
:10C4E0004654AB000700320048C0B30068805700D4
:10C4F000D69A0200000000000844E900060032005D
:10C50000FAFF370041002000C0452100FA9A0200DE
:10C51000000000006C34A800EFF09700E4C0500069
:10C52000E1F79F000300370068805700D69A0200A9
:10C53000000000006FF297000440E900E0F79F0060
:10C54000E14F4000F8FF3A00A1FF37006A80570032
:10C55000D69A0200000000006FF09700E34F5000F1
:10C560007C0036004654AB0018003A004100200021
:10C5700040462100FA9A0200000000006C74A800F6
:10C58000EFF0970064C05000E0F79F00E34F5000C9
:10C590000E0036004654AB000C003A00410020006B
:10C5A00080462100FA9A0200000000006C94A80066
:10C5B0006FF2970064425200E4F79F0003003700D7
:10C5C00068805700D69A020000000000EFF0970044
:10C5D0000140E900E0F79F00E14F4000F8FF3A001A
:10C5E0007BFF370008007800D69A020000000000A8
:10C5F0000FF89700E44F500056003A006380570050
:10C60000D69A02000000000064805700D69A02000B
:10C610000000000065805700D69A0200000000006C
:10C6200066805700D69A02000000000068FF3700BD
:10C6300008007800D69A0200000000000FF897006A
:10C64000E44F500043003A004654AB00080032006B
:10C650000044EB0068805700D69A020000000000FA
:10C660000844E800E44F540059FF3200F9FF370056
:10C6700030452100D69A020000000000204521002C
:10C68000D69A02000000000010452100D69A020050
:10C690000000000000452100D69A020000000000C2
:10C6A00080A2800091A28000C509DE004B0ADD0057
:10C6B0004501DE0002017200020050008380580034
:10C6C00080A2880091A2880041FF37006A8057004D
:10C6D0000100370068805700D69A02000000000071
:10C6E000EFF097000140E900E0F79F00E14F4000C4
:10C6F000F8FF3A0036FF37007FF09700E24F500016
:10C7000006003A005FB89700EFB89700A0A2880033
:10C71000B1A288004654A80009003700A2A28000F8
:10C72000B3A280005FB89700EFB89700800F510068
:10C73000818F5900020032000040EB00F0F79F00AB
:10C74000229B0200000000007FF097000080FB00A9
:10C7500003003700229B0200000000000000EB00F5
:10C760004F0478000080FA0000000600889FBE0099
:10C770008A1F7800804478000105780010C0B3005B
:10C78000FA9902000000000010C0B300FA990200FC
:10C790000000000060C0B300FA9902000000000031
:10C7A0000040EB00FA9902000000000020C1B30035
:10C7B000FA9902000000000030C2B300FA990200AA
:10C7C0000000000040C3B300FA990200000000001E
:10C7D00060C5B300FA990200000000000040EB00C1
:10C7E000FA990200000000000040EB00FA990200F4
:10C7F000000000000040EB004694AB0001003A004E
:10C8000000C8B300FA990200000000000040EB00ED
:10C81000FA99020000000000E3CF540007003A003C
:10C820000A00E000050032004100200080452100A0
:10C83000209A0200000000000C0037000040EB00CE
:10C84000FA990200000000000040EB00FA99020093
:10C85000000000000040EB00FA9902000000000018
:10C860000040EB00FA990200000000000044EB00D9
:10C870000040EB00FA990200000000000844E800C4
:10C88000EC4F5400FAFF3A0061002000F0A12000B4
:10C89000209A020000000000A8CCB3000040EB008A
:10C8A000FA990200000000000844E900FBFF3A008A
:10C8B00030C6B300FA9902000000000020C8B3009F
:10C8C000FA9902000000000030C5B300FA99020096
:10C8D0000000000030C6B300FA990200000000001A
:10C8E00050C3B300FA9902000000000010C0B3006A
:10C8F000FA9902000000000009407800FA9902004D
:10C9000000000000E1CF540002003A004654A900A4
:10C9100016003700E3CF540014003A000A00E0008C
:10C9200012003A0060C3B300FA9902000000000050
:10C9300040C0B300FA9902000000000057D4BF00C5
:10C94000FA9902000000000056D4BF00FA990200D4
:10C950000000000055D4BF00FA990200000000005A
:10C9600054D4BF00FA9902000000000070C3B30065
:10C97000FA9902000000000040C0B300FA990200DA
:10C980000000000010C0B300FA990200000000008F
:10C9900030C0B300FA9902000000000060C0B3008C
:10C9A000FA99020000000000C0C0B300FA9902002A
:10C9B00000000000E3CF540003003A000A00E0004A
:10C9C0000800320011003700E1CF54000F003A0098
:10C9D000C0A28000D1A28000E00F5000E08F58007C
:10C9E0000A00320020C3B300FA99020000000000E0
:10C9F00040C0B300FA99020000000000410020008E
:10CA000080452100209A020000000000C0C0B30051
:10CA1000FA990200000000000004EB00E2A02000F0
:10CA200001C2B30068407900814F5000030032001A
:10CA30000804E800EF0F5400FAFF3A0008407800BD
:10CA4000FA9902000000000088007800E0A02000B1
:10CA5000209A02000000000000C0EB000100370037
:10CA60000040EB00FA99020000000000419D8000A8
:10CA7000B0122000808F5000F9FF3600219F200067
:10CA8000914078008180FB00F3C9BF004800DD00C1
:10CA900001047000419F2000914078008180FB00DC
:10CAA000F5C9BF004800DD00810470000A00E00005
:10CAB00006003A000005FD00F2E9B700F3E9B7000F
:10CAC000F4E9B700F5E9B7000005FD00629A02003D
:10CAD0000000000008007800F2E9B7004840DE00DE
:10CAE000F3E9B70009007800F4E9B7004848DE0030
:10CAF000F5E9B7004F0578004F04BE0000000600BE
:10CB0000889FBE008A9FBE008C9FBE0020A280002E
:10CB10000100200061005000E0805800EB0F500041
:10CB2000E08F58007A013E00006001000B003700E2
:10CB300015003700570037006200370092003700B9
:10CB4000F7003700220137004A0137002001370083
:10CB5000480137001E013700460137003404200029
:10CB6000430420000041EB006000B800129802006E
:10CB70000000000042F4B700E14F400064013200C1
:10CB80002000200020A28800C003200080A288008E
:10CB90005234EF006C74EF004614A9004654A9000B
:10CBA0000A5A0200000000000000E00058013200B4
:10CBB00042D4BF00D099020000000000B112200052
:10CBC000810F50005201360031A280004408DE007F
:10CBD0000080EA00610060004400DD000140A10027
:10CBE0008080700031A2880042D4BF0082C1B300AF
:10CBF0000440BC00C03A210000004100A200200017
:10CC0000F10F2000180C0200000000008000EB0073
:10CC100010C0B300D5FE07001ED5020000000000C2
:10CC20000006BE0060A2800071A280006011B80002
:10CC3000A4252600250020006033B800E407020088
:10CC4000000000000205BE000004BE004A9302007E
:10CC5000000000000100200002002000030020006E
:10CC6000A4252600250020006033B80042090200F8
:10CC70000000000008044000898448000C044400BF
:10CC80008D844C0048A2880059A288003000200002
:10CC90001E01370042D4BF00BA9A02000000000013
:10CCA000910F2000810F50003D0036004674A8000F
:10CCB000A2FD0700E24F500015013A00400020009D
:10CCC00020A2880042D4BF00D099020000000000DA
:10CCD00011102000810F50000D01360042D4BF001A
:10CCE00082C1B3000440BC00C03A210000004100F2
:10CCF000A20020008180E900180C02000000000062
:10CD00008000EB0030C0B30098FE07001ED5020083
:10CD1000000000000006BE0060A2800071A280003A
:10CD20006011B800A4252600250020006033B8005B
:10CD3000E4070200000000000205BE000004BE007F
:10CD40004A930200000000000100200002002000C1
:10CD500003002000A4252600250020006033B80031
:10CD600042090200000000000804400089844800D5
:10CD70000C0444008D844C0048A2880059A288000D
:10CD800050002000E100370042D4BF00BA9A0200F0
:10CD900000000000910F2000810F500013003E00A2
:10CDA0001ED502000000000042A2800053A28000B5
:10CDB00002005000838058004240A900D400340093
:10CDC00060A2800071A28000F2032000820F500058
:10CDD000E08F5800CC003E000000400081804800F9
:10CDE00060A2880071A28800C700370053FD0700C9
:10CDF000E54F5000B5003A0042D4BF00E097020072
:10CE00000000000042F4EF001ED502000000000008
:10CE100040A2880051A288006000200020A2880063
:10CE20004634A8004614A80063A380000308A300AA
:10CE30000A003200C0A28000D1A28000F2E9B7004F
:10CE40004801DE0002007800F3E9B7000100780035
:10CE5000F4E9B7004808DE00F5E9B7000328A300AD
:10CE60000A00320000A3800011A38000F6E9B70099
:10CE70004801DE0002007800F7E9B7000100780001
:10CE8000F8E9B7004808DE00F9E9B7000318A30085
:10CE90000A003200E0A28000F1A28000FAE9B700A7
:10CEA0004801DE0002007800FBE9B70001007800CD
:10CEB000FCE9B7004808DE00FDE9B7000338A3002D
:10CEC0000800320020A38000FEE9B7004800DE0021
:10CED000FFE9B70030A3800000EAB7004800DE0099
:10CEE00001EAB700026AEF00036AEF00046AEF008C
:10CEF000056AEF000348A3008500320040A38000CC
:10CF000002EAB7004800DE0003EAB70050A3800041
:10CF100004EAB7004800DE0005EAB7007C003700ED
:10CF20001ED502000000000048A2800059A2800027
:10CF30000800500089805800922526002300200018
:10CF4000820F5000838F580071003600320020009D
:10CF50000300200060A2800071A280008C03020008
:10CF60000000000082A2800093A28000800F510088
:10CF7000818F59000B003600A025260021002000DB
:10CF8000080040008980480040A2880051A2880023
:10CF900061005100E080590080A2880091A28800C1
:10CFA0005B00370034042000430420000041EB0004
:10CFB0006000B800129802000000000042F4B700C0
:10CFC000E14F4000520032007000200020A2880093
:10CFD00042D4BF00D09902000000000011102000D0
:10CFE000810F50004A0036001100200030C0B3000D
:10CFF000DEFD07004654A9001ED502000000000017
:10D000000006BE0060A2800071A280006011B8001E
:10D01000A4252600250020006033B800E4070200A4
:10D02000000000000205BE000004BE004A9302009A
:10D03000000000000100200002002000030020008A
:10D04000A4252600250020006033B8004209020014
:10D050000000000008044000898448000C044400DB
:10D060008D844C0048A2880059A288004434EC000A
:10D070002700370042D4BF00BA9A02000000000027
:10D08000910F2000810F50000D003E001ED50200C0
:10D090000000000042A2800053A280000200500065
:10D0A000838058004240A900190034004414EC0069
:10D0B00020A28800EC0F5000150036001200370047
:10D0C0009EFC0700E54F500003003200E64F500081
:10D0D0000F003A000C00370042D4BF00E097020076
:10D0E0000000000042F4EF001ED502000000000026
:10D0F00040A2880051A288006000200020A2880081
:10D100004634A800020037002000200020A288003A
:10D110004F06BE004F05BE004F04BE0000000600D3
:10D120008040EB0021D098006011B80012009800F8
:10D13000230098003200980043009800F0489000C7
:10D140000104A10071489800F04890000114A1006A
:10D1500071489800F04890000124A100714898009F
:10D16000F04890000154A1007148980011C0B3002C
:10D1700041C098000006B00052C104000000000049
:10D1800061C4B30011509800F1C6B300215098005B
:10D19000ECC0500031509800F2C04000415098005F
:10D1A00081C0E90051509800EEC0500061509800D5
:10D1B000EDC04000715098008040EB00015898008D
:10D1C00011589800215898003158980041589800FB
:10D1D00051589800615898004012900002102E009B
:10D1E000030020005200980063009800120098008D
:10D1F00023009800320098004300980012C4B30046
:10D2000002509800017898004178980001C8980071
:10D21000610520005110980061109800711098006D
:10D2200001189800111898004270980081C2B3004C
:10D2300021609800C1FF2F00010262000420A000BD
:10D240004410980000000600889FBE008A9FBE0020
:10D250008C9FBE008004780000309000E20F5000E8
:10D2600008003200794890000054A100F04C98006A
:10D27000794890000034A100F04C98000000EB00C9
:10D280001C00370019309000E10F50004A003A00AE
:10D29000098E9000EE0F560018003C001995900082
:10D2A000A995900079899000899190000A00BE00AC
:10D2B00030070200000000000000E00041003200E2
:10D2C000FA8C98008B9498000C0446002807B00054
:10D2D00002002400C36124000A00BE0034070200DB
:10D2E00000000000760602000000000000B47C0090
:10D2F0000C00E800808C9800320037002A072000DC
:10D30000090545006066B8008005EB001A04780046
:10D310006140B90054050200000000000800E00070
:10D3200004003D000200200003782400AC05020048
:10D33000000000000001BE000C00BE00AC050200B1
:10D34000000000000002BE000006BE008B05E800E1
:10D350000A85E800EF8F5500ECFF3A000000EB0073
:10D36000808C980002002000031724000400BE00F7
:10D37000AC060200000000009C0702000000000054
:10D380004200DD00A2002000110009000280D80048
:10D39000E292200000015100A28C9800820C7800DB
:10D3A000794890000054A000F04C98007948900013
:10D3B0000034A10002003700794890000054A10019
:10D3C000F04C98004F06BE004F05BE004F04BE0053
:10D3D00000000600881F78000004780010319000DB
:10D3E000E20F510004003200704890000034A100A8
:10D3F000704C98002E003700704890000034A00058
:10D40000704C9800784890000018A3002A003A0059
:10D4100038889000E10F50001A003200B890900058
:10D42000E20F50001C003200E0232000808F5000EB
:10D4300007003E00784890000018A3001E003A0044
:10D4400010002000308C98006011B80009003700EF
:10D45000502D2000808F5000170036007848900033
:10D460000018A30014003A00328C9800482990005C
:10D47000D829900008007800AA840200000000006B
:10D480000D003700B8909000E0232000808F5000FE
:10D490000900360003003700502D2000808F500017
:10D4A00005003E0008007800A28402000000000091
:10D4B0000000EB00308C98004F047800000006005C
:10D4C000881F7800000478000006B000E2C1020066
:10D4D0000000000051A980000100E80050A9880068
:10D4E000E18F50000700320003003900E28F500046
:10D4F000070032002A35EF000800780052FF0700CD
:10D500000600370008007800B2FF0700030037006C
:10D5100008007800E6C7020000000000080078005C
:10D52000C2850200000000004F04780000000600E1
:10D530000002BE000000E00004003D00D0C2B300C5
:10D54000804878000402EA0002003700B0C2B3004D
:10D550008048780042062000110009000202D8002D
:10D5600001C3B30081414000934298000280B9009A
:10D5700000005200A2002000801F78001100090066
:10D580000200D800000178004F00780001C3B3000A
:10D5900001424100A4429800E4C2B300B4429800A2
:10D5A0006A11B9000200500001404000C0429800DA
:10D5B0000040EB00D042980000000600E000FA00B6
:10D5C000889FBE008A9FBE008C9FBE0080047800AA
:10D5D00000F52F00000147007E289700CC00DE00F8
:10D5E000E1C0600041DF9900CB00DE00E1C06000D7
:10D5F00021DF9900CD00DE00E1C0600061DF99000D
:10D60000CA00DE00E1C66000C900DE0061C660003D
:10D610004800DE00E14560003E289700CE289700D4
:10D6200010079800210798001E289700AE28970041
:10D630003007980041079800120F780072054700E4
:10D64000A1142A00C7000900315D78008A0CB100DE
:10D65000CED99100E1806100CC08DD007E289700E2
:10D6600000C0A10001007000AED99100E18061000E
:10D67000CB08DD0000B0A10001007000EED99100E0
:10D68000E1806100CD08DD0000D0A1000100700044
:10D69000E1806600CA08DD0000A0A1000100700062
:10D6A000E1006600C908DD000090A10001007000E3
:10D6B000E1806500C808DD000080A1000100700065
:10D6C000702F9F001E009000AE009000302F9F0032
:10D6D000412F9F003E009000CE009000102F9F0031
:10D6E000212F9F001E0978007ED896000058A300C5
:10D6F0000C0032006A04470021142A0007000900C8
:10D70000315C78008800B1001E0078008800780045
:10D7100087FF0700881F780023212A00831F7800D5
:10D720000400370000222A00801F780021212A00EF
:10D73000811F78000A0078007A0C020000000000C7
:10D74000E4875700720447001901900011C0B3002C
:10D7500008007800020001003E009000CE0090001A
:10D76000809FBE0091222A00811F78000800780067
:10D770007A0C0200000000001901900011C0B300F3
:10D7800008007800020001001E009000AE0090002A
:10D79000809FBE0081232A00811F78000800780046
:10D7A0007A0C0200000000001901900011C0B300C3
:10D7B0000800780002000100E19F650073242A0040
:10D7C000831F7800080078007A0C02000000000037
:10D7D0001901900011C0B300080078000200010098
:10D7E000E11F660050252A00801F7800080078009D
:10D7F0007A0C0200000000001901900011C0B30073
:10D800000800780002000100E19F660031262A002E
:10D81000811F7800080078007A0C020000000000E8
:10D820001901900011C0B300080078000200010047
:10D83000EED99100E19F610010272A00801F780037
:10D84000080078007A0C0200000000001901900026
:10D8500011C0B3000800780002000100AED89100AA
:10D86000E19F6000F3272A00831F780008007800FA
:10D870007A0C0200000000000F02B10019019000B4
:10D8800011C0B30008007800020001004ED89100DA
:10D89000E11F6000D1282A00811F7800080078006D
:10D8A0007A0C0200000000001901900011C0B300C2
:10D8B0000800780002000100E48757004F06BE0010
:10D8C0004F05BE004F04BE000080FA0000000600B5
:10D8D000C800FA00889FBE008A1F78008004780084
:10D8E00020F32F000F004000B1292A00C7000900D3
:10D8F00031587800800CB10000F52F0021F32F0083
:10D900008F80400000844000F11F440032362A001E
:10D91000821F7800E0F22F000F0040007A0C020016
:10D92000000000001901900011C0B300E0F22F00C8
:10D930000F0040000200010048289000D828900005
:10D94000809FBE0011372A00811F780080F22F00CF
:10D950000F0040007A0C0200000000001901900046
:10D9600011C0B30080F22F000F0040000200010040
:10D970000F4895000000FB00801F780002382A0045
:10D98000821F780040F22F000F0040007A0C020046
:10D99000000000001901900011C0B30040F22F00F8
:10D9A0000F0040000200010008C890000000FB00CA
:10D9B000801F7800E0382A00801F780000F22F00D6
:10D9C0000F0040007A0C02000000000019019000D6
:10D9D00011C0B30000F22F000F0040000200010050
:10D9E000AA0220000805450018042000F28757000D
:10D9F000BA1F7800881F7800D1392A00811F78006B
:10DA0000C0F22F000F0040007A0C0200000000005E
:10DA10001901900011C0B300C0F22F000F004000A8
:10DA2000020001000804E800E687570060042000B7
:10DA3000800F5400EEFF3A0000F52F0022F32F0074
:10DA40000F01410000044100487090000000FB00FD
:10DA5000801F7800C03A2A00801F7800E0F22F0073
:10DA60000F0040007A0C0200000000001901900035
:10DA700011C0B300E0F22F000F00400002000100CF
:10DA8000481090000000D100E11F6000A13B2A0077
:10DA9000811F7800A0F22F000F0040007A0C0200D6
:10DAA000000000001901900011C0B300A0F22F0087
:10DAB0000F00400002000100286090000080FB0081
:10DAC000801F7800823C2A00821F780060F22F00BD
:10DAD0000F0040007A0C02000000000019019000C5
:10DAE00011C0B30060F22F000F00400002000100DF
:10DAF00048109000E11F6000603D2A00801F780000
:10DB000020F22F000F0040007A0C020000000000FD
:10DB10001901900011C0B30020F22F000F00400047
:10DB200002000100481090004200DE00E11F60008A
:10DB3000413E2A00811F7800E0F12F000F004000D5
:10DB40007A0C0200000000001901900011C0B3001F
:10DB5000E0F12F000F00400002000100F4875700A1
:10DB60004F0578004F04BE000080FA000000060058
:10DB70000000FA00889FBE008A1F78000005780028
:10DB8000810478000204780001012000020078007E
:10DB9000D0D70200000000000004E00005003A00B9
:10DBA0002100200009007800DCCB0200000000000A
:10DBB000100037007100450088007800080C020052
:10DBC00000000000AF0AB00060F52F00008447009D
:10DBD000540009003A1C7800A80AB100AA0AB10052
:10DBE000127802000000000088077800E87902003F
:10DBF000000000004F0578004F04BE000080FA00CE
:10DC0000000006000000FA00881F780080017800FC
:10DC10000102780092407800F0CBB30000C04000D1
:10DC2000E44F500005003600210020000400780079
:10DC3000DCCB0200000000000D003700C17198002D
:10DC4000AF0AB00060F52F000084470054000900BF
:10DC5000331C7800A80AB100A30AB10012780200B0
:10DC60000000000088077800E8790200000000004A
:10DC70004F0478000080FA00000006000000FA005F
:10DC8000881F780080037800810178008202780084
:10DC900092407800F0CBB30000C04000E44F500049
:10DCA0000B003E000100FB00F1FB2F0001034000D0
:10DCB00092409000B0C2B30080CF50000900320003
:10DCC0000084EB0000C0E80080CF50000600320066
:10DCD0002100200003007800DCCB020000000000DF
:10DCE0002400370018002000354190000201FB009D
:10DCF000400620000091B900254090000000FB0084
:10DD00000003B100843E20000480B90000014100FE
:10DD1000454090000000FB006A00B900000141008E
:10DD2000554090000000FB000001410000B32E00B0
:10DD30000001410006024300A402B0000890B900AF
:10DD400000B27B00AF0AB00060F52F0000844700EE
:10DD500054000900371C7800A80AB100A70AB100D6
:10DD6000127802000000000088077800E8790200BD
:10DD7000000000004F0478000080FA000000060058
:10DD80000000FA00881F7800000278008101780006
:10DD900010C4B300924F10000500320011002000A3
:10DDA00003007800DCCB0200000000000D0037000B
:10DDB00000529800AF0AB00060F52F0000844700C1
:10DDC00054000900341C7800A80AB100A40AB1006C
:10DDD000127802000000000088077800E87902004D
:10DDE000000000004F0478000080FA0000000600E8
:10DDF0000101780070489000110020000018A30075
:10DE0000050032005100200002007800DCCB020047
:10DE1000000000008000EB00010078000000060018
:10DE20000000FA00881F78008180FB008100EA0072
:10DE3000CF08DE0081804000401190000210A10058
:10DE40000101710042109800AF0AB00061F52F0087
:10DE50000184470054000900301C7800A80AB10072
:10DE6000A00AB100127802000000000088077800C4
:10DE7000E8790200000000004F0478000080FA00FA
:10DE8000000006000000FA00881F78002260980059
:10DE9000AF0AB00061F52F0001844700540009006B
:10DEA000301C7800A80AB100A00AB1001278020064
:10DEB0000000000088077800E879020000000000F8
:10DEC0004F0478000080FA00000006000000FA000D
:10DED000881F78008180FB008100EA00CF08DE0007
:10DEE000C208DD00401190000220A1000101710074
:10DEF00042109800AF0AB00061F52F00018447007E
:10DF000054000900301C7800A80AB100A00AB10032
:10DF1000127802000000000088077800E87902000B
:10DF2000000000004F0478000080FA0000000600A6
:10DF30000000FA00881F7800800178000102780054
:10DF4000704890000058A30005003A0071002000BE
:10DF500004007800DCCB0200000000000D00370058
:10DF600082C99800AF0AB00060F52F000084470016
:10DF700054000900331C7800A80AB100A30AB100BC
:10DF8000127802000000000088077800E87902009B
:10DF9000000000004F0478000080FA000000060036
:10DFA0000000FA00881F7800E180600040119000B6
:10DFB0000200A1000101710042109800AF0AB000F8
:10DFC00061F52F000184470054000900301C7800DF
:10DFD000A80AB100A00AB1001278020000000000F7
:10DFE00088077800E8790200000000004F047800FC
:10DFF0000080FA0000000600706B8800A10A200073
:10E0000080804000616B8800506B88000000060033
:10E0100062D7200021E0200000D72000A0D202001B
:10E020000000000020E020000000060000000600C4
:10E030000000EB002855E200020032002875EF00D6
:10E04000100020000000060060D72000000006003D
:10E05000881F78000004780072002000E19E2A00EA
:10E06000C40B0200000000000000E00008003200C5
:10E0700042002000619F2A0008007800C40B0200C3
:10E0800000000000010820000000E00001003A004C
:10E090008000EB00010078004F04780000000600CB
:10E0A000881F780001047800B19F2A00F80B020055
:10E0B000000000000000E00007003A0011A02A0064
:10E0C00008007800F80B02000000000001082000A2
:10E0D0000000E000010032008000EB000100780049
:10E0E0004F04780000000600889FBE00B1A02A00FF
:10E0F00000E32000D8450200000000000004780082
:10E100000000E00017003200C0C3B300984F1000B9
:10E1100014003A008004EB00E8C07C0000D7200027
:10E1200046D30200000000000000E00006003200BC
:10E13000E20F5000060032008904E800FE8F540010
:10E1400008003200F4FF370028F5B700050037005B
:10E1500010C0B30028F5B70000D72000AAD20200F3
:10E16000000000000000EB004F04BE0000000600AD
:10E170004A00FA00889FBE008A9FBE0000FB2F0065
:10E180000084470028CEBF004201200088007800AC
:10E19000AE820200000000009200200031A12A009F
:10E1A00008007800C40B0200000000000000E0003E
:10E1B00003003A00400120000000E900FEFF3A00A1
:10E1C0002201200001A22A0003FB2F000380470048
:10E1D000C40B0200000000000002EB000000E000A1
:10E1E000FC003A00A8708000B9708000CBE02000ED
:10E1F0000ACEBF000080FB004200DD000080E80086
:10E2000060C07D00E42E02000000000000057800E0
:10E210000ACEBF000080FB004200DD000080E80065
:10E2200060C07D00082F02000000000000004500D3
:10E2300001002000800F5400818F5C00DC003E0054
:10E240000ACEBF000080FB004200DD000080E80035
:10E2500060C07D00E42E0200000000006101B800F3
:10E2600014002000A0708000B1708000800F510069
:10E27000818F5900D70039003303200040FC2F0064
:10E28000008147006000200001002000D0C3020090
:10E29000000000000FB897000060A100A500370043
:10E2A0006100200000E32000384702000000000069
:10E2B0000000E000BE003A000107200060E32000FB
:10E2C00058470200000000000000E000B8003A00DB
:10E2D00008E3200031A32A0008007800F80B0200B0
:10E2E000000000000000E0000D003A0041FC2F009B
:10E2F000018447008800780060E320005294020007
:10E30000000000000000E000A900320018007800C2
:10E31000BFA09700C0AF9F00D1AF9F00860037001D
:10E3200061A32A0008007800F80B0200000000003A
:10E330000000E00003003A00C3FC2F008380470088
:10E340002200370091A32A0008007800F80B020091
:10E35000000000000000E0000D003A0080FC2F00EB
:10E36000008447008800780060E320005294020097
:10E37000000000000000E0008D003200180078006E
:10E38000DFA09700E0AF9F00F1AF9F006A00370069
:10E39000D1A32A0008007800F80B0200000000005A
:10E3A00001FD2F000000E0000700320021A42A0038
:10E3B00008007800F80B0200000000000000E000F8
:10E3C00008003A0041FD2F008180470060E32000F3
:10E3D00052940200000000000000E00056003A00E5
:10E3E0007300370071A42A0008007800F80B0200BF
:10E3F000000000000000E00033003A0063E320006A
:10E400000041780007CDB300F6CBB300F5C9B300E7
:10E4100044E1200008C3B300010037008301E80095
:10E42000934078000104E0000A00320007C0400079
:10E43000E94F50000E00360006C04000E54F500086
:10E440000B00360005C04000E54F5000F3FF3E00D2
:10E45000070037000280FB007C00400008707A0053
:10E460000241E800EB4F510008003E00F9FF370081
:10E470000280FB007C00400001707A008301E8000C
:10E480000241E800EB4F5100E5FF360008E32000B1
:10E490006F85570098407800F16F9F009841900079
:10E4A000E36F9F007F909700F2950200000000004C
:10E4B000005D78000884E800C0E32000800F54006D
:10E4C0001D003200F3FF3700B1A42A0008007800D5
:10E4D000F80B0200000000000000E0000A003A0013
:10E4E00060E32000429702000000000000FE2F00C1
:10E4F0000080470061E320000F00090031587800D8
:10E500000001B1000C00370001A52A0008007800C6
:10E51000F80B0200000000000000E00006003A00D6
:10E5200010C3B300364EE30003003A000FB8970063
:10E530000060A00080BF9F00A0708000B1708000CC
:10E54000E00F5000E08F580055FF3A0043FC2F00C9
:10E55000038447000800780042B502000000000074
:10E5600051A52A0000E32000080C02000000000072
:10E570007C04440040E420000F0009003858780073
:10E580000801B100546EEF0040E4200002C2B30065
:10E5900041E52000904F110001003A000048EB00D7
:10E5A0000000E800810F5000FAFF3A000600370033
:10E5B00010002000306B8800A1A62A0000E3200094
:10E5C000080C020000000000C000200060718800FC
:10E5D0000002EB00040078004F05BE004F04BE00AF
:10E5E0000080FA0000000600881F7800100020005C
:10E5F00000718800222EEF00C8E020000ACEBF0084
:10E600000080FB004200DD000080E80060407C00EC
:10E610009A2E020000000000F30F50000A0036009E
:10E62000202EEF00222EEF000ACEBF000080FB005C
:10E630004200DD000080E800E1A72A0060407C0085
:10E6400028440200000000004F047800000006008B
:10E650000ACEBF000080FB004200DD0031A92A0085
:10E66000E2E020006040790028440400000000003F
:10E67000881F7800C8E0200091A92A0000E320004C
:10E68000D845020000000000A2E0200012417800FE
:10E69000800078000000E000040032000280FB00EF
:10E6A0004200DD000080E800040037000280FB002B
:10E6B0004200DD000080E800E1A92A0060407C0003
:10E6C00028440200000000004F047800000006000B
:10E6D000881F78001000200000718800222EEF00B3
:10E6E000C8E020000ACEBF000080FB004200DD0031
:10E6F0000080E80060407C009A2E020000000000CC
:10E7000091042000810F50000A0036000ACEBF009D
:10E710000080FB004200DD000080E80061AA2A00C2
:10E7200060407C002844020000000000202EEF0022
:10E73000222EEF004F047800000006000800FA00C7
:10E74000889FBE006C84570000ACBE000D003700EF
:10E750006880570000405400E14F4000080032003C
:10E760000ACEBF000080FB004200DD000080E80010
:10E77000E1C2B30060C07C0042440200000000001F
:10E780000804E8001880FB00EC805700B8950200F0
:10E7900000000000C9E020000ACEBF000080FB009E
:10E7A0004200DD000080E800EC80570060C07C0083
:10E7B000284402000000000065805700800F5400CC
:10E7C000E3FF3A004F04BE000080FA00000006009C
:10E7D0000ACEBF000080FB004200DD00E1A0200067
:10E7E000E2E02000604079002844040000000000BE
:10E7F0001ECAAB00080032000ACEBF000080FB003A
:10E800004200DD00B1AB2A00E2E020006040790068
:10E81000284402000000000000000600239F2000A2
:10E82000934178008381FB00329F200012417800E1
:10E830004811DD0003007100439F200093417800E0
:10E840008381FB00529F2000124178004811DD00B7
:10E8500083007100B9FF3700A39F20009341780027
:10E860008381FB00B29F2000124178004811DD0037
:10E8700003007100C39F2000934178008381FB0057
:10E88000D29F2000124178004811DD008300710002
:10E89000AAFF3700639F2000934178008381FB002B
:10E8A000729F2000124178004811DD0003007100C2
:10E8B000839F2000934178008381FB00929F20007A
:10E8C000124178004811DD00830071009BFF370082
:10E8D000E39F2000934178008381FB00F29F20009A
:10E8E000124178004811DD000300710003A02000F0
:10E8F000934178008381FB0012A020001241780030
:10E900004811DD00830071008CFF370023A0200038
:10E91000934178008381FB0032A0200012417800EF
:10E920004811DD000300710043A0200093417800EE
:10E930008381FB0052A02000124178004811DD00C5
:10E94000830071007DFF3700889FBE008A1F78001A
:10E950000ACEBF000080FB004200DD00E1E02000A5
:10E9600060C078009A2E020000000000F10F5000F5
:10E97000030036000045EB00F9A120000F0037002E
:10E980001000200000718800222EEF0027003700C1
:10E990000A04E000080032000ACEBF000080FB003D
:10E9A0004200DD000080E800A1C3B30060407C00AD
:10E9B00042440200000000008904E8001940780089
:10E9C0004E9602000000000080407800C8E0200061
:10E9D0000ACEBF000080FB004200DD000080E8009E
:10E9E00060407C00424402000000000019407800B2
:10E9F0006296020000000000804078000ACEBF004E
:10EA00000080FB004200DD000080E80060407C00E8
:10EA100042440200000000000A45E800E64F5500AD
:10EA2000DBFF3A00202EEF00222EEF004F0578008A
:10EA30004F04BE00000006000000060000000600B3
:10EA40000000FE00000006000ACEBF000080FB00B0
:10EA50004200DD0001E32000E2E020006040790098
:10EA6000284404000000000000000600000006002A
:10EA700000000600000006000ACEBF000080FB0078
:10EA80004200DD0031AC2A00E2E020006040790065
:10EA90002844040000000000881F7800C8E020001F
:10EAA0000ACEBF000080FB004200DD000080E800CD
:10EAB00060407C009A2E020000000000A1042000AB
:10EAC000810F500004003E001000200000718800FB
:10EAD000222EEF000A0037000ACEBF000080FB00A4
:10EAE0004200DD000080E80081AC2A0060407C002C
:10EAF0002844020000000000202EEF00222EEF002C
:10EB00004F047800000006000ACEBF000080FB0022
:10EB10004200DD00F1AE2A00E2E020006040790012
:10EB200028440400000000000ACEBF000080FB0063
:10EB30004200DD0041AF2A00E2E0200060407900A1
:10EB40002844040000000000C2E020000ACEBF00FC
:10EB5000680DE200050032000080FB004200DD008D
:10EB60000080E80041AF2A00040037000080FB006D
:10EB70004200DD000080E800F1AE2A00604079002C
:10EB80002844020000000000682DEF00000006008D
:10EB9000C2E020000ACEBF00660DE2000500320090
:10EBA0000080FB004200DD000080E80041AF2A0049
:10EBB000040037000080FB004200DD000080E80018
:10EBC000F1AE2A00604079002844020000000000F5
:10EBD000662DEF0000000600716B8000F1804000A0
:10EBE0000ACEBF000080FB004200DD00E2E0200012
:10EBF0006040790028440400000000000800FA008A
:10EC000068805700A1AF2A0006000900315878003B
:10EC10007000B100706B800010019000A0019000A6
:10EC2000829FBE0013B02A00831F78006E805700B9
:10EC30007A0C0200000000000ACEBF000080FB003A
:10EC40004200DD00EE805700E2E0200060407900E5
:10EC50002844020000000000E68757000080FA0008
:10EC6000000006000600FA006680570051B02A0036
:10EC700005000900315878006000B100706B800019
:10EC800010007800E6805700986A0200000000003B
:10EC90000ACEBF000080FB004200DD00E680570086
:10ECA000E2E02000604079002844020000000000FB
:10ECB0000080FA00000006000200FA000000EB00ED
:10ECC000F0BF9F00706B800000C890000043B00050
:10ECD000E0FF9F000ACEBF000080FB004200DD0085
:10ECE0008F80E900E2E020006040790028440200C3
:10ECF000000000000080FA00000006000600FA0094
:10ED000066805700B1B02A0005000900315878002C
:10ED10006000B100706B800040289000E6805700D2
:10ED2000B8950200000000000ACEBF000080FB0082
:10ED30004200DD00E6805700E2E0200060407900FC
:10ED400028440200000000000080FA0000000600D5
:10ED50000800FA00606B80001000BE0012A80200DC
:10ED6000000000000001BE00606B800030109000C9
:10ED70000028A3000400320000E427005100200016
:10ED800002015000838158006880570011B12A00A9
:10ED900006000900315878007000B100829FBE0063
:10EDA00010B02A00801F78006E8057007A0C020095
:10EDB000000000000ACEBF000080FB004200DD0022
:10EDC000EE805700E2E02000604079002844020015
:10EDD00000000000E68757000080FA0000000600EF
:10EDE0000600FA006680570081B12A00050009007C
:10EDF000315878006000B100706B800040289000AE
:10EE0000E6805700B8950200000000000ACEBF005F
:10EE10000080FB004200DD00E6805700E2E02000B9
:10EE20006040790028440200000000000080FA00E1
:10EE300000000600616B8000EE8040000ACEBF003B
:10EE40000080FB004200DD00E2E02000604079002D
:10EE50002844040000000000606B80001000BE0029
:10EE600012A80200000000000001BE00606B8000DC
:10EE7000301090000028A3000400320000E42700B6
:10EE80005100200002015000838158000200BE00A2
:10EE900000000600C482A800201220001013880081
:10EEA0000000280000138800000006000000FA009F
:10EEB00000C0EB0099F2B7009AF2B7009BF2B700DE
:10EEC0009CF2B7009DF2B7009EF2B7009FF2B70028
:10EED000A0F2B700A1F2B700A2F2B700A3F2B70008
:10EEE000A4F2B700A5F2B700A6F2B700A7F2B700E8
:10EEF000A8F2B700A9F2B700AAF2B700ABF2B700C8
:10EF0000ACF2B70060FB2F0000824700AFC2970051
:10EF10001401BE000580FB004200DD0081292100B4
:10EF20000100400012409800C810DE002140980007
:10EF300033409800C818DE00414098000500780072
:10EF400098F2B7006E00420061282100100009000D
:10EF5000B05878001001B1005FD0970085F2B7007B
:10EF60000460900097F2B700341090000000D100C8
:10EF7000614060004300DD00312B210091407800AA
:10EF80000134A10080C0700001007800B3F2B70026
:10EF9000341090004200DE00614060004400DD005B
:10EFA0000144A10080C0700001007800B3F2B700F6
:10EFB00024609000AFF2B70034609000B0F2B70068
:10EFC00044609000B1F2B70054609000B2F2B70014
:10EFD00034109000614060004500DD000154A10044
:10EFE00080C0700001007800B3F2B7002478900070
:10EFF000ADF2B70034789000AEF2B7003FC0970092
:10F000004200DE00610060004700DD000174A100E5
:10F0100080C0700001007800B3F2B7000080FA00F1
:10F02000000006000000FA0000C0EB0071F2B7001B
:10F0300072F2B70073F2B70074F2B70075F2B7005E
:10F0400076F2B70077F2B70078F2B70079F2B7003E
:10F050007AF2B7007BF2B7007CF2B7007DF2B7001E
:10F060007EF2B7007FF2B70080F2B70081F2B700FE
:10F0700082F2B70083F2B70084F2B70000F52F00E8
:10F0800000824700EFDA96001F299700AF2997000A
:10F090000580FB004200DD00012721000100400047
:10F0A00012409800C810DE002140980033409800BC
:10F0B000C818DE00414098000500780070F2B700E3
:10F0C0000478900050F2B7004478900065F2B700E1
:10F0D00084C89000E1C06000E2CFB300B3D2BF00AB
:10F0E0000240600001407000B3F2B70071004200BE
:10F0F0002123210010000900B05878001001B10050
:10F10000A0022000040040003003BE0036928800B8
:10F11000479288003003BE005692880067928800AC
:10F1200010007800709288004470900045F2B7009B
:10F130000FE0960031F2B700246090000080FB00E1
:10F1400043F2B7004472EF00441090000000D10079
:10F15000614060004200DD00312B210091407800C9
:10F160000124A10080C0700001007800B3F2B70054
:10F170004410900061406000004040000114A10074
:10F1800080C0700001007800B3F2B7004410900016
:10F190004200DE00614060004600DD000164A10025
:10F1A00080C0700001007800B3F2B700FFD896006D
:10F1B000C208DE00E1806000B4D2BF0002406000FF
:10F1C00001407000B4F2B7000080FA0000000600B1
:10F1D0000000FA006FF0950030F2B7000080FA00EE
:10F1E000000006000080FB004013880060C2BF00E2
:10F1F0000008A300FDFF3200401380000080FB00E8
:10F2000000000600C482A90050C0B300F5FF07004B
:10F210000040EB00F3FF0700C482A8000080FB0061
:10F2200000000600889FBE0080447800F5FF0700BC
:10F2300063046000FDFF3A00C482A90030C0B3003F
:10F24000E8FF070009407800E6FF07000840780063
:10F25000E4FF0700C482A8000080FB004F04BE004A
:10F2600000000600889FBE008A9FBE008044780090
:10F270008105780002457800E2FF07006304600022
:10F28000FDFF3A00C482A90030C0B300D5FF0700DB
:10F2900009407800D3FF0700880478000500370094
:10F2A0000040EB00CFFF07008880FB0080F07D006E
:10F2B0008904E800094478008ACF5400F8FF390037
:10F2C000C482A8004F05BE004F04BE000000060027
:10F2D00092C8B300C1222100E2FF3700C482A90016
:10F2E00060C0B300BFFF0700C482A8000000060092
:10F2F000889FBE008A9FBE00804478000105780088
:10F3000082457800BFFF070063006000FDFF3A0000
:10F31000F2FF0700C482A90020C0B300B1FF0700BC
:10F3200009407800AFFF07000A0478000F0037009B
:10F3300038407800ABFF07008944E8006F80640024
:10F340000A003A00C482A800AEFF07000008A3002C
:10F35000FDFF3A00E1FF0700C482A90020C0B3000E
:10F36000A0FF0700094078009EFF07000A405400F4
:10F370008B4F5000EEFF3900C482A800A1FF0700A8
:10F380000008A300FDFF3A004F05BE004F04BE0079
:10F390000000060092C8B300C122210010C0B300D3
:10F3A000D3FF3700C1222100914078008180FB000B
:10F3B0002DD2BF004800DD00010070000000E80011
:10F3C0002CF2B7004800DE002DF2B700F1FF370045
:10F3D000B0C0B3002CF2B7002D72EF00EDFF370084
:10F3E000889FBE00004478008144780085FF0700B4
:10F3F00063006000FDFF3A00B8FF0700C482A90067
:10F4000020C0B30077FF07000840780075FF0700B1
:10F410000940780073FF0700C482A8004F04BE00B3
:10F4200000000600804078002EF2B70030C0B30024
:10F43000EBFF3700889FBE008A9FBE008C9FBE00F6
:10F440008E1F78006055B800000778004E49900084
:10F45000C42221000281FB004211DD00902921001D
:10F4600000004100840450001E00BE00C206B0002F
:10F470000401410010419800C801DE0023419800BA
:10F48000314198004808DE004041980084864400DD
:10F490001800200009404400BD407800D0FF07005C
:10F4A0000804E800E50F5400FAFF3A001E00BE0011
:10F4B00040079800510798000940E80059FF0700ED
:10F4C0000080FB0008F02F000805650000057500AE
:10F4D00009C0E80053FF07004800DD00FA0FB20042
:10F4E0000005750063C044004EFF07000080FB006C
:10F4F000888565008085750064C0440049FF070069
:10F500004800DD00FB0FB20080857500CE4A9000F8
:10F510008580FB00C208DD0080292100808040003A
:10F52000114290000482FB00214090004800DD0061
:10F5300004017000314290000482FB0041409000C1
:10F540004800DD0084017000820F5500838F5D004C
:10F55000030032000540E800404F9800BBFF370031
:10F560004F0778004F06BE004F05BE004F04BE0097
:10F5700000000600889FBE008A9FBE008C9FBE00D0
:10F580008E1F78006055B800000778006E49900023
:10F59000C42221000281FB004211DD00102721005E
:10F5A00000004100840450001E009000AE00900056
:10F5B0004204B0000401410010419800C801DE007F
:10F5C00023419800314198004808DE0040419800EE
:10F5D000848644001800200009404400BD407800A3
:10F5E0007FFF07000804E800E50F5400FAFF3A0027
:10F5F0001E009000AE009000500798006107980030
:10F600000940E80007FF07000080FB0008F02F001A
:10F61000080565000005750009C0E80001FF070046
:10F620004800DD00FA0FB2000005750063C0440019
:10F63000FCFE07000080FB00888565008085750062
:10F6400064C04400F7FE07004800DD00FB0FB20075
:10F6500080857500EE4A90008580FB00C208DD00C1
:10F660000027210080804000114290000482FB00AE
:10F67000214090004800DD000401700031429000FC
:10F680000482FB00414090004800DD0084017000CE
:10F69000820F5500838F5D00030032000540E800B3
:10F6A000604F9800B9FF37004F0778004F06BE0043
:10F6B0004F05BE004F04BE0000000600889FBE003C
:10F6C0008A9FBE008C9FBE008E1F78006055B800D8
:10F6D000000778000E7990000281FB004211DD00E6
:10F6E0001025210000004100C122210081045000AA
:10F6F0004202B000010141003E18900001002000CC
:10F70000104198004800DE00204198000000EB0006
:10F710003041980040419800C22221008286440076
:10F720001800200009404400BD4078002CFF07006D
:10F730000804E800E50F5400FAFF3A000940E80029
:10F74000B8FE07000080FB0008F02F0008056500E8
:10F750000005750009C0E800B2FE07004800DD00A2
:10F76000FA0FB2000005750063C04400ADFE07004B
:10F770000080FB00888565008085750064C04400BA
:10F78000A8FE07004800DD00FB0FB2008085750071
:10F790008E7A90008580FB00C208DD0000252100E4
:10F7A00080804000114290000482FB0021409000C4
:10F7B0004800DD0004017000314290000482FB002B
:10F7C000414090004800DD0084017000820F550028
:10F7D000838F5D00030032000540E800007F980041
:10F7E000BCFF37004E7890000080FB000000400016
:10F7F0006126210081004000C222210002845000C5
:10F80000A003B00082007800020040002E79900032
:10F81000024878003E7990001240980001064400AA
:10F820001900200008C04400BC407800ECFE07002E
:10F830008904E800E38F5400FAFF3A000840E8002A
:10F8400078FE07000080FB0001F02F000105650035
:10F850000005750008C0E80072FE07004800DD00E2
:10F86000FA0FB20000057500CE7990000380FB000E
:10F870000000400061262100010040001081FB00D3
:10F88000104090004800DD0002007000CF80DE00D4
:10F89000800F5500818F5D00030032000340E800B7
:10F8A000407F9800CFFF37004F0778004F06BE001B
:10F8B0004F05BE004F04BE0000000600D10220002C
:10F8C0008080400062C0B300A0CFB30065FE370067
:10F8D000889FBE008A1F78000004BE0002057800E1
:10F8E000C482A80020122000101388000000280005
:10F8F0000013880010C0B30075FE0700C12221006C
:10F90000914078008180FB002DD2BF004800DD00CF
:10F910000100700011002000EB0F5000C0003A0001
:10F9200071004400212321001000090031587800A3
:10F930001001B100A00220000800400032928000B7
:10F94000439280000298BE00529280006392800031
:10F950000298BE00739280000308780045D2BF0071
:10F9600040749800B3D2BF006140600000CC9800A2
:10F9700010C0B30040C498001123210091407800CA
:10F9800001549800412B21009140780080C0600014
:10F99000C208DD00784890000024A10001407000FA
:10F9A000704C9800322421001241780022649800A3
:10F9B000B3D2BF000000D10062006000C812900006
:10F9C0000510A100808272004514980001272100D3
:10F9D00091407800614C98008180FB00C208DD00F6
:10F9E0004104B000C62221008680400011429000F0
:10F9F0000482FB00214090004800DD0004017000FB
:10FA0000314290000482FB00414090004800DD003C
:10FA10008401700052049800630498000200BE0044
:10FA200010049800210498003004980041049800C4
:10FA300065D2BF00407C98000080FB0000004000C1
:10FA4000A003B000060040009080FB001040900032
:10FA50004800DD0001007000501C980001252100C5
:10FA600091407800017C98008180FB00C208DD0095
:10FA70004102B00086804000114290000482FB00E9
:10FA8000214090004800DD0004017000321C980005
:10FA9000B3D2BF000000D100610060000500A100EA
:10FAA0008082720045149800B3D2BF004400DE008B
:10FAB000640060000520A100808272004514980057
:10FAC0006E8044006328210010000900335878003C
:10FAD0001001B10085D2BF00F05C9800B3D2BF0026
:10FAE0000080FB004700DE004200DD00D9489000A6
:10FAF0000124A10080C07000D14C980097D2BF00B3
:10FB00000080FB0080149800B3D2BF004200DE00EA
:10FB100062006000B91290000510A100808272009E
:10FB2000B51498008129210091407800C14C9800BB
:10FB30008180FB00C208DD00C106B0008680400065
:10FB4000114290000482FB00214090004800DD003B
:10FB500004017000314290000482FB00414090009B
:10FB60004800DD0084017000C2049800D3049800AE
:10FB700049019000D9019000828CBE00A204980037
:10FB8000B3049800B3D2BF004200DE0064006000FE
:10FB90000520A10080827200B5149800B3D2BF0086
:10FBA0004500DE00610060000500A1008082720057
:10FBB000B5149800F12A2100914078008180FB0063
:10FBC000B0D2BF004800DD0001017000112B210000
:10FBD000914078008180FB00B2D2BF004800DD0078
:10FBE0008101700092149800A3149800E122210072
:10FBF00091407800C17C9800D12A21009140780082
:10FC00008180FB00AED2BF004800DD000100700023
:10FC1000D01C980030D2BF00004D78008000EB006F
:10FC2000010078004F0578004F04BE000000060078
:10FC3000804078000040E900E64F500007003E0099
:10FC400001407800A2C0B3000440BC006035210030
:10FC5000000141000099EB000091EB00000006005C
:10FC6000889FBE008A1F780001057800E74F50008A
:10FC700036003E00A2C0B3000440BC000200780081
:10FC800061352100810441001901BE00E10F4100EE
:10FC9000E08F49002D003200640040000104400064
:10FCA0001800BE00E00F5000E08F5800270032001F
:10FCB0000A00E00009003A001400200005002000BE
:10FCC000841C4100859449000080EB008080EB009B
:10FCD000180C4000589448001A003700B49980006E
:10FCE000C599800061004200E0804A00800F510009
:10FCF000818F5900050032009208B0000380B000E7
:10FD00000200BE00BEC302000000000064C4020086
:10FD100000000000004D78001900BE00B099880076
:10FD2000C19988001200200003002000821C4000BE
:10FD3000839448000082EB008082EB00180C4200A4
:10FD400058944A0010002000010037000000EB002A
:10FD50004F0578004F04BE0000000600889FBE00DB
:10FD60008A9FBE008C1F780001037800020578008E
:10FD7000E74F500029003E00A2C0B3000440BC0081
:10FD8000020278006400410065352100050640004C
:10FD90001C01BE006150B800820F5000838F5800D4
:10FDA0000100360002057800850542001B00BE00F8
:10FDB000E10F4000E08F4800180032000A00E00028
:10FDC000160032006154B8000600E00005003A0059
:10FDD000881D4000899548001C1E14001C961C00BC
:10FDE0000C0037009008B0000180B0008A01780054
:10FDF00006017800D0C30200000000009B0D440003
:10FE0000DB954C001C1E14001C961C0036B3EF0042
:10FE100038B3EF000A017800010037000001EB0061
:10FE2000020078004F0678004F05BE004F04BE0068
:10FE300000000600881F780000047800E099800028
:10FE4000800F540012003200D2998000820F5400BB
:10FE50000F00310060012000D09A88005C33EF0071
:10FE60006B40B90000004100000040006800400005
:10FE700001002000B09A8800C19A88006201200029
:10FE8000E13321000040EB00B4FF0700E89988004F
:10FE90004F04780000000600889FBE0080047800B0
:10FEA000A09A8000E10F500024003200D099800019
:10FEB000808F540021003E0018C0B300003621009E
:10FEC0000081EB008081EB00B00F1100A08F1900C2
:10FED000050032000844E8006A004000E84F540082
:10FEE00003003200F8FF3700E74F540013003200E0
:10FEF00009007800CFFF07008881FB0008407800E8
:10FF0000A2C0B3000440BC00E800410060352100FD
:10FF10008930780080004100149A8000259A800082
:10FF20008488BE0001017800309A8000419A8000E8
:10FF3000200198003101980001003700F30F2000E4
:10FF4000030078004F04BE00000006001200FA0013
:10FF5000889FBE008A9FBE008C9FBE00000678006E
:10FF60000040EB00A0E79F001C04E00061003200AD
:10FF7000A09A8000E10F50005E0032008C007800F3
:10FF80008006EB00040037000080FB000080460084
:10FF9000800640008100E800114078000004E00085
:10FFA000F9FF3A001BC0B300003621000081EB00CE
:10FFB0008081EB00B00F1100A08F19000500320006
:10FFC0008B45E8006A004000E8CF5500440032004D
:10FFD000F8FF3700E7CF550041003A0045003700F1
:10FFE0008B81FB000B407800A2C0B3000440BC0032
:10FFF0006135210001004100149A8000259A80009B
:020000040001F9
:100000000488BE00349A8000459A8000240098003D
:10001000350098006801410009B1780036003700CA
:10002000678464000A003A006150B800B09A880002
:10003000C19A880005012000D59A88005C33EF0042
:1000400002012000FC8057000840780043FF0700B1
:1000500008004400FC805700608078008D0F50003D
:100060001C003A000900780072FF0700F099800038
:10007000019A8000B09A8800C19A8800F10F200090
:10008000D19A88005C33EF000C0478000700370039
:10009000FE8057000040EB00F1FE07002FE29700C2
:1000A000984F120003003A000804E8001804E0002A
:1000B000F7FF3A00FE8057000040EB00E8FE070023
:1000C000AFE297000504E00002003A001804E000E7
:1000D000C3FF32008904E8000A85E8000200370007
:1000E0008004EB008A002000D0998000808F5400AB
:1000F000CBFF3900F30F2000030078004F06BE004D
:100100004F05BE004F04BE000080FA00000006004C
:100110004200200011FF0700800078000120A200AB
:100120000100EA00010070004F00DE0061001000D5
:1001300000000600E74F500010003E00A2C0B300D0
:100140000440BC00820178006435210004014100B4
:100150000080EB008080EB00B20F1000A28F18002F
:10016000060032006880410060007A0031FF07001D
:10017000309A8000419A80000000060001002000B3
:1001800000000500004178006000B800E74F510012
:1001900012003E0002407800A2C0B3000440BC0040
:1001A0008200780064352100040041000081EB00EA
:1001B0008081EB00B00F1100A08F190002003A00FF
:1001C0000200BE00000006006880400060007A0067
:1001D00018FF0700109A8000219A80000000060096
:1001E000E74F500014003E00A2C0B3000440BC0022
:1001F0008201780064352100040141000080EB0099
:100200008080EB00B20F1000A28F18000A003200AD
:100210006880410060007A0006FF0700309A800085
:10022000419A8000129A8000239A800002004000C8
:1002300083804800000006000080EB008080EB0017
:1002400000000600889FBE008A9FBE008C9FBE00F3
:100250008E1F7800004578000204BE000106780079
:10026000E74F50004C003E00A2C0B3000440BC0069
:100270000207780060352100800541001B01BE00A7
:10028000E10F4100E08F490043003200E18F500050
:100290003200320005003900E28F500013003200B6
:1002A000E38F50003C003A001C0037000A40780001
:1002B000A0FF07000006BE00800F5400818F5C0085
:1002C00035003E000A407800AEFF0700881D400060
:1002D0008995480064004700613521000100400015
:1002E0000818560009905E000A00370064004700B5
:1002F0006135210001004000B00F5400A08F5C0068
:1003000025003E00881D4100899549001018140001
:1003100010901C0011002000200037000A407800D7
:1003200098FF07001B01BE000000440081804C00C4
:10033000800F5100818F590017003900881D51002E
:100340008995590064004700623521000200400091
:100350001008440050904C00EEFF37000A4078002F
:1003600074FF0700800F5400818F5C000A003E007C
:100370000A4078009AFF0700881D500089955800B0
:1003800061352100010047002800980039009800DD
:100390008C007800010037008000EB00010078003D
:1003A0004F0778004F06BE004F05BE004F04BE0049
:1003B0000000060060352100C13921000098EB00E3
:1003C0000090EB006A004000810F5000FBFF3A00F4
:1003D00010002000A09A88005633EF005833EF0039
:1003E0005EB3EF00623521001241780069014100DF
:1003F000F203B200000420000100200002005000BF
:10040000E0805800D09A8800E19A88009008200087
:1004100001002000C8C3020000000000F10F20000E
:100420000000E00001003A00800078000100780040
:1004300000000600E74F500010003E00A2C0B300CD
:100440000440BC00820178006435210004014100B1
:100450000080EB008080EB00B20F1000A28F18002C
:10046000060032006880410060007A0071FE0700DB
:10047000509A8000619A8000000006000100200070
:1004800000000500E74F500010003E00A2C0B3007E
:100490000440BC0082017800643521000401410061
:1004A0000080EB008080EB00B20F1000A28F1800DC
:1004B000060032006880410060007A005DFE07009F
:1004C000709A8000819A80000000060001002000E0
:1004D00000000500E74F50000F003E00A2C0B3002F
:1004E0000440BC0082017800643521000401410011
:1004F0000080EB008080EB00B20F1000A28F18008C
:10050000050032006880410060007A0049FE070063
:10051000909A80000000060000000500E74F5000A0
:100520000C003E00A2C0B3000440BC0064352100B2
:10053000040141000080EB008080EB00B20F10004E
:10054000A28F18000300320022009000B200900039
:10055000000006000100200000000500889FBE008A
:100560008104780002047800E74F50001A003E0032
:10057000A2C0B3000440BC008201780064352100B1
:10058000040141000080EB008080EB00B20F1000FE
:10059000A28F1800100032006880410060007A00CD
:1005A00024FE0700F0998000019A8000B09A88002C
:1005B000C19A8800F10F2000D19A88005C33EF00C7
:1005C00008017800890078000040EB00E3FD070097
:1005D00010002000010037000000EB004F04BE00B7
:1005E00000000600889FBE00A2C0B3000440BC000B
:1005F00061352100010141001204BE00E1FE070047
:100600000004540081845C000800BE004F04BE005A
:1006100000000600A2C0B3000440BC006801410015
:100620006035210062007800000006005633EF00BC
:100630005833EF0080002000D09A88005C33EF0030
:1006400062002000E13321000040EB00C3FD070001
:100650006200200041E22A00E0332100C40B0200C6
:10066000000000000000E00004003A00220020002A
:10067000A1332100B9FD0700010037003A33EF0034
:100680003CB3EF0000000600881F780000047800EB
:100690005433EF00B2C50200000000009CC4020009
:1006A000000000000000E000FCFF3A000800E0004D
:1006B00001003200DDFF07004F0478000000060053
:1006C000889FBE008A9FBE008C9FBE008046780037
:1006D00001067800820578000005EB002400370051
:1006E0006C407D00BAC50200000000000D4078009B
:1006F000A2C0B3000440BC006035210000044100EA
:100700001400200005002000180C420058944A00F4
:1007100064014100800441000081EB008081EB0016
:1007200039004100A9804900808CBE00E00F5000D4
:10073000E08F58000D003A000000EB00D2FF0700E8
:1007400010002000A09A88009408200005002000D6
:1007500038004200A8804A00C8C302000000000020
:100760000004200001002000808CBE000A05E80083
:100770008B0F5500DAFF39000A0078004F06BE00E3
:100780004F05BE004F04BE000000060000362100E9
:10079000613A21000098EB000090EB006A004000F5
:1007A000810F5000FBFF3A00A6C3020000000000CA
:1007B00036B3EF0038B3EF009CFF07005433EF006F
:1007C0000000060000017800800C200060299800DD
:1007D00000192000702998008250900010C4B300C6
:1007E00080CF500005003A0000202C0011002000AE
:1007F00040299800512998000000060020C4B30049
:1008000080CF500004003A0000202C00110020008E
:10081000402998005129980000000600881F7800A0
:1008200000047800C0009000300090001004980090
:10083000210498008000EB0010C0B30094C00200B7
:1008400000000000C112200010C0B3000EC1020061
:1008500000000000784890000004A100704C98004F
:10086000784890000014A100704C980078489000DF
:100870000024A100704C9800FD74EF004F04780034
:1008800000000600881F7800000478008000EB005C
:1008900010C0B30094C0020000000000784890002F
:1008A0000004A100704C9800784890000014A1004A
:1008B000704C98000040EB00FCF4B700FDF4B7006A
:1008C00008007800BA7A0200000000004F047800A7
:1008D00000000600881F780000047800A000900047
:1008E0001000900030049800410498008000EB0054
:1008F00010C0B30094C0020000000000C11220002C
:1009000010C0B3000EC10200000000007848900043
:100910000004A100704C9800784890000014A100D9
:10092000704C9800784890000024A100704C98000A
:100930000040EB00FCF4B700FDF4B7004F04780072
:100940000000060030C0B300FCF4B700FD74EF00F7
:100950000000060011C0B30041C09800522098006A
:100960006320980020C0B300FCF4B700FD74EF00D2
:10097000000006008000780070489000624160002E
:1009800005003A0010C0B300C0C09800FCF4B700E6
:1009900002007800FDF4B7000000060012C0B300AA
:1009A00042C09800D24F210012417800100320006D
:1009B000808F500007003A006F405100E14F500017
:1009C00002003E0050C0B3000600370050C0B30024
:1009D000080037006D405100E14F500004003E0018
:1009E00060C0B300FCF4B700FD74EF000000060027
:1009F00060C0B300FCF4B7000000060010019000D6
:100A0000A001900032009800430098009DFF37003D
:100A10000000FA00889FBE0080047800401090001B
:100A20000008A30003003200794890000058A3009A
:100A300006003A00794890000024A000F04C98008D
:100A4000794890000014A10033003700A9D290002B
:100A50000504E00028003A0059199000190111001E
:100A6000497090000000FB000000400009004000B9
:100A7000409097000091B900A400200011000900E7
:100A80000401D800000178006110B9003919900004
:100A900002014000E081480049289000D9289000D8
:100AA000800F5100818F5900010036000001BE0007
:100AB000794890000024A000F04C980079489000FC
:100AC0000014A100F04C9800794890000004A100A7
:100AD000F04C980010C0B300C0C49800D224980015
:100AE000E324980020C0B300FCF4B70005007800B0
:100AF000FDF4B70012003700794890000024A000F0
:100B0000F04C9800794890000014A100F04C980037
:100B1000794890000004A100F04C98005901900021
:100B2000E901900010C0B300C0C49800D22498001E
:100B3000E324980020C0B300FCF4B700FD74EF007C
:100B4000AF0AB00060F52F00008447005400090090
:100B5000391C7800A80AB100A90AB1001278020075
:100B60000000000088077800E8790200000000001B
:100B700010C0B300A0D498004F04BE000080FA005B
:100B8000000006000000FA00889FBE008004780084
:100B9000FDD4BF000000FB00CF80DE00F00F50004E
:100BA000E08F5800D0013E000060010010003700C7
:100BB000CB003700F6003700080137001701370077
:100BC000C9013700C801370024013700640137002C
:100BD000C5013700C4013700C3013700C201370027
:100BE00095013700B7013700A4013700B501370080
:100BF000FCD4BF00BC013200E34F500012003A00A9
:100C000019009000A9009000B0049800C104980059
:100C10008000EB0010C0B30094C002000000000090
:100C2000794890000014A100F04C98007948900099
:100C30000004A100F04C98000040EB0080CC98002C
:100C4000FCF4B700A8013700E64F50000E003A0050
:100C5000E115200010C0B30094C0020000000000A5
:100C6000C112200010C0B3000EC10200000000003D
:100C700049289000D9289000B0049800C104980039
:100C8000F0C0B3000E003700E54F500013003A00EB
:100C9000E115200010C0B30094C002000000000065
:100CA000C112200010C0B3000EC1020000000000FD
:100CB0006000B800B0049800C1049800D0C0B30030
:100CC000FDF4B700FC74EF001ED502000000000028
:100CD000A02C9800B12C980083013700E14F500000
:100CE00076013200E24F500030003A00E11520005A
:100CF00010C0B30094C0020000000000C112200028
:100D000010C0B3000EC102000000000019009000E6
:100D1000A9009000C0A78800D1A7880049109000C2
:100D20000018A30008013200296390000604E000C7
:100D30000501320059219000E9219000492A9000D4
:100D4000D92A9000840F5100858F5900FE0032008F
:100D500019009000A9009000800F5100818F590068
:100D6000F90036000680FB00010020000200400070
:100D700083804800840F5000858F580003003600A0
:100D8000F4249800852C980002003700F024980085
:100D9000812C98007920900089289000B004980058
:100DA000C104980070C0B30044013700E44F500004
:100DB0004D013A0079489000624460000200320020
:100DC000FC74EF004801370059209000E9209000A2
:100DD000E00F5000E08F580018003A001900900012
:100DE000A9009000E00F5000E08F58003200320060
:100DF000794890000004A000F04C9800E115200014
:100E000010C0B30094C00200000000008125200043
:100E100010C0B3000EC102000000000039009000B5
:100E2000C900900061005000E0805800B0049800B4
:100E3000C104980090C0B300190037001901900058
:100E4000A901900049289000D9289000800F5100F6
:100E5000818F590018003100794890000004A000EB
:100E6000F04C9800E115200010C0B30094C00200BF
:100E7000000000008125200010C0B3000EC1020058
:100E80000000000039009000C9009000610040009F
:100E9000E0804800B0049800C1049800A0C0B300EE
:100EA000FDF4B7001ED5020000000000C08C9800C1
:100EB000D18C98000C013700794890000004A10003
:100EC000F04C9800C112200010C0B3000EC1020007
:100ED0000000000008007800FDF4B70002013700B0
:100EE000794890000014A000F04C980079489000D8
:100EF0000024A100F04C9800794890000004A00064
:100F0000F04C9800AF0AB00060F52F000084470055
:100F100054000900391C7800A80AB100A90AB100E0
:100F2000127802000000000088077800E8790200CB
:100F300000000000FC74EF00E115200010C0B300B9
:100F400094C00200000000008125200010C0B30002
:100F50000EC1020000000000C242E200090035009C
:100F60006000B80090049800A1049800803E200022
:100F700001002000B0049800C104980020C0B30014
:100F8000CE00370049289000D92890001C00370077
:100F9000C242E20009003D006000B80090049800E1
:100FA000A1049800803E200001002000B0049800B9
:100FB000C104980030C0B300C00037001901900090
:100FC000A901900039009000C9009000800F5100E5
:100FD000818F5900C4003A001D00370019019000AC
:100FE000A901900039009000C9009000800F5100C5
:100FF000818F5900BC003A00004B20000100200006
:1010000090049800A10498006000B800B004980013
:10101000C104980040C0B300A8003700C242E200FB
:10102000060035006000B80090049800A104980004
:101030000900780076FE0700AB0037001900900029
:10104000A9009000E00F5000E08F5800A6003A0081
:1010500009007800F1FD0700A3003700C2A7800057
:1010600019009000A90090008000510001003B0091
:101070008100EA00B0122000808F500006003C0082
:10108000E115200010C0B30094C002000000000071
:10109000C11220001500370019009000A90090002F
:1010A0008000510001003B008100EA00C0122000D6
:1010B000808F50001100340019009000A9009000AA
:1010C0008000510001003B008100EA00301F200039
:1010D000808F500009003C00E115200010C0B300D3
:1010E00094C0020000000000211C200010C0B300CA
:1010F0000EC10200000000000C0037001900900033
:10110000A90090008000510001003B008100EA002E
:10111000401F2000808F500004003400E1152000A3
:1011200010C0B30094C0020000000000190190003C
:10113000A901900039009000C9009000800F510073
:10114000818F590068003A0059209000E9209000F2
:10115000B0049800C104980080C0B3005700370065
:10116000C2A7800019009000A900900080005100E3
:1011700001003B008100EA00B0122000808F500087
:1011800006003C00E115200010C0B30094C002002E
:1011900000000000C1122000230037001900900059
:1011A000A90090008000510001003B008100EA008E
:1011B000C0122000808F50000E00340019009000F3
:1011C000A90090008000510001003B008100EA006E
:1011D000301F2000808F500006003C00E1152000E9
:1011E00010C0B30094C0020000000000211C2000C9
:1011F0000D00370019009000A900900080005100F8
:1012000001003B008100EA00401F2000808F500059
:101210002C003400E115200010C0B30094C002007F
:10122000000000008125200010C0B3000EC10200A4
:1012300000000000230037001ED50200000000005F
:1012400029299000B929900002005000838058009D
:10125000E270220073002000820F5000838F58003C
:10126000210036008125200010C0B3000EC102000D
:1012700000000000E0C0B300100037001ED50200DF
:101280000000000029299000B929900002005000B8
:1012900083805800E270220073002000820F50000B
:1012A000838F5800100036008125200010C0B30045
:1012B0000EC102000000000000C1B300FDF4B70041
:1012C0000900370019019000A90190003900900031
:1012D000C9009000800F5100818F590002003A0030
:1012E0000900780067FD07004F04BE000080FA0087
:1012F000000006000000EB009414AB0002003A006E
:101300009414A800100020000000060014D5BF00AF
:10131000E14F400003003200E097020000000000AF
:1013200014F5EF0070002000B0A888009414A90004
:1013300094D4BF000000D1006100600000000600EE
:10134000889FBE000004780081447800C1492100D4
:1013500052940200000000000000E000040032008F
:101360009434A80070002000B0A888000600370060
:1013700058A5880040A58800B0A88800090078001A
:10138000A6F4B7009434A9004F04BE000000060084
:10139000889FBE008A9FBE008C1F780000057800E1
:1013A0008045E80000067800010037008B45E80022
:1013B0003C4478000804E0000C003200E0C2B300B6
:1013C000804F5400090032000040E800804F540074
:1013D0000600320063405000804F5400030032008A
:1013E00072404000804F5400F0FF3A000AC05500A0
:1013F0008044E90009407800FA99020000000000EA
:101400008980FB000A007800209A0200000000009A
:10141000000045000005E8000804E0000900320073
:10142000F0C2B300804F5400060032006340500009
:10143000804F54000300320072404000804F54003F
:10144000DAFF3A000040EB00FA99020000000000C9
:101450004F0678004F05BE004F04BE000000060096
:101460000200FA000F80E900D69A02000000000096
:101470000000E000120032006FF997008281FB004B
:1014800083007800010CB200000C2000808F500017
:1014900004003A000F80E900D69A02000000000024
:1014A000070037000204E0000500320083007800E6
:1014B0000000EB00FA9A020000000000E9FF37008C
:1014C0000080FA00000006001A00FA00889FBE00A3
:1014D0008A9FBE0080057800B0A88000E30F50000E
:1014E0004800320004003E00E10F50000C003200C2
:1014F00015003E0008003700E50F50009000320054
:101500004C003900E60F5000B9013200E70F5000DF
:1015100006023A00A10137009674EF009574EF00BF
:10152000E09F200010B80200000000009674EC005C
:101530001ED5020000000000C0A48800D1A48800CD
:1015400020002000F8013700014A2100E09F200020
:10155000E8B60200000000000000E00013003A00BE
:101560001ED5020000000000C2A48000D3A48000A9
:101570000200500083805800A2252600230020008E
:10158000820F5000838F5800E80136006100200070
:101590006049210022C0B300904F110001003E00BD
:1015A00011002000B1A88800E0013700E19F200071
:1015B000914078008180FB00FFC9BF004800DD003A
:1015C0000101700001A02000914078008180FB00A3
:1015D00001CABF004800DD008101700002007800F0
:1015E0009CF4B7004810DE009DF4B70003007800BB
:1015F0009EF4B7004818DE009FF4B70030002000CA
:10160000B0A88800540320008001EB0042C0B30062
:10161000C0492100010020001298020000000000D3
:1016200014F5B700E14F4000C00132004000200037
:10163000B0A8880014D5BF00D099020000000000B7
:101640000000E000B90132003035EC0031D5BF00B8
:10165000FA9902000000000030D5BF00FA9902009C
:101660000000000010C0B300FA9902000000000062
:101670000040EB00FA990200000000000040EB007F
:10168000FA9902000000000010C0B300FA990200AD
:10169000000000000040EB00FA990200000000008A
:1016A0000040EB00FA990200000000000040EB004F
:1016B000FA990200000000000040EB00FA990200D5
:1016C000000000000040EB00FA990200000000005A
:1016D0000040EB00FA9902000000000050A58000D5
:1016E0000000E00001003A0040A5800028FF07004C
:1016F0000040EB00FA99020000000000A6D4BF00F1
:10170000FA990200000000000040EB00FA99020084
:101710000000000010C0B300FA99020000000000B1
:10172000629A0200000000001ED5020000000000C6
:10173000C0A48800D1A48800500020007A0137009E
:1017400014D5BF00BA9A020000000000000478001F
:101750000000E0000F003A001ED50200000000006B
:10176000C2A48000D3A480000200500083805800EF
:10177000A225260023002000820F5000838F5800EE
:101780006A01360060002000B0A8880008007800D8
:10179000670137007484570073805700D69A02009F
:1017A0000000000008007800D69A02000000000047
:1017B00080A98000980F100003003200229B0200D5
:1017C000000000005901370071805700D69A0200CE
:1017D0000000000072805700D69A0200000000004E
:1017E0006F805700D69A02000000000070805700FA
:1017F000D69A0200000000006D805700D69A0200C1
:10180000000000006E805700D69A02000000000021
:101810006B805700D69A0200000000006C805700D1
:10182000D69A02000000000069805700D69A020094
:10183000000000006A8057000E00370008FF070014
:1018400000FE2F00808447007F8457000800780046
:10185000D69A02000000000009007800D69A020023
:101860000000000008007800D69A02000000000086
:1018700009007800D69A0200000000000FB8970017
:101880000000E90080BF9F00E10F4000EBFF3A003D
:1018900034003700F2FE07007E8457007D80570039
:1018A000D69A02000000000008007800D69A0200D4
:1018B000000000007B805700D69A02000000000064
:1018C0007C8557000A007800D69A020000000000CC
:1018D00077805700D69A02000000000078805700F9
:1018E000D69A02000000000079805700D69A0200C4
:1018F0000000000064004400D69A020000000000CE
:1019000075805700D69A020000000000F684570048
:1019100009007800D69A02000000000012002000A2
:10192000980F11000A003A009A0F110008003A00BF
:1019300040002000990F100005003A0073003700A6
:10194000E0FD2F000F004000D69A020000000000CA
:101950005FB097000000E900D0B79F00E10F4000A2
:10196000F7FF3A001FB897000000E90090BF9F0002
:10197000E10F4000C7FF3A0034003700B8FE07000F
:101980007E8457007D805700D69A02000000000038
:1019900008007800D69A0200000000007B80570003
:1019A000D69A0200000000007C8557000A007800EB
:1019B000D69A02000000000077805700D69A0200F5
:1019C0000000000078805700D69A02000000000056
:1019D00079805700D69A020000000000640044009D
:1019E000D69A02000000000075805700D69A0200C7
:1019F00000000000F684570009007800D69A020023
:101A00000000000012002000980F11000A003A00A8
:101A10009A0F110008003A0040002000990F1000B2
:101A200005003A0039003700E0FD2F000F004000AC
:101A3000D69A0200000000005FB097000000E900A5
:101A4000D0B79F00E10F4000F7FF3A002FB8970092
:101A50000000E900A0BF9F00E10F4000C7FF3A006F
:101A6000410037007EFE07007E8457007D805700CE
:101A7000D69A02000000000008007800D69A020002
:101A8000000000007B805700D69A02000000000092
:101A90007C8557000A007800D69A020000000000FA
:101AA00077805700D69A0200000000007880570027
:101AB000D69A02000000000079805700D69A0200F2
:101AC0000000000064004400D69A020000000000FC
:101AD00075805700D69A020000000000F684570077
:101AE00009007800D69A02000000000012002000D1
:101AF000980F110017003A009A0F110015003A00D4
:101B000040002000990F100012003A009434A80001
:101B1000C0492100D69A020000000000D0492100EF
:101B2000D69A020000000000E0492100D69A020087
:101B300000000000F0492100D69A020000000000D9
:101B40000E003700E0FD2F000F004000D69A020083
:101B5000000000005FB097000000E900D0B79F00D0
:101B6000E10F4000F7FF3A003FB897000000E9009E
:101B7000B0BF9F00E10F4000BAFF3A00229B020075
:101B80000000000014D5BF00E09702000000000034
:101B900014F5EF0070002000B0A8880094D4BF00B6
:101BA0006240600004003A009CF4B7009DF4B70066
